:020000020000FC
:032000000230406B
:032003000221D5E2
:01200B0032A2
:032013000221FDAA
:01201B003292
:0320230002204454
:03202B0002223757
:10202E00210901A101E52106212721342118213F93
:10203E004113617501E1C0D0C0E020980820992BB2
:10204E00D0E0D0D032C298E51604B51707E599D086
:10205E00E0D0D032F516C082C083758381F582E55B
:10206E0099F0D083D082D0E0D0D032C299E528B595
:10207E002707C21DD0E0D0D03204F528C082C0831D
:10208E00758382F582E0F599D083D082D21DD0E09F
:10209E00D0D032C0D0C8C0E0752B00C2AF201D0911
:1020AE00D299E4F527F528D21DE52704B5280AD2E2
:1020BE00AF052BE52B70E480E7F527C083C0827552
:1020CE008382F582C8F0D082D083D2AFC8D0E0C868
:1020DE00D0D022201DFD22C2ACE517B51605E4D2E4
:1020EE00ACD32204F517C082C083F582758381E0DC
:1020FE00D083D082D2ACC3223108C4C0E0540F24A6
:10210E0090D43440D411A1D0E022C0E0740D12203E
:10211E00A1740A1220A1D0E022C0E0E5833106E5C9
:10212E00823106D0E022E493A360051220A180F64E
:10213E00227800D8FED8FEC2AF43878053890F4362
:10214E008920C28EC28F74FEF58DF58B75985075F1
:10215E002700752800C21DD28ED2ACD2AF22E490D9
:10216E00FF5DF0E51EB51D0F74FFF51EF51DD0E0E9
:10217E00D083D082D0D03204B43C01E4F51E2323A8
:10218E002400F582E43483F583E0FAA3E0FBA3E0B8
:10219E00FCA3E0FD90FF12EAF0A3EBF090FF28E421
:1021AE00F0A37490F090FF2AECF0A3EDF0E490FF12
:1021BE0059F0908004E02401F0A3E03400F0D0E068
:1021CE00D083D082D0D032C0D0C082C083C0E07560
:1021DE00D00890FF50E020E185D0E0D083D082D0AF
:1021EE00D03290FF5CF0D0E0D083D082D0D032C01D
:1021FE00D0C082C08375D008FF90FF6EE0EFD08311
:10220E00D082D0D032C2AD75C80075CA0075CBD0A1
:10221E0075CC0075CDD0C215C216C217C21875295D
:10222E0000752A00D2ADD2CA22C0D075D008FFAE3A
:10223E0082AD83C2CFC29400D2940020960D301787
:10224E0002800AD217740371758002C217C295D22A
:10225E009520960D301602800AD216740271758082
:10226E0002C216C295D29520960D301802800AD25F
:10227E0018740471758002C218C295D295209614F6
:10228E00052AE52A14600724F4500C752A017406F9
:10229E0071758003752A00C295D29520960D301562
:1022AE0002800AD215740171758002C215C295D2D0
:1022BE00952096140529E52914600724F4500C7511
:1022CE002901740571758003752900908023E0241F
:1022DE00FC40062405F002236DE4F03019189080BE
:1022EE0024E024FFF0F8A3E034FFF07009E8700654
:1022FE00C219740A7175301A18908026E024FFF006
:10230E00F8A3E034FFF07009E87006C21A740B717E
:10231E0075301B18908028E024FFF0F8A3E034FFFE
:10232E00F07009E87006C21B740C7175301C1890A1
:10233E00802AE024FFF0F8A3E034FFF07009E87083
:10234E0006C21C740D717590802CE02401F0500FA4
:10235E00A3E03400F0A3E03400F0A3E03400F08DED
:10236E00838E82EFD0D032F8E51004B44001E4B58C
:0F237E00110122F51024C0F582758380E8F0224A
:020000020000FC
:10300000A5E5E0A523FF000000000000000000008F
:10301000000000000000000000000000FFFFFFFFB4
:103020004D503320506C617965722C2056657220AA
:08303000302E362E332E340041
:10CF0000A5E5E0A5FD000000000000000000000015
:10CF1000000000000000000000000000FFFFFFFF15
:0BCF20004175746F2D53746172740032
:04CF40000230382261
:0430400002A0863232
:01304B003252
:01305300324A
:01305B003242
:01306300323A
:01306B003232
:0DA086007581A0129DA0E582600302307379
:03A10000023073B7
:1030730012307880FE90101D74FFF0901019E4F068
:10308300A3F0A3F0A3F0901019C201C2049041CDA4
:103093001244FA9042771244FA124782AA82BA0083
:1030A30002800312451512451D9012EBE4F0124500
:1030B3002090429A124CA29042BD124CA212452972
:1030C300AA82EA60F812624212693512461DAA8288
:1030D300BA0003124515126C54C203C21F12455B9A
:1030E3001278989042E2124CA2904305124CA2121D
:1030F3008D3812455B904333124CA21285379013DF
:1031030010E0FAA3E0FBA3E0FCA3E0FD90130CEABC
:10311300F0A3EBF0A3ECF0A3EDF090130CE0FAA313
:10312300E0FBA3E0FCA3E0FDBA000CBB0009BC007C
:1031330006BD00030231958A828B838CF0ED1278F1
:1031430046AA82AB83901021EAF0A3EBF0740C2A19
:10315300F582E43BF583E0FCA3E0FDA3E0FEA3E0FE
:10316300FFBC002EBD002BBE0028BF002574082A1B
:10317300F582E43BF583E0FAA3E0FBA3E0FCA3E0E4
:10318300FD90130CEAF0A3EBF0A3ECF0A3EDF00237
:10319300311D901021E0240CFAA3E03400F5838A5A
:1031A30082E0FAA3E0FBA3E0FCA3E0FDBA001ABBB4
:1031B3000017BC0014BD0011904356124CA290435B
:1031C30079124CA2124515800E90100BEAF0A3EB76
:1031D300F0A3ECF0A3EDF0901001E4F0A3F0901055
:1031E300011295B19010C8E4F075820E12472AAA15
:1031F30082901014EAF0901015E4F0A3F0901017E9
:10320300E4F0A3F0901017EA60031240AE9010C8E8
:103213007401F075820912472AAA82901013EAF00A
:10322300BA05028003BA0203123D04C202901000E1
:103233007401F075822C125B3B90438D124CA27586
:103243008201125FA890101F7401F090101E740188
:10325300F012697E124701AA82BA00030235D9BA75
:10326300010302335FBA0202806FBA03030233A27F
:10327300BA040302346BBA05030234D1BA0603025B
:1032830034DBBA0A030234F1BA0B030234E5BA0C95
:103293000302353ABA0D03023543BA14030234E587
:1032A300BA15030234E5BA16030233E5BA1703026B
:1032B3003428BA18030234E5BA19030234E5BA1AFA
:1032C300030234E5BA1B030234E5BA1C030234E5F6
:1032D300BA51030235B30235C290101EE0FBBB06A0
:1032E300319043AC124CA290101FE0FC90101EF0E2
:1032F300C002C0031245AAD003D00290100074018B
:10330300F075822CC002C003125B3BD003D00202D3
:1033130035D98B048C82C002C003124018AC82D012
:1033230003D002EC602A9043B3124CA290101FEB1F
:10333300F090101E7406F0C0021245B0D002901037
:1033430000E4F075822CC002125B3BD0020235D937
:103353008A82C002124707D0020235D990101EE0BC
:10336300FBF582C002124018AB82D002EB602490BE
:1033730043BB124CA2C0021245B6D002C002124592
:103383002FD002C002123D04D00290101E7405F02B
:103393000235D98A82C002124707D0020235D9907A
:1033A300101EE0FBF582C002124018AB82D002EB84
:1033B30060249043C7124CA2C0021245B6D002C08B
:1033C3000212452FD002C002123E98D00290101E66
:1033D3007405F00235D98A82C002124707D002026F
:1033E30035D990101EE0FBF582C002124018AB8263
:1033F300D002EB60249043D7124CA2C0021245B610
:10340300D002C00212452FD002C0021239A6D00248
:1034130090101E7405F00235D98A82C00212470744
:10342300D0020235D990101EE0FBF582C002124093
:1034330018AB82D002EB60249043E8124CA2C00286
:103443001245B6D002C00212452FD002C002123B71
:103453005FD00290101E7405F00235D98A82C00233
:10346300124707D0020235D9901013E0FBBB0508C1
:103473009010137401F080310B901013EBF0BB012B
:10348300028003BB03089043FD124CA280069044C4
:103493000A124CA2C0021296C2D002C0021296C2F5
:1034A300D002C0021296C2D002D20275822BC00291
:1034B300125B3BD0029010D07464F0A3E4F0901040
:1034C300D0758203C00212474CD0020235D9C00224
:1034D300126E23D0020235D9C002126E66D00202E8
:1034E30035D98A82C002124EC1D0020235D990105A
:1034F300D07405F0A3E4F09010D0758200C00212DE
:10350300474CD002758200C002125453D002758218
:1035130000C0021256E3D00290101EE0FBBB030270
:103523008008BB040280030235D9758200C00212F1
:1035330059AED0020235D9904416124CA20235D9A5
:10354300904426124CA2300309C002126D8FD002A0
:10355300C20330021B901013E0FB7880A603901087
:10356300C97480F0758209C002124719D002C202E1
:10357300300109C00212961AD002C20120040302CC
:1035830035D990101DE0FB90100FE0FCA3E0FDA3E4
:10359300E0FEA3E0FF90146DECF0A3EDF0A3EEF0DA
:1035A300A3EFF08B82C0021296F0D002C2048026F1
:1035B300EA24B0FBF582C00212636BD00280177B52
:1035C30000C002C0037436C0E07444C0E01249AACC
:1035D300E58124FCF58175820612453590101EE0C5
:1035E300FAC364809481500302395AC374868AF003
:1035F30063F08095F0500302395A1AEA25E02A90C5
:103603003606730236180237650237CF02384D0289
:10361300387A0238EA90130CE0FAA3E0FBA3E0FC4B
:10362300A3E0FD8A828B838CF0127846E0FAA3E054
:10363300FBA3E0FCA3E0FD8A828B838CF012785F0E
:10364300AA82AB8312556390100BE0FAA3E0FBA3AD
:10365300E0FCA3E0FD8A828B838CF0127846E0FACB
:10366300A3E0FBA3E0FCA3E0FD8A828B838CF01232
:10367300785FAA82AB83901023EAF0A3EBF0C00239
:10368300C0031257F3D003D002740D2AF582E43B32
:10369300F583E0FCA3E0FDA3E0FEA3E0FF8C828DB5
:1036A300838EF0127846AC82AD83C002C0031252FF
:1036B30090D003D00274052AF582E43BF583E0FC45
:1036C300A3E0FDA3E0FEA3E0FF8C828D838EF0C018
:1036D30002C003124629AC82D003D00290101DEC25
:1036E300F074092AF582E43BF583E0FAA3E0FBA337
:1036F300E0FDA3E0FE9010B1E4F0A3F0A3F0A3F08B
:103703009010B5EAF0A3EBF0A3EDF0A3EEF08C82FA
:10371300C004124636D00490101E7402F09010209C
:10372300E4F0AA81EA3395E0FBEC3395E0FDC002B7
:10373300C003C004C0057454C0E07444C0E012491F
:1037430097E58124FAF581127468AA82AB83ACF001
:10375300FD901019EAF0A3EBF0A3ECF0A3EDF00257
:103763003254AA81EA3395E0FB90101DE0FCFD334F
:1037730095E0FEC004C002C003C005C0067470C05B
:10378300E07444C0E0124997E58124FAF581D0043E
:103793008C82C00412465BD004901020E02401F018
:1037A300FAC374868AF063F08095F04003023254C2
:1037B3009010C1E4F0A3F0A3F0A3F09010C18C82A9
:1037C30012466390101E7403F002325490101DE0F1
:1037D300FAFB3395E0FCC002C003C004748AC0E066
:1037E3007444C0E0124997E58124FCF581D0028A34
:1037F3008212465BAA82EA700302384D90101E744F
:1038030004F012453D901023E02409FAA3E03400AC
:10381300F5838A82E0FAA3E0FBA3E0FCA3E0FD903A
:10382300100FEAF0A3EBF0A3ECF0A3EDF0D20475D4
:1038330082031247649010D07432F0A3E4F0901026
:10384300D075820312474C1246CB74A9C0E074446E
:10385300C0E01249971581158190101DE0FAF58299
:10386300124039AA82BA0003023254123D04901066
:103873001E7405F00232541245BCAA827B00C002BA
:10388300C00374B5C0E07444C0E0124997E58124D5
:10389300FCF5811245C2AA82EA6031124549AA8227
:1038A300EA602990101DE0FAF58212469E1246CB7B
:1038B30012455B124543AA82EA600B124523124567
:1038C30029AA82EA60F890101E7401F0127468AAA3
:1038D30082AB83ACF0FD901019EAF0A3EBF0A3ECFC
:1038E300F0A3EDF002325490101FE0FABA03028005
:1038F3000302325490101DE0FAF58212465BAA824D
:10390300EA700302325490101F7404F012453D9084
:103913001023E02409FAA3E03400F5838A82E0FA55
:10392300A3E0FBA3E0FCA3E0FD90100FEAF0A3EB00
:10393300F0A3ECF0A3EDF0D2047582031247649078
:1039430010D07432F0A3E4F09010D07582031247C4
:103953004C1246CB0232549044CC124CA290101E0F
:10396300E0FA3395E0FB8A82F583124CEC124D2684
:1039730002325422E582901094F0D2019010D07458
:1039830064F0A3E4F09010D075820312474C9010BA
:1039930094E0FABA01091296C2AA82AB8380031299
:1039A300969022901013E0FABA0502800D9010133E
:1039B300E0FABA04028003023A20758201123977D1
:1039C300AA82AB83901097EAF0A3EBF0901433E054
:1039D300FCA3E0FDC3EC9AED9B4003023A2C901448
:1039E30033E0FAA3E0FB901097E0FCA3E0FD901412
:1039F300B1EAF0A3EBF08C828D83129F31AA82ABE4
:103A030083901097EAF0A3EBF0BA001DBB001A9065
:103A130010977401F0A3E4F0901097800C90109726
:103A23007401F0A3E4F090109790130CE0FAA3E074
:103A3300FBA3E0FCA3E0FD8A828B838CF012784623
:103A4300AA82AB83901095EAF0A3EBF074082AF5F1
:103A530082E43BF583E0FAA3E0FBA3E0FCA3E0FDF3
:103A6300BA000CBB0009BC0006BD0003023AAA90D1
:103A73001095E02408FAA3E03400F5838A82E0FA83
:103A8300A3E0FBA3E0FCA3E0FD90130CEAF0A3EB9F
:103A9300F0A3ECF0A3EDF0901015E0FA2401F0A3ED
:103AA300E0FB3400F08026901310E0FAA3E0FBA3C0
:103AB300E0FCA3E0FD90130CEAF0A3EBF0A3ECF021
:103AC300A3EDF0901015E4F0A3F090101590130CF3
:103AD300E0FAA3E0FBA3E0FCA3E0FD8A828B838CE6
:103AE300F0127846AA82AB83740C2AF582E43BF584
:103AF30083E0FAA3E0FBA3E0FCA3E0FD90100BEA54
:103B0300F0A3EBF0A3ECF0A3EDF0901017E4F0A317
:103B1300F0901017BA0025BB0022BC001FBD001C8B
:103B2300901097E0FA2401F0A3E0FB3400F090102A
:103B330015E024FFF0FAA3E034FFF0FB901097E0C8
:103B430024FFF0FAA3E034FFF0FBEA4B6003023AF0
:103B53002C901014E0FA600312416A22901013E0D3
:103B6300FABA0502800D901013E0FABA040280033A
:103B7300023BD97582FF123977AA82AB8390109BDF
:103B8300EAF0A3EBF0901433E0FCA3E0FDC3EC9A5E
:103B9300ED9B4003023BE5901433E0FAA3E0FB9076
:103BA300109BE0FCA3E0FD9014B1EAF0A3EBF08CD2
:103BB300828D83129F31AA82AB8390109BEAF0A37C
:103BC300EBF0BA001DBB001A90109B7401F0A3E444
:103BD300F090109B800C90109B7401F0A3E4F09084
:103BE300109B90130CE0FAA3E0FBA3E0FCA3E0FD21
:103BF3008A828B838CF0127846AA82AB83901099C9
:103C0300EAF0A3EBF074042AF582E43BF583E0FACF
:103C1300A3E0FBA3E0FCA3E0FDBA000CBB0009BCDE
:103C23000006BD0003023C63901099E02404FAA34C
:103C3300E03400F5838A82E0FAA3E0FBA3E0FCA36F
:103C4300E0FD90130CEAF0A3EBF0A3ECF0A3EDF08E
:103C5300901015E024FFF0FAA3E034FFF0FB801C82
:103C6300901314E0FAA3E0FBA3E0FCA3E0FD9013A0
:103C73000CEAF0A3EBF0A3ECF0A3EDF090130CE04F
:103C8300FAA3E0FBA3E0FCA3E0FD8A828B838CF024
:103C9300127846AA82AB83740C2AF582E43BF5833F
:103CA300E0FAA3E0FBA3E0FCA3E0FD90100BEAF035
:103CB300A3EBF0A3ECF0A3EDF0BA0025BB0022BC0C
:103CC300001FBD001C90109BE0FA2401F0A3E0FB51
:103CD3003400F0901015E0FA2401F0A3E0FB340067
:103CE300F090109BE024FFF0FAA3E034FFF0FBEA2E
:103CF3004B6003023BE5901014E0FA600312416A43
:103D03002290130CE0FAA3E0FBA3E0FCA3E0FD8AFE
:103D1300828B838CF0127846AA82AB8390109FEA41
:103D2300F0A3EBF0901013E0FABA0502800D9010A7
:103D330013E0FABA02028003023DA175820112392F
:103D430077AA82AB8390109DEAF0A3EBF090142D39
:103D5300E0FCA3E0FDC3EC9AED9B4003023DAD9074
:103D6300142DE0FAA3E0FB90109DE0FCA3E0FD908E
:103D730014B1EAF0A3EBF08C828D83129F31AA82F7
:103D8300AB8390109DEAF0A3EBF0BA001DBB001AC1
:103D930090109D7401F0A3E4F090109D800C90109E
:103DA3009D7401F0A3E4F090109D90100BE0FAA332
:103DB300E0FBA3E0FCA3E0FD8A828B838CF0127806
:103DC3005FAA82AB839010A1EAF0A3EBF074082AF8
:103DD300F582E43BF583E0FAA3E0FBA3E0FCA3E078
:103DE300FDBA000BBB0008BC0005BD000280030246
:103DF3003E42901013E0FABA01028008901013E0DB
:103E0300FABA023590109FE0240CFAA3E03400F5CF
:103E1300838A82E0FAA3E0FBA3E0FCA3E0FD901019
:103E23000BEAF0A3EBF0A3ECF0A3EDF0901017E492
:103E3300F0A3F0901017023E781239A6023E789054
:103E430010A1E02408FAA3E03400F5838A82E0FAA3
:103E5300A3E0FBA3E0FCA3E0FD90100BEAF0A3EBCF
:103E6300F0A3ECF0A3EDF0901017E0FA2401F0A317
:103E7300E0FB3400F090109DE024FFF0FAA3E0345F
:103E8300FFF0FBEA4B6003023DAD901014E0FA60D3
:103E93000312416A2290130CE0FAA3E0FBA3E0FCB7
:103EA300A3E0FD8A828B838CF0127846AA82AB83CF
:103EB3009010A3EAF0A3EBF0901013E0FABA050216
:103EC300800D901013E0FABA02028003023F3575A9
:103ED30082FF123977AA82AB839010A7EAF0A3EB93
:103EE300F090142DE0FCA3E0FDC3EC9AED9B40039E
:103EF300023F4190142DE0FAA3E0FB9010A7E0FCF1
:103F0300A3E0FD9014B1EAF0A3EBF08C828D831251
:103F13009F31AA82AB839010A7EAF0A3EBF0BA001B
:103F23001DBB001A9010A77401F0A3E4F09010A732
:103F3300800C9010A77401F0A3E4F09010A79010E8
:103F43000BE0FAA3E0FBA3E0FCA3E0FD8A828B83F2
:103F53008CF012785FAA82AB839010A5EAF0A3EBF2
:103F6300F074042AF582E43BF583E0FAA3E0FBA3B3
:103F7300E0FCA3E0FDBA000BBB0008BC0005BD00DC
:103F8300028003023FCC901013E0FABA01028008CA
:103F9300901013E0FABA022B9010A3E02410FAA3B6
:103FA300E03400F5838A82E0FAA3E0FBA3E0FCA3FC
:103FB300E0FD90100BEAF0A3EBF0A3ECF0A3EDF01F
:103FC300024002123B5F0240029010A5E02404FA73
:103FD300A3E03400F5838A82E0FAA3E0FBA3E0FCCC
:103FE300A3E0FD90100BEAF0A3EBF0A3ECF0A3ED3C
:103FF300F0901017E024FFF0FAA3E034FFF0FB90F9
:1040030010A7E024FFF0FAA3E034FFF0FBEA4B60D3
:1040130003023F4122E5829010A9F09010A9E0FA33
:10402300BA04028008BA03028003BA050575820147
:10403300800375820022E5829010AAF09010AAE016
:10404300FAC0021245BCAB82D002EB605A8A82C02E
:1040530002124696AB82AC83D002C002C003C004F6
:10406300C003C00474DBC0E07444C0E0124997E5A8
:104073008124FCF581D004D003D002BB0005BC0031
:10408300028024BBFF05BCFF0280179010CAE4F036
:10409300A37410F08B828C83C002124598D0020265
:1040A30040447582018003758200229010C8E4F0B9
:1040B30075820A12472AAA829010C8E4F075820B0F
:1040C300C00212472AAB82D0028A04E4FAFDEB2A2B
:1040D300FBED3CFA9010137403F0901014E4F0C35A
:1040E300E49BE49A50257C017D00C3EB9CEA9D4050
:1040F3001AC002C003C004C0051239A6D005D004FB
:10410300D003D0020CBC00E20D80DF9010C8E4F0B5
:1041130075820C12472AAA829010C8E4F075820DAA
:10412300C00212472AAB82D0028A04E4FAFDEB2ACA
:10413300FBED3CFAC3E49BE49A50257C017D00C36C
:10414300EB9CEA9D401AC002C003C004C005123DA7
:1041530004D005D004D003D0020CBC00E20D80DFF4
:104163009010147401F022901015E0FAA3E0FBFC08
:104173007D007B007880A6029010C97480F0758260
:104183000BC004124719D0047880A6049010C97498
:1041930080F075820A124719901017E0FAA3E0FB2A
:1041A300FC7D007B007880A6029010C97480F075B6
:1041B300820DC004124719D0047880A6049010C958
:1041C3007480F075820C124719220D0A0D0A5C5B8C
:1041D3005C41305C402130504A5243204D503320E3
:1041E300506C6179657220302E362E332E34205C6C
:1041F3005D0D0A4D503320506C617965722C205649
:10420300657273696F6E20302E362E332E3420285C
:10421300435653292C2041756775737420322C2023
:10422300323030310D0A436F7079726967687420D8
:1042330028432920323030312C20504A52432E4318
:104243004F4D2C204C4C430D0A0D0A5479706520B8
:1042530027515549542720746F2072657475726E07
:1042630020746F20746865206D6F6E69746F720DB2
:104273000A0D0A005C5B5C422027455850455249B1
:104283004D454E54414C204445562052454C4541E2
:1042930053455C5D0D0A005C5B5C422021576169FC
:1042A30074696E6720666F7220486172642044727D
:1042B30069766520205C5D0D0A0057616974696E3B
:1042C3006720666F72204861726420447269766564
:1042D30020746F2062652072656164790D0A005C49
:1042E3005B5C4220215363616E6E696E6720646973
:1042F300726563746F72696573202020205C5D0DA5
:104303000A004275696C64696E6720506C61796C50
:104313006973742873293A205363616E20416C6C6E
:10432300204469726563746F726965733A0D0A009C
:104333005C5B5C4220224275696C64696E67204D48
:10434300335520706C61796C6973747320205C5DE4
:104353000D0A005C5B5C4220222020202D204E6F42
:104363002066696C657320666F756E64202D20204E
:10437300205C5D0D0A004E6F2066696C65732066D4
:104383006F756E642E2E2E0D0A000D0A4D503320CC
:10439300506C617965722C20426567696E20506CA0
:1043A30061796261636B0D0A00506C61790D0A00DB
:1043B30050617573650D0A004E6578742046696C0B
:1043C300650D0A0050726576696F75732046696CD6
:1043D300650D0A004E65787420506C6179204C6934
:1043E30073740D0A0050726576696F757320506C93
:1043F3006179204C6973740D0A0052616E646F6DAC
:10440300204F66660D0A0052616E646F6D204F6E19
:104413000D0A0054696D65722032204576656E740D
:104423000D0A0054696D65722033204576656E74FC
:104433000D0A000D0A0D0A556E737570706F727454
:104443006564206576656E74202325640D0A0D0A64
:1044530000535F524541445F4449522C206D7033F1
:104463005F66643D2568642025780D0A00535F4329
:10447300414348494E472C206D70335F66643D25A8
:10448300642025780D0A00535F504C4159494E472B
:104493005F43414348494E472C206D70335F666448
:1044A3003D25640D0A00535F504C4159494E470D59
:1044B3000A00535F46494E4953485F504C4159499E
:1044C3004E472C20713D0D0A00494C4C4547414C49
:1044D3002053544154453A004652422C20723D2504
:1044E300780D0A00E582020030120032F58222E5DF
:1044F30082020034020036020038E582120040F5E1
:104503008222E58202004DE582020050020053023E
:104513000048122042C2AF02006D02203C02203E3E
:10452300903052020FE0903055020FE09030580265
:104533000FE0AA8290305B020FE090305E020FE042
:10454300903061020FE0903064020FE09030670218
:104553000FE090306A020FE090306D020FE0AA8204
:10456300AB839010ACE0C4540F232400F582E434F1
:10457300FFF583EAF0A3EBF022AA82903073020FD7
:10458300E0AA82AB83903076020FE0AA82AB8390DD
:104593003079020FE0AA82AB839010CAE0FCA3E05B
:1045A300FD90307C020FE090307F020FE09030826C
:1045B300020FE0903085020FE0903088020FE09008
:1045C300308B020FE09030D0020FE0903043020FA7
:1045D300E0AC8290304C120FE0C0E09010ADE0FAF6
:1045E300A3E0F5838A82EBF0D08222AC829010AFF5
:1045F300E0FBA3E0F5838B82E0FB90304F020FE0FA
:104603009030E2020FE090308E020FE0AB829030E8
:1046130091020FE0903094020FE0903097020FE088
:104623009030D3020FE0AA82AB83ACF0FD90309AB6
:10463300020FE08582F09010B1E0F8A3E0F9A3E067
:10464300FAA3E0FB9010B5E0FCA3E0FDA3E0FEA31A
:10465300E0FF90309D020FE0AC829030A0020FE0AB
:10466300AE829010C1E0FAA3E0FBA3E0FCA3E0FD5F
:104673009030A3020FE0AC829030BE020FE0AC8218
:104683009010C5E0FEA3E0FF9010C7E0F99030A6BC
:10469300020FE0AC829030A9020FE0AC829030AC04
:1046A300020FE08582F09010B9E0F8A3E0F9A3E0EF
:1046B300FAA3E0FB9010BDE0FCA3E0FDA3E0FEA3A2
:1046C300E0FF9030C1020FE09030AF020FE0AC8208
:1046D3009010CCE0FEA3E0FF9030B2020FE0AC827A
:1046E3009010CEE0FEA3E0FF9030E5020FE0AC8235
:1046F300AD839030E8020FE09030B5020FE09030C8
:10470300B8020FE0AC829030BB020FE0E582C2AF8B
:10471300122040D2AF22AA829010C9E0F89030C490
:10472300020FE075820122AA829010C8E0F890304F
:10473300C7020FE0903049020FE0903046020FE0CD
:1047430002F0409030CD020FE0AC829010D0E0FA3E
:10475300A3E0FB9030D6020FE0AC829030D9020F79
:10476300E0AC829030DC020FE09030DF020FE00219
:104773002042AC829010D2E0FE9030EB020FE012A8
:1047830047467A00BA0A0040030248459048981207
:1047930044FAC002124737AB82D002BB0002800941
:1047A3009048BF1244FA0248419048C81244FABAEA
:1047B300000D9048CD1244FAC002124523D002C026
:1047C30002124555AB82D002BB00139048E4124459
:1047D300FAC002124849D002758201024848904843
:1047E300FA1244FAC0021245CEAB82D002BB0002D9
:1047F30080089049201244FA80449049291244FACF
:10480300C002124617AB82D002BB003290492E126F
:1048130044FAC00212454FAB82D002BB0002800CA7
:10482300C002124849D0027582018019C0021245A4
:10483300C8D00290494A1244FA75820080070A02DE
:1048430047877582012212485BAA82BA0009904900
:10485300651244FA1247432290F000E493B4A53062
:10486300A3E493B4E52AA3E493B4E024A3E493B4C8
:10487300A51EA3E493B4231890F030E493B430104E
:10488300A3E493B42E0AA3E493B431047582002203
:104893007582012222436F6E6669677572696E675E
:1048A3002058696C696E78205843533130584C2036
:1048B3004650474120436869703A20004572726F41
:1048C30072210D0A004F4B0D0A005265736574691E
:1048D3006E672049444520446576696365730D0A14
:1048E30000426164206F72204D697373696E6720A3
:1048F30053494D4D0D0A00436F6E666967757269C2
:104903006E6720535441303133204D50332044657A
:10491300636F64657220436869703A200045727260
:104923006F72210D0A004F4B0D0A00496E697469BD
:10493300616C697A65204D656D6F7279204D616E8A
:10494300616765720D0A0068617264776172655F01
:10495300696E6974282920636F6D706C6574650DC9
:104963000A0052756E6E696E67204F6C642046694B
:10497300726D776172652C207468617420646F6551
:10498300736E277420757365207468652053494DD1
:104993004D0D0A00C06B85816B201F028003024905
:1049A300AF856B81D06B22C06B85816BE56B24FD7A
:1049B300F8868318868218E493A3B4255DC205C2E2
:1049C30006C207C208C209753C00E493A324C6408B
:1049D30012240A5010D209F9E53C75F00AA429F50E
:1049E3003C80E7240A2430B46C04D20580DCB4682C
:1049F30004D20680D5B47303024A27B46406124B6B
:104A030096024A81B47506124B96024AA1B4630416
:104A1300E6188008B47803024A606005124C90805F
:104A230096024C9CC083C08286F0188683188682C7
:104A330018300917C082C08312A05E6007A3153C1B
:104A4300E53C70F4124C7BD083D08212A05E6006EA
:104A5300A3124C9080F5D082D0830249BA124A78CF
:104A630020060C124A78300506124A78124A781248
:104A73004C940249BAE6124C80E618024C81ED30A0
:104A8300E71CD208E9F43401F9200612EAF43400F1
:104A9300FA30050AEBF43400FBECF43400FC200696
:104AA30010300508EB701DEC701AC205EA7015D2C0
:104AB30006E97010300905153C124C7B7430124C1A
:104AC300900249BAC082C083124BB0300960790AA0
:104AD30030051DEB54F0703619EB540F703019EAA2
:104AE30054F0702A19EA540F702419EF54F0701E11
:104AF300790520060BEF540F701419EE54F0700E65
:104B03007903EE540F700719ED54F0700119E53C69
:104B1300A208994019F53CC003C002C007C006C0F3
:104B230005124C7BD005D006D007D002D003300845
:104B330005742D124C9020064030052CC005C0068C
:104B4300C0078A82EBF583124C80E583124C81E522
:104B530082124C80E582124C81D0E0F582124C80A7
:104B6300E582D083D08280058D828E83EF124C81C3
:104B7300E583124C80E58380038D82EE124C81E540
:104B830082124C80E582124C81124C94D083D082E5
:104B93000249BAE6F9FD18200612AA01E6F918300F
:104BA300050AAC02AB01E6FA18E6F91822E9540F3C
:104BB300904D3193FDE9C4540FF9904D41932DD499
:104BC300FDE94410933400D4FE30060122EA540F69
:104BD300F9904D61932DD4FDE94410933ED4FEEA40
:104BE300C4540FF9904D81932DD4FDE94410933EA5
:104BF300D4FEE94420933400D4FF20050122EB5472
:104C03000FF9904DB1932DD4FDE94410933ED4FE9A
:104C1300E94420933FD4FFE43400FAEBC4540FF982
:104C2300904DE1932DD4FDE94410933ED4FEE94425
:104C330020933FD4FFE94430933AD4FAEC540FF96C
:104C4300904E217B00124C53ECC4540FF9904E71DB
:104C5300932DD4FDE94410933ED4FEE94420933FC1
:104C6300D4FFE94430933AD4FAE94440933BD4FB6C
:104C7300227420124C90153CE53C70F522C4540F6D
:104C8300700330070BD2072490D43440D402203071
:104C9300222007FC7430024C90856B81D06B22E498
:104CA300936006122030A380F622E06006122030C3
:104CB300A380F7742002203022D207C0E0124C8078
:104CC300D0E0124C81E5F0124C80E5F0124C81E506
:104CD30083124C80E583124C81E582124C80E5827D
:104CE300124C81742002203022D207024CD222C2FD
:104CF30007E58275F0648460072430122030D20700
:104D0300E5F075F00A847003300705243012203073
:104D1300E5F02430122030742002203022E5820294
:104D2300203022740D122030740A02203022000138
:104D330002030405060708091011121314150016BF
:104D4300324864809612284460769208244000001A
:104D530000000000000101010101010202020056EE
:104D63001268248036924804601672288440000238
:104D730005071012151720232528303335380096E0
:104D8300928884807672686460565248444000403A
:104D93008122630445862768095091327314000009
:104DA30000010102020203030404040505060036A0
:104DB3007208448016528824609632680440005575
:104DC30010662176328742985308641975300006BD
:104DD30013192632394552586572788591980076B1
:104DE3005228048056320884603612886440008555
:104DF3007157432814008671574329140086000411
:104E0300091419242934384348535863687200013C
:104E130002030405060708091011121314150016DE
:104E230032486480961228446076920824400072C7
:104E330044168860320577492193653810820077DC
:104E430055331088664421997754321088650016CB
:104E530033506783001734506784011834510000BE
:104E630000000000010101010101020202020056DB
:104E730012682480369248046016722884400054D5
:104E8300096318722781369145005409631800435A
:104E93008730741761044891357922660953006895
:104EA300360573421079471584522189582600022A
:0E4EB300050810131618212426293234374022
:10A093009012ACE4F09012ADF09012AEF0C20A90C0
:10A0A30010D3E4F0A3F09010D39010D5E4F0901106
:10A0B3006FE4F0901170E4F0A3F0901170901172BE
:10A0C300E4F090120CE4F0901294E4F0A3F09012F8
:0CA0D300949012977401F0901298E4F041
:104EC100E58290129AF09010D07450F0A3E4F09023
:104ED10010D075820112474C90129AE0FABA0B0376
:104EE10002523CBA1402801BBA1503024FD8BA1AF7
:104EF100030250C7BA1B030250B2BA1C030250DBB3
:104F0100025278901297E0FBBB0103024F87BB026C
:104F110002800BBB03028003024FCF02528F90121B
:104F210098E0FBC374089B500302528FEB25E02BE2
:104F3100904F3573024F50024F53024F56024F5953
:104F4100024F5C024F5F024F69024F73024F7D02B5
:104F5100528F02528F02528F02528F02528FC00221
:104F6100126EB1D00202528FC0021270F3D002024F
:104F7100528FC002126FD2D00202528FC00212723F
:104F81000ED00202528F901298E0FBC374059B5021
:104F91000302528FEB25E02B904F9D73024FAF021E
:104FA1004FB9024FBC024FBF024FC2024FC5C002F0
:104FB100126E23D00202528F02528F02528F02527E
:104FC1008F02528FC002126E23D00202528F9012B2
:104FD100977401F002528F901297E0FBBB0103021C
:104FE1005061BB0202800BBB030280030250A90285
:104FF100528F901298E0FBC374089B405AEB25E056
:105001002B90500673025021025024025027025067
:105011002A02502D02503002503A02504402504EA2
:1050210002528F02528F02528F02528F02528FC050
:1050310002126F44D00202528FC00212717CD00260
:1050410002528FC002127065D00202528FC002124A
:105051007297D00202528F9012977401F002528F10
:10506100901298E0FBC374059B500302528FEB250D
:10507100E02B9050777302508902509302509602B0
:10508100509902509C02509FC002126E66D00202DB
:10509100528F02528F02528F02528F02528FC002E0
:1050A100126E66D00202528F9012977401F0025272
:1050B1008F901298E0FB2401F0758200C002125F0C
:1050C100A8D00202528F901298E0FB14F075820072
:1050D100C002125FA8D00202528F901297E0FBBB70
:1050E10001030251C7BB0202805EBB0302800302BF
:1050F1005233901298E0FBC374039B500302528F0A
:10510100EB25E02B905109730251150251220251F6
:105111002F02513C758201C002125FA8D0020252D7
:105121008F758202C002124707D00202528F758228
:1051310004C002124707D00202528F758201C002D9
:10514100124707D00202528F901298E0FBC37408F5
:105151009B500302528FEB25E02B90515F7302515C
:105161007A0251870251940251A10251AE0251BB00
:105171000251BE0251C10251C4758201C002125FC7
:10518100A8D00202528F758202C002124707D002D4
:1051910002528F758204C002124707D00202528F59
:1051A100758201C002124707D00202528F75821622
:1051B100C002124707D00202528F02528F02528F51
:1051C10002528F02528F901298E0FBC374059B50DC
:1051D1000302528FEB25E02B9051DD730251EF0258
:1051E10051FC0252090252160252230252307582B8
:1051F10001C002125FA8D00202528F758202C00262
:10520100124707D00202528F758204C0021247076B
:10521100D00202528F758201C002124707D00202EA
:10522100528F758216C002124707D00202528F02B6
:10523100528F9012977401F002528F901297E0FBF7
:10524100BB0107901298E0FB60159012977401F072
:10525100901298E4F0758200C002125FA8D002900B
:1052610010D07450F0A3E4F09010D0758201C00208
:1052710012474CD00280177B00C002C0037492C059
:10528100E07463C0E01249AAE58124FCF58122C0E3
:1052910083E58290129BF0D0E0A3F0758200124763
:1052A100649010D5E4F090116FF090129BE0FAA396
:1052B100E0FB7CD67D108A828B83E0FE90129BEA14
:1052C100F0A3EBF0EE601A0ABA00010B8C828D8319
:1052D100EEF0A3AC82AD8390116FE0FE2401F0806B
:1052E100D58C828D83E4F090116FE0FABA0400400E
:1052F10028EA24D2FBE43410FC8B82F583126C3053
:10530100AB82EB60141A1A1A1A90116FEAF024D6C4
:10531100F582E43410F583E4F07A0090116FE0FB3C
:10532100C3EA9B501BEA24D6FCE43410FD8C82F5C1
:1053310083E0FEBE5F078C828D837420F00A80DBE0
:10534100BB1800502CC374189BFAE49400FC43046E
:10535100208A418C42EB24D6FAE43410FC8A82F58F
:1053610083126BF590116F7418F09010D5E4F080F2
:105371002E7AD67C107D019014A374B4F0A37463CB
:10538100F0A37402F08A828C838DF0C003129DA475
:10539100D00390116F74032BF09010D57401F0902D
:1053A1001299E0FA60030253FD7A00BA1800501C0A
:1053B100EA2456FBE43411FCEA24D6F582E43410E5
:1053C100F583E0FD8B828C83F00A80DF90116EE41F
:1053D100F09010D37417F0A3E4F09010D37A567BB9
:1053E100117C01C002C003C00474B8C0E07463C082
:1053F100E01249AAE58124FBF581804A9010D5E0AD
:10540100FABA001F7A567B117C01C002C003C004A6
:1054110074C5C0E07463C0E01249AAE58124FBF5BC
:105421008180239063D8124CA27AD67B107C01C074
:1054310002C003C00474DEC0E07463C0E01249AA74
:10544100E58124FBF58175820A1247079012EBE48E
:10545100F022E58290129DF090129F7420F090123C
:1054610098E0FABA030690129F7421F0901299E025
:10547100FA60030255169010D5E0FABA00030254FF
:10548100F09010D3E02401F0FAA3E03400F0FB9097
:10549100116FE0FC7D00C3EA9CEB9D400A9010D3A4
:1054A100E4F0A3F09010D390129EE4F090129EE0ED
:1054B100FABA17005021EA2456FBE43411FC0AEA37
:1054C1002456F582E43411F583E0FD8B828C83F060
:1054D10090129EEAF080D59010D3E0FAA3E0FBEAA7
:1054E10024D6F582EB3410F583E0FA90116DF07A51
:1054F100567B117C0190129FE0FDC002C003C004E5
:10550100C00574F4C0E07463C0E01249AAE58124C7
:10551100FAF581804C90129DE0FA60459010D5E03B
:10552100FA601A90129FE0FAC0027408C0E0746435
:10553100C0E01249AA15811581158180247A567B14
:10554100117C0190129FE0FDC002C003C004C005A0
:105551007414C0E07464C0E01249AAE58124FAF52C
:105561008122C083E5829012A0F0D0E0A3F0758281
:1055710000124764901172E4F090120CF09012A0A6
:10558100E0FAA3E0FB7C737D118A828B83E0FE90BD
:1055910012A0EAF0A3EBF0EE601A0ABA00010B8C3C
:1055A100828D83EEF0A3AC82AD8390120CE0FE24D9
:1055B10001F080D58C828D83E4F07A0090120CE0AA
:1055C100FBC3EA9B501BEA2473FCE43411FD8C827B
:1055D100F583E0FEBE5F078C828D837420F00A8024
:1055E100DBBB18005026C374189BFAE49400FC43FB
:1055F10004208A418C42EB2473FAE43411FC8A8240
:10560100F583126BF5901172E4F0802E7A737C11A0
:105611007D019014A37428F0A37464F0A37402F0C4
:105621008A828C838DF0C003129DA4D00390120C4A
:1056310074032BF09011727401F0901299E0FA60EA
:10564100030256987A00BA1800501CEA24F3FBE4CE
:105651003411FCEA2473F582E43411F583E0FD8B07
:10566100828C83F00A80DF90120BE4F09011707449
:1056710017F0A3E4F09011707AF37B117C01C00262
:10568100C003C004742CC0E07464C0E01249AAE5F0
:105691008124FBF5818044901172E0FABA001F7AEF
:1056A100737B117C01C002C003C0047437C0E07475
:1056B10064C0E01249AAE58124FBF581801D7A735B
:1056C1007B117C01C002C003C004744AC0E0746451
:1056D100C0E01249AAE58124FBF58175820A1247CF
:1056E1000722E5829012A2F09012A47420F0901289
:1056F10098E0FABA04069012A47421F0901299E08D
:10570100FA60030257A6901172E0FABA0003025739
:1057110080901170E02401F0FAA3E03400F0FB90D6
:10572100120CE0FC7D00C3EA9CEB9D400A901170D5
:10573100E4F0A3F09011709012A3E4F09012A3E0B2
:10574100FABA17005021EA24F3FBE43411FC0AEA07
:1057510024F3F582E43411F583E0FD8B828C83F030
:105761009012A3EAF080D5901170E0FAA3E0FBEA71
:105771002473F582EB3411F583E0FA90120AF07A82
:10578100F37B117C019012A4E0FDC002C003C004B0
:10579100C0057460C0E07464C0E01249AAE58124C8
:1057A100FAF581804C9012A2E0FA6045901172E006
:1057B100FA601A9012A4E0FAC0027474C0E0746432
:1057C100C0E01249AA15811581158180247A737B65
:1057D100117C019012A4E0FDC002C003C004C00509
:1057E1007480C0E07464C0E01249AAE58124FAF52E
:1057F1008122E4F54275418790120D126BF5D20AB0
:105801007582001259AE2290122AE4F0901249E4F6
:10581100F0901268E4F090128CE4F0D20A22127433
:1058210068AA82AB83ACF0FD901019E0FEA3E0FF03
:10583100A3E0F8A3E0F9C3EA9EFAEB9FFBEC98FC26
:10584100ED99FD9012F2E0FE9014A9F0A3E4F0A30B
:10585100F0A3F08A828B838CF0ED129E15AA82ABA5
:1058610083ACF0FD90148E74E8F0A37403F0A3E40C
:10587100F0A3F08A828B838CF0ED129C01AA82AB9B
:1058810083ACF0FD9014B6743CF0A3E4F09014B630
:105891008A828B83C002C003129FDFAC82AD83D0AA
:1058A10003D0029014AD743CF0A3E4F09014AD8ADF
:1058B100828B83C004C005129EB2AA82AB83D0053D
:1058C100D004C3EC940AED6480948050089012A532
:1058D1007430F0802F9014B6740AF0A3E4F09014A1
:1058E100B68C828D83C002C003C004C005129FDF45
:1058F100AE82AF83D005D004D003D00274302EFE27
:105901009012A5F09014AD740AF0A3E4F09014ADD8
:105911008C828D83C002C003129EB2AC82AD83D053
:1059210003D00274302CFC9012A6F09012A7743AA6
:10593100F0C3EA940AEB6480948050089012A87432
:1059410030F080279014B6740AF0A3E4F09014B6F6
:105951008A828B83C002C003129FDFAC82AD83D0E9
:1059610003D00274302CFC9012A8F09014AD740A8C
:10597100F0A3E4F09014AD8A828B83129EB2AA82C6
:10598100AB8374302AFA9012A9F09012AAE4F07A4B
:10599100A57B127C01C002C003C0047494C0E074F2
:1059A10064C0E01249AAE58124FBF58122E58290D9
:1059B10012ABF0901297E0FABA0102800FBA02031B
:1059C100025AF8BA0303025B37025B3A9012EBE426
:1059D100F01273299012EBE0FA7003025A809012D0
:1059E100ABE0FA6003025A2C9012EFE0FAA3E0FB5D
:1059F1009012ACE0FC7D00B50231EDB5032D9012A3
:105A0100F1E0FA9012ADE0FBB502209012ECE0FA61
:105A1100A3E0FBA3E0FC8A828B838CF012A05EFAE8
:105A21009012AEE0FBB50203025A939012EFE0FA36
:105A3100A3E0FB9012ACEAF09012ECE0FBA3E0FCD7
:105A4100A3E0FD8B828C838DF012A05EFE9012AEDE
:105A5100F09012F1E0FE9012ADF07F007800C003EB
:105A6100C004C005C006C007C002C00074A1C0E0E8
:105A71007464C0E01249AAE58124F7F5818013908E
:105A810064BF124CA29012ACE4F09012ADF09012EF
:105A9100AEF0200A079012ABE0FA603A7A4F7B121F
:105AA1007C017D307E127F01753D11753E12753F7F
:105AB10001C002C003C004C005C006C007C03DC08C
:105AC1003EC03F74E0C0E07464C0E01249AAE581C1
:105AD10024F5F581C20A9012ABE0FA60159010032B
:105AE100E0FA9012B1E4F09012B27407F08A8212D7
:105AF1005D6A12581F8042901004E0FAF582125E2E
:105B010055901007E0FA901008E0FB9012B8F08A67
:105B110082125F41901005E0FAF582125DC3901088
:105B210009E0FA90100AE0FB9012B6F08A82125E48
:105B3100E712581F800312581F22E5829012AFF01E
:105B41009012AFE0FABA28005003025BD7C3742E5B
:105B51009A5003025BD7EA24D8FA25E02A905B62C7
:105B610073025B77025B8F025B9C025BA8025BA8FE
:105B7100025BAD025BC2901003E0FA9012B1E4F057
:105B81009012B27407F08A82125D6A025BF3901080
:105B910004E0FAF582125E55025BF3901005E0FA1B
:105BA100F582125DC3804B125BF48046901007E0D2
:105BB100FA901008E0FB9012B8F08A82125F4180DF
:105BC10031901009E0FA90100AE0FB9012B6F08AC9
:105BD10082125EE7801C9012AFE0FA7B00C002C027
:105BE100037404C0E07465C0E01249AAE58124FC95
:105BF100F58122901000E0FA60247A227B657C0214
:105C01009012BFE4F09012C0EAF0A3EBF0A3ECF025
:105C11009012C37401F075820012614280227A2BC6
:105C21007B657C029012BFE4F09012C0EAF0A3EB16
:105C3100F0A3ECF09012C37401F07582001261427E
:105C4100901013E0FAC3648094815003025D2BC36A
:105C510074858AF063F08095F05003025D2B1AEA97
:105C610025E02A905C6873025C77025C9C025CC14F
:105C7100025CE5025D097A347B657C029012BFE427
:105C8100F09012C0EAF0A3EBF0A3ECF09012C37411
:105C910002F0758208126142025D2B7A3F7B657CBE
:105CA100029012BFE4F09012C0EAF0A3EBF0A3EC73
:105CB100F09012C37402F0758208126142025D2BEA
:105CC1007A4A7B657C029012BFE4F09012C0EAF040
:105CD100A3EBF0A3ECF09012C37402F075820812EA
:105CE100614280467A557B657C029012BFE4F09058
:105CF10012C0EAF0A3EBF0A3ECF09012C37402F02F
:105D010075820812614280227A607B657C02901262
:105D1100BFE4F09012C0EAF0A3EBF0A3ECF0901214
:105D2100C37402F075820812614222E5829012B0BA
:105D3100F09012B0E0FAC374409AFA0303543FFAA8
:105D410090656B124CA27B00BB11005015EBB502A4
:105D510008906578124CA28006906581124CA20BC6
:105D610080E6906583124CA222E5829012B3F090F6
:105D710012B1E0FA9012B2E0FB7C877D657E029061
:105D810012BFEBF09012C0ECF0A3EDF0A3EEF09097
:105D910012C37405F08A821261429012B3E0FABA1A
:105DA100000890658D124CA280177B00C002C003D1
:105DB100749EC0E07465C0E01249AAE58124FCF537
:105DC1008122E5829012B4F09012B4E0240CFAC260
:105DD100D5EA30E704D2D5F40475F011A430D50A20
:105DE100F42401C5F0F43400C5F0FAABF09014B618
:105DF1007419F0A3E4F09014B68A828B83129FDFAA
:105E0100AA82AB837BB17C657D029012BF7405F0E1
:105E11009012C0EBF0A3ECF0A3EDF09012C3740765
:105E2100F0758200C002126142D0029065B7124C37
:105E3100A27B00BB11005015EBB502089065BF12A3
:105E41004CA280069065C8124CA20B80E69065CAF0
:105E5100124CA222E5829012B5F09012B5E0240C0A
:105E6100FAC2D5EA30E704D2D5F40475F011A430B2
:105E7100D50AF42401C5F0F43400C5F0FAABF09072
:105E810014B67419F0A3E4F09014B68A828B8312CD
:105E91009FDFAA82AB837BD07C657D029012BF74A9
:105EA10003F09012C0EBF0A3ECF0A3EDF09012C35D
:105EB1007405F0758200C002126142D0029065D66D
:105EC100124CA27B00BB11005015EBB50208906586
:105ED100DE124CA280069065E7124CA20B80E69080
:105EE10065E9124CA222E5829012B7F09012B7E058
:105EF100FB7A009012B6E0FC7D002AFAED3BFB7CB8
:105F0100EF7D657E029012BF7406F09012C0ECF036
:105F1100A3EDF0A3EEF09012C37408F0758200C0F7
:105F210002C003126142D003D002C002C00374FD5B
:105F3100C0E07465C0E01249AAE58124FCF5812224
:105F4100E5829012B9F09012B9E0FB7A009012B894
:105F5100E0FC7D002AFAED3BFB7C0E7D667E029023
:105F610012BF7404F09012C0ECF0A3EDF0A3EEF0B8
:105F71009012C37406F0758200C002C00312614220
:105F8100D003D002C002C003741CC0E07466C0E03C
:105F91001249AAE58124FCF5812290662D124CA2BA
:105FA1009012967401F022E5829012BAF09012BB21
:105FB100E4F09012BC7405F09012BD7408F09012D8
:105FC100BE7404F09012BAE0FABA0114901297E08C
:105FD1002401F0FAC374039A50069012977401F0E9
:105FE100901297E0FA24BBF582E43412F583E0FACB
:105FF100901298E0FBC3EA9B5005901298E4F09050
:106001001298E0FABA00005014901297E0FA24BBFB
:10601100F582E43412F583E0FA901298F090129927
:10602100E0FABA000474018001E4FA700690664E49
:10603100124CA2906652124CA2901297E0FBBB0147
:1060410002800EBB02028057BB03030260ED0261B6
:1060510038C002125BF4D002758201C0021254539F
:10606100D002758201C0021256E3D002758201C0CE
:10607100021259AED0027B5D7C667D029012BF7424
:1060810007F09012C0EBF0A3ECF0A3EDF09012C377
:10609100E4F075820EC002126142D002026138C082
:1060A10002125BF4D002758201C002125453D00275
:1060B100758201C0021256E3D002758201C002123C
:1060C10059AED0027B687C667D029012BF7407F0E6
:1060D1009012C0EBF0A3ECF0A3EDF09012C3E4F04A
:1060E10075820EC002126142D002804BC002125B67
:1060F100F4D002758201C002125453D0027582019C
:10610100C0021256E3D002758201C0021259AED00C
:10611100027B737C667D029012BF7407F09012C0FF
:10612100EBF0A3ECF0A3EDF09012C3E4F075820E56
:10613100C002126142D002EA700690667E124CA241
:1061410022E5829012C4F0901298E0FA9012C3E016
:10615100FBB502339012BFE02420FA9012C4E02470
:1061610020FB9012C0E0C0E0A3E0C0E0A3E0C0E0EB
:10617100C002C0037485C0E07466C0E01249AAE59C
:106181008124F9F58180319012BFE02420FA901228
:10619100C4E02420FB9012C0E0C0E0A3E0C0E0A373
:1061A100E0C0E0C002C003749AC0E07466C0E012AF
:1061B10049AAE58124F9F58122C0F0C083E58290E6
:1061C10012C5F0D0E0A3F0D0E0A3F09012E1E4F02A
:1061D1009012C5E0FAA3E0FBA3E0FC7D00BD18002E
:1061E100503C9012E1E0FE7011ED2AF582E43BF59E
:1061F100838CF012A05EFEBE0015ED24C8F582E48A
:106201003412F5837420F09012E17401F0800CEDEA
:1062110024C8F582E43412F583EEF00D80BF9012AC
:10622100E0E4F07AC87B127C01C002C003C00474B0
:10623100AFC0E07466C0E01249AAE58124FBF58194
:10624100229066BC124CA29066C1124CA29066D1FB
:10625100124CA29066E1124CA29066F1124CA290EF
:106261006701124CA2906711124CA2906721124C47
:10627100A2906731124CA2906741124CA2906751D3
:10628100124CA2906761124CA2906771124CA290BD
:106291006781124CA2906791124CA29067A1124C97
:1062A100A29067B1124CA29067C1124CA29067D123
:1062B100124CA29067E1124CA29067F1124CA2908D
:1062C1006801124CA2906811124CA2906821124CE4
:1062D100A2906831124CA2906841124CA290685170
:1062E100124CA2906861124CA2906871124CA2905B
:1062F1006881124CA2906891124CA29068A1124C34
:10630100A29068B1124CA29068C1124CA29068D1BF
:10631100124CA29068E1124CA29068F1124CA2902A
:106321001299E4F0906901124CA2906904124CA2F6
:106331009012967401F075417F7542209010D6122B
:106341006C02754118754220901156126C0275410C
:106351007F754220901173126C02754118754220AD
:106361009011F3126C021257F322E5829012E2F0BF
:106371009012E2E0FA901299F07B00C002C003741F
:1063810007C0E07469C0E01249AAE58124FCF581E7
:1063910022556E737570706F72746564204C43443E
:1063A100204E617669676174696F6E2C20232564C4
:1063B1000D0A00202020005C5B5C4220213C2573FB
:1063C1003E5C5D005C5B5C4220215C432025735C8C
:1063D10043205C5D0D0A005C4B303430005C5B5C3B
:1063E1004B33213125735C4B3321305C4B322131EE
:1063F1005C5D005C5B5C4220215C43256325735C32
:1064010043205C5D0D0A005C4B312125635C4B32FE
:106411002131005C5B5C4220215C43256325735C78
:1064210043205C5D0D0A00202020005C5B5C422063
:106431002225735C5D005C5B5C4220225C4320256D
:10644100735C43205C5D0D0A005C5B5C4B33223165
:1064510025735C4B3322305C4B3222315C5D005C36
:106461005B5C4220225C43256325735C43205C5DB9
:106471000D0A005C4B312225635C4B322231005CFA
:106481005B5C4220225C43256325735C43205C5D99
:106491000D0A005C5B5C42332025735C5D0D0A00D4
:1064A1005C5B5C422026253364206B627073202084
:1064B100253264206B487A202025735C5D005C5B8B
:1064C1005C422026202020206B6270732020202037
:1064D100206B487A20202020202020205C5D005C59
:1064E1004C235C4C245C4C25255C5B5C42202325C1
:1064F100735C42202425735C4220252525735C5D55
:106501000D0A00556E6B6E6F776E204C434420630D
:1065110068616E6765206576656E743A2025640A48
:1065210000506C6179696E67200050617573656414
:1065310020200020446972204F6E6C792000204495
:1065410069722052616E642000205365716E746916
:10655100616C200020506C73742052616E640020C5
:10656100416C6C2052616E6420005C5B5C422027B0
:10657100566F6C3A205B005C43215C775C432000E2
:106581002D005D5C5D00566F6C3A20005C5B5C42E7
:1065910025272020302064425C5D0D0A005C5B5C95
:1065A100422525272D2532642064425C5D0D0A00B9
:1065B1004261733A20005C5B5C4225255B005C43D1
:1065C100215C775C4320002D005D5C5D0D0A005469
:1065D10072653A20005C5B5C4225235B005C4321D1
:1065E1005C775C4320002D005D5C5D0D0A0042611B
:1065F100737320467265713A202020005C5B5C4217
:106601002D2625346420487A5C5D0D0A005472659C
:10661100626C6520467265713A20005C5B5C422DBC
:106621002425346420487A5C5D0D0A005C5B5C4281
:106631002027202020202020202020202020202052
:10664100202020202020202020205C5D005C493A71
:10665100005C5B5C4020305C5D0D0A002020436FD4
:106661006E666967313E002020436F6E666967324E
:106671003E0020202020204D61696E3E005C49389B
:106681005C4939005C5B5C42256325635C432125E1
:10669100735C43205C5D0D0A005C5B5C42256325F5
:1066A100635C432025735C43205C5D0D0A005C5BE9
:1066B1005C42202225735C5D0D0A006C63643A0024
:1066C1005C4830494E4320202020202020202000FB
:1066D1005C48402020202020202020202020200055
:1066E1005C4850494E4320202020202020202000BB
:1066F1005C483144454320202020202020202000D8
:106701005C48412020202020202020202020200023
:106711005C48514445432020202020202020200097
:106721005C48325052565F4C49535420202020007F
:106731005C484220202020202020202020202000F2
:106741005C48525052565F4C49535420202020003F
:106751005C48334E58545F4C49535420202020004C
:106761005C484320202020202020202020202000C1
:106771005C48534E58545F4C49535420202020000C
:106781005C483420202020202020202020202000B0
:106791005C484450524556494F5553202020200013
:1067A1005C48545245564552534520202020200034
:1067B1005C4835504C4159202020202020202000C9
:1067C1005C4845202020202020202020202020005F
:1067D1005C4855202020202020202020202020003F
:1067E1005C4836202020202020202020202020004E
:1067F1005C48464E4558542020202020202020006F
:106801005C4856464F5257415244202020202000D8
:106811005C483755502020202020202020202000B7
:106821005C484720202020202020202020202000FC
:106831005C48575550202020202020202020200077
:106841005C48384C45465420202020202020200040
:106851005C484820202020202020202020202000CB
:106861005C48584C45465420202020202020200000
:106871005C483952494748542020202020202000DC
:106881005C4849202020202020202020202020009A
:106891005C4859524947485420202020202020009C
:1068A1005C483A444F574E202020202020202000D1
:1068B1005C484A2020202020202020202020200069
:1068C1005C485A444F574E20202020202020200091
:1068D1005C483B454E54455220202020202020007A
:1068E1005C484B2020202020202020202020200038
:1068F1005C485B454E54455220202020202020003A
:106901005C45000D0A000D0A537769746368696E6E
:106911006720746F20646973706C61792070726F85
:10692100746F636F6C2076657273696F6E20256476
:106931002E0D0A007895760078947600789376008B
:10694100789276007891760078907600788F76004C
:10695100788E7600788D7600788C7600788B76004C
:10696100788A76007889760078887600788776004C
:1069710078867600788576007884760022126AC35C
:10698100AA828A40E54060028003026AC2906B2AB3
:10699100126ADBAA82EA6003126AFC906B34126A03
:1069A100DBAA82EA6002B21F906B02126ADBAA8242
:1069B100EA600675820112470F906B0C126ADBAA1E
:1069C10082EA600675820312470F906B16126ADB2A
:1069D100AA82EA600675820212470F906B20126A42
:1069E100DBAA82EA600675820412470F906B3E12A1
:1069F1006ADBAA82EA600675821412470F906B481F
:106A0100126ADBAA82EA600675821512470F906B43
:106A110052126ADBAA82EA600675821612470F904B
:106A21006B5C126ADBAA82EA600675821712470F55
:106A3100906B66126ADBAA82EA60067582181247B9
:106A41000F906B70126ADBAA82EA600675821912D6
:106A5100470F906B7A126ADBAA82EA600675821B85
:106A610012470F906B84126ADBAA82EA6006758274
:106A71001A12470F906B8E126ADBAA82EA600675C2
:106A8100821C12470F906B98126ADBAA82EA600699
:106A910075821D12470F906BA2126ADBAA82EA600F
:106AA1000675821E12470F906BAC126ADBAA82EA4E
:106AB100600675825112470F854082126AD50269BC
:106AC1007E22122032B461004007B47B00500224C0
:106AD100E0F58222E58202203022E493F8E6049375
:106AE100C39540700F06E60493600475820022F698
:106AF1007582012276007582002222C2AF02006DEA
:106B010022844E45585400000000008550524556DD
:106B1100494F55530086504C4159000000000089EF
:106B210052414E444F4D00000087515549540000D9
:106B3100000000884445425547000000008A494E44
:106B4100430000000000008B4445430000000000AA
:106B5100008D4E58545F4C495354008C5052565F2F
:106B61004C495354008E5550000000000000008F26
:106B7100444F574E000000000091524947485400CD
:106B8100000000904C454654000000000092454E24
:106B91005445520000000093464F52574152440061
:106BA100009452455645525345000095564552535F
:106BB100494F4E310005A285418285428305A205D8
:106BC100A2E0A3B461004007B47B00500224E0F5C9
:106BD100F005A2E0A3B461004007B47B0050022499
:106BE100E0B5F00670D97582002250047582FF224B
:106BF1007582012288F0A841E542F0A3D8FCA8F0F3
:106C010022126BF5E4F02205A2854182854283E0E0
:106C11006009A305A2F0A305A280F405A2E4F02275
:106C210075F000E06005A305F080F885F08222E0B0
:106C3100B42E1BA3E04420B46D14A3E04420B4702F
:106C41000DA3E0B43308A3E07004758201227582BC
:106C51000022229010C8740CF075820112472AAAF2
:106C610082901003EAF08A8212460F9010C8E4F075
:106C710075820312472AAA82901004EAF09010C884
:106C8100E4F0758204C00212472AAB82D002901050
:106C910005EBF0901006E4F0901004E0FB90100674
:106CA100E0FCC364808AF063F08095F05005901099
:106CB10006EBF0901005E0FA901006E0FBC364804B
:106CC1008AF063F08095F05009901005E0FA901079
:106CD10006F09010AF7406F0A37410F075827D1267
:106CE10045EE9010AF7404F0A37410F075827B121E
:106CF10045EE9010AF7405F0A37410F075827C120C
:106D010045EE9010C8740BF075820512472AAA82CD
:106D1100901007EAF09010AF7407F0A37410F075AB
:106D210082781245EE9010C874B8F0758206124749
:106D31002AAA82901008EAF09010AF7408F0A374A8
:106D410010F07582771245EE9010C8E4F075820755
:106D510012472AAA82901009EAF09010AF7409F044
:106D6100A37410F075827A1245EE9010C874A0F0E9
:106D710075820812472AAA8290100AEAF09010AF91
:106D8100740AF0A37410F07582791245EE22901006
:106D910003E0FA7880A6029010C97480F075820130
:106DA100124719901004E0FA7880A6029010C97475
:106DB10080F0758203124719901005E0FA7880A6D9
:106DC100029010C97480F07582041247199010075F
:106DD100E0FA7880A6029010C97480F075820512DD
:106DE1004719901008E0FA7880A6029010C97480C3
:106DF100F0758206124719901009E0FA7880A60210
:106E01009010C97480F075820712471990100AE03A
:106E1100FA7880A6029010C97480F0758208124732
:106E21001922901003E014F0FABAFF05901003E460
:106E3100F0901003E014F0FABAFF05901003E4F0AB
:106E4100901003E0FAF58212460F758228125B3B1F
:106E5100D2039010D07464F0A3E4F09010D0758246
:106E61000312474C22901003E004F0FAC374409AD5
:106E710050069010037440F0901003E004F0FAC340
:106E810074409A50069010037440F0901003E0FA99
:106E9100F58212460F758228125B3BD2039010D007
:106EA1007464F0A3E4F09010D075820312474C2271
:106EB100901004E004F0FAC3748C8AF063F08095BA
:106EC100F05006901004740CF0901006E4F090104D
:106ED10004E0FA901006E0FBC364808AF063F0805E
:106EE10095F05009901004E0FA901006F09010050A
:106EF100E0FA901006E0FBC364808AF063F08095AD
:106F0100F05005901006EAF09010AF7406F0A374EB
:106F110010F075827D1245EE9010AF7404F0A374E9
:106F210010F075827B1245EE758229125B3BD2030C
:106F31009010D07464F0A3E4F09010D07582031225
:106F4100474C22901004E014F0FAC364809474500A
:106F51000690100474F4F0901006E4F0901004E030
:106F6100FA901006E0FBC364808AF063F08095F02C
:106F71005009901004E0FA901006F0901005E0FA24
:106F8100901006E0FBC364808AF063F08095F050B6
:106F910005901006EAF09010AF7404F0A37410F09D
:106FA10075827B1245EE9010AF7406F0A37410F059
:106FB10075827D1245EE758229125B3BD2039010DA
:106FC100D07464F0A3E4F09010D075820312474CA2
:106FD10022901005E004F0FAC3748C8AF063F0800B
:106FE10095F05006901005740CF0901006E4F090A6
:106FF1001004E0FA901006E0FBC364808AF063F0AD
:107001008095F05005901006EAF0901005E0FA9096
:107011001006E0FBC364808AF063F08095F05009AC
:10702100901005E0FA901006F09010AF7406F0A3EE
:107031007410F075827D1245EE9010AF7405F0A3C7
:107041007410F075827C1245EE75822A125B3BD278
:10705100039010D07464F0A3E4F09010D075820313
:1070610012474C22901005E014F0FAC36480947426
:10707100500690100574F4F0901006E4F09010049E
:10708100E0FA901006E0FBC364808AF063F080951B
:10709100F05005901006EAF0901005E0FA90100605
:1070A100E0FBC364808AF063F08095F05009901092
:1070B10005E0FA901006F09010AF7405F0A374107B
:1070C100F075827C1245EE9010AF7406F0A3741037
:1070D100F075827D1245EE75822A125B3BD20390D8
:1070E10010D07464F0A3E4F09010D07582031247BD
:1070F1004C22901007E0FB7A00901008E0FC7D0024
:107101002AFAED3BFB9012E3EAF0A3EBF0C3EA9419
:1071110006EB648094A7500B9012E3740A2AF0E402
:107121003BA3F09012E3E0FAA3E0FB7C00FDEDFC51
:107131003395E0FD901007ECF07B00901008EAF029
:107141009010AF7407F0A37410F07582781245EEB9
:107151009010AF7408F0A37410F07582771245EEA9
:1071610075822D125B3BD2039010D07464F0A3E4BE
:10717100F09010D075820312474C22901007E0FB6B
:107181007A00901008E0FC7D002AFAED3BFB90129A
:10719100E5EAF0A3EBF0C3740A9A74808BF063F014
:1071A1008095F05010EA24F6FAEB34FFFB9012E5DB
:1071B100EAF0A3EBF09012E5E0FAA3E0FB7C00FD1E
:1071C100EDFC3395E0FD901007ECF07B009010088A
:1071D100EAF09010AF7407F0A37410F07582781282
:1071E10045EE9010AF7408F0A37410F07582771219
:1071F10045EE75822D125B3BD2039010D07464F082
:10720100A3E4F09010D075820312474C229010092C
:10721100E0FB7A0090100AE0FC7D002AFAED3BFBCE
:107221009012E7EAF0A3EBF0C3EA9406EB648094D2
:10723100A7500B9012E7740A2AF0E43BA3F09012D6
:10724100E7E0FAA3E0FB7C00FDEDFC3395E0FD9067
:107251001009ECF07B0090100AEAF09010AF74096D
:10726100F0A37410F075827A1245EE9010AF740A93
:10727100F0A37410F07582791245EE75822E125BBF
:107281003BD2039010D07464F0A3E4F09010D07559
:10729100820312474C22901009E0FB7A0090100AF9
:1072A100E0FC7D002AFAED3BFB9012E9EAF0A3EB4A
:1072B100F0C3740A9A74808BF063F08095F05010DB
:1072C100EA24F6FAEB34FFFB9012E9EAF0A3EBF0C3
:1072D1009012E9E0FAA3E0FB7C00FDEDFC3395E0C0
:1072E100FD901009ECF07B0090100AEAF09010AFCD
:1072F1007409F0A37410F075827A1245EE9010AF04
:10730100740AF0A37410F07582791245EE75822E1D
:10731100125B3BD2039010D07464F0A3E4F09010A0
:10732100D075820312474C229012EBE0FA600302FF
:107331007464124603AA82AB83ACF0FD9012F3EAA7
:10734100F0A3EBF0A3ECF0A3EDF09012F6E0FABAA3
:10735100020280067582000274679012F5E0FA203D
:10736100E3030273B39012F4E0C4540F75F002A466
:10737100FAABF02436F582EB3475F583E493FAA386
:10738100E493FB9012EFEAF0A3EBF09012F4E0FA31
:107391000303540390757693FA9012F1F09012F46E
:1073A100E0FA0303540390758293FA9012F2F0020B
:1073B100742B9012F4E0C4540F75F002A4FAABF0F0
:1073C1002456F582EB3475F583E493FAA3E493FB39
:1073D1009012EFEAF0A3EBF09012F5E0FA30E42618
:1073E1009012F4E0FA0303540390757A93FA901221
:1073F100F1F09012F4E0FA0303540390758693FAC6
:107401009012F2F080249012F4E0FA0303540390F6
:10741100757E93FA9012F1F09012F4E0FA0303549E
:107421000390758A93FA9012F2F09012F3E054C02F
:10743100FABAC0137A8E7B757C029012ECEAF0A343
:10744100EBF0A3ECF080117A957B757C029012EC45
:10745100EAF0A3EBF0A3ECF09012EB7401F075826B
:10746100018003758200229012F8E4F0A3F0A3F0EA
:10747100A3F09010AD74F7F0A37412F07582691245
:1074810045D4AA82EA70199012F7E0FC7A007B00D9
:107491007D009012F8EAF0A3EBF0A3ECF0A3EDF07D
:1074A1009010AD74F7F0A37412F07582681245D490
:1074B100AA82EA702B9012F7E0FB7A009012F8E0B2
:1074C100FCA3E0FDA3E0FEA3E0FF780079009012A9
:1074D100F8EA2CF0EB3DA3F0E83EA3F0E93FA3F07E
:1074E1009010AD74F7F0A37412F07582671245D451
:1074F100AA82EA702B9012F7E0FA9012F8E0FBA34F
:10750100E0FCA3E0FDA3E0FE7F007800790090128B
:10751100F8EA2BF0EF3CA3F0E83DA3F0E93EA3F03D
:107521009012F8E0FAA3E0FBA3E0FCA3E0FD8A825D
:107531008B838CF022FFFF200028003000380040B0
:10754100005000600070008000A000C000E000005A
:10755100014001FFFFFFFF08001000180020002874
:107561000030003800400050006000700080009042
:1075710000A000FFFF2C302000161810000B0C0893
:10758100001A1824001A1824003030480020204D19
:0B7591006F6E6F0053746572656F0031
:05A0DF00E4F544F54327
:10759C00C083E5829012FCF0D0E0A3F09012FCE0E6
:1075AC00FAA3E0FBC374FA9A740F9B500AE4F582B9
:1075BC00F583F5F00276E290FF0EE0FCA3E0FDE52A
:1075CC00437004E54460028045758201C002C0032B
:1075DC00C004C00512457CAE82AF83D005D004D068
:1075EC0003D0028E458F468E438F4490FF0EEEF0F3
:1075FC00A3EFF0907000E4F0A3F090700274FAF036
:10760C00A3740FF0907004E4F0A3F002767190FF75
:10761C000EE545F0A3E546F0907002E0FEA3E0FF16
:10762C00C3EE9AEF9B503E758201C004C005124513
:10763C007CAA82AB83D005D0048A458B469070001F
:10764C00EAF0A3EBF090FF0EEAF0A3EBF0907000E1
:10765C00E4F0A3F090700274FAF0A3740FF0907041
:10766C0004E4F0A3F090FF0EE0FAA3E0FB9013000B
:10767C00EAF0A3EBF0907002E0FAA3E0FBC3E49A0B
:10768C00FA74109BFB9012FEEAF0A3EBF0907002E0
:10769C00E0FAA3E0FB9012FCE0FEA3E0FFC3EA9E3D
:1076AC00FAEB9FFB907002EAF0A3EBF0907004E011
:1076BC002401F0FAA3E03400F0FB90FF0EECF0A3F1
:1076CC00EDF09012FEE0FAA3E0FBA3E0FCA3E0FDDA
:1076DC008A828B838CF022C0E0C0F0C083E582905C
:1076EC001302F0D0E0A3F0D0E0A3F0D0E0A3F09030
:1076FC00FF0EE0FAA3E0FB901302E0FCA3E0FDA375
:10770C00E0FEA3E0FF901308ECF0A3EDF0A3EEF085
:10771C00A3EFF090130AE0FCA3E0FD90FF0EECF059
:10772C00A3EDF0907004E0FCA3E0FD1CBCFF011D78
:10773C00907004ECF0A3EDF0907004E0FCA3E0FD7D
:10774C00BC0005BD0002800302782C90130AE0FCFB
:10775C00A3E0FDECB54306EDB544028002802C900D
:10776C007000E0F543A3E0F54490130AE0FCA3E0BD
:10777C00FD8C82F583C002C003124584D003D00275
:10778C0090FF0EEAF0A3EBF002782C907000E0FC76
:10779C00A3E0FD90130AE0FEA3E0FF8E82F583C008
:1077AC0002C003C004C005124584D005D004D00328
:1077BC00D002901306E543F0A3E544F0901306E0E5
:1077CC00FEA3E0FFBE0006BF000302781E90FF0E72
:1077DC00EEF0A3EFF0907000E0FEA3E0FF90130A30
:1077EC00E0F8A3E0F9EEB50016EFB50112907000C9
:1077FC00ECF0A3EDF090FF0EEAF0A3EBF0802190FB
:10780C007000E0FCA3E0FD901306ECF0A3EDF00299
:10781C0077C890FF0EEAF0A3EBF0907878124CA2A8
:10782C0022C083C082C5F090FF0AF0A3E5F0F0D02F
:10783C0082D0E0540F2450F58322C083C082C5F05F
:10784C0090FF0CF0A3E5F0F0D082D0E0540F246050
:10785C00F58322C083C082C5F090FF0EF0A3E5F043
:10786C00F0D082D0E0540F2470F583224572726FF1
:10787C00723A20636F756C642066696E6420667260
:10788C0065656420626C6F636B0D0A00901310E4E5
:10789C00F0A3F0A3F0A3F0901314E4F0A3F0A3F082
:1078AC00A3F090130CE4F0A3F0A3F0A3F090130C4E
:1078BC0022C0E0C0F0C083E582901318F0D0E0A3A2
:1078CC00F0D0E0A3F0D0E0A3F090001412759CAAC5
:1078DC0082AB83ACF0FD8A4F8B508C51F5529013D8
:1078EC0010E0FAA3E0FBA3E0FCA3E0FDBA000BBBA5
:1078FC000008BC0005BD00028003027959901310EA
:10790C00E54FF0A3E550F0A3E551F0A3E552F0905C
:10791C001314E54FF0A3E550F0A3E551F0A3E552A5
:10792C00F0854F828550838551F0127846AA82AB40
:10793C008390131CEAF0A3EBF074042AF582E43B69
:10794C00F583E4F0A3F0A3F0A3F00279CA9013142A
:10795C00E0FAA3E0FBA3E0FCA3E0FD8A828B838C1E
:10796C00F0127846AE82AF8374082EF582E43FF5B0
:10797C0083E54FF0A3E550F0A3E551F0A3E552F0F9
:10798C00854F828550838551F0127846AE82AF8345
:10799C0090131CEEF0A3EFF074042EF582E43FF587
:1079AC0083EAF0A3EBF0A3ECF0A3EDF0901314E555
:1079BC004FF0A3E550F0A3E551F0A3E552F090137E
:1079CC000CE54FF0A3E550F0A3E551F0A3E552F020
:1079DC0090131CE0FAA3E0FB74082AF582E43BF553
:1079EC0083E4F0A3F0A3F0A3F0740C2AF582E43B3B
:1079FC00F583E4F0A3F0A3F0A3F074102AF582E46D
:107A0C003BF583E4F0A3F0A3F0A3F0901318E0FC93
:107A1C00A3E0FDA3E0FEA3E0FF8A828B83ECF0A33E
:107A2C00EDF0A3EEF0A3EFF022C0E0C0F0C083E5D0
:107A3C008290131EF0D0E0A3F0D0E0A3F0D0E0A32E
:107A4C00F090130CE0FAA3E0FBA3E0FCA3E0FD8AAA
:107A5C00828B838CF0127846AA82AB83901322EA35
:107A6C00F0A3EBF090000CC002C00312759CAC822A
:107A7C00AD83AEF0FFD003D0028C4F8D508E518F62
:107A8C0052740C2AF582E43BF583E0FAA3E0FBA3E5
:107A9C00E0FCA3E0FDBA000BBB0008BC0005BD0078
:107AAC00028003027B16901322E0FAA3E0FB740C15
:107ABC002AF582E43BF583E54FF0A3E550F0A3E50E
:107ACC0051F0A3E552F074102AF582E43BF583E5FE
:107ADC004FF0A3E550F0A3E551F0A3E552F0854F2C
:107AEC00828550838551F012785FAA82AB83901304
:107AFC0024EAF0A3EBF074042AF582E43BF583E46A
:107B0C00F0A3F0A3F0A3F0027BA6901322E02410C4
:107B1C00FAA3E03400FB8A82F583E0FCA3E0FDA32A
:107B2C00E0FEA3E0FF8C828D838EF012785FAC8236
:107B3C00AD8374082CF582E43DF583E54FF0A3E5A5
:107B4C0050F0A3E551F0A3E552F0854F82855083A8
:107B5C008551F012785FAC82AD83901324ECF0A3C6
:107B6C00EDF074042CFCE43DFD8A828B83E0FEA3D3
:107B7C00E0FFA3E0F8A3E0F98C828D83EEF0A3EF95
:107B8C00F0A3E8F0A3E9F08A828B83E54FF0A3E53C
:107B9C0050F0A3E551F0A3E552F0901324E0FAA3C2
:107BAC00E0FB74082AF582E43BF583E4F0A3F0A330
:107BBC00F0A3F090131EE0FCA3E0FDA3E0FEA3E015
:107BCC00FF8A828B83ECF0A3EDF0A3EEF0A3EFF031
:107BDC002290130CE0FAA3E0FBA3E0FCA3E0FD8AE7
:107BEC00828B838CF012785FAA82AB83740C2AF59B
:107BFC0082E43BF583E0F54FA3E0F550A3E0F551AB
:107C0C00A3E0F552E54F700FE550700BE55170078E
:107C1C00E5527003027C9D854F828550838551F01F
:107C2C00E552127846E0FAA3E0FBA3E0FCA3E0FDEA
:107C3C008A828B838CF012785FAA82AB83740D2AB4
:107C4C00F582E43BF583E0FAA3E0FBA3E0FCA3E0C0
:107C5C00FD8A828B838CF0127846AA82AB83124CFD
:107C6C00AD124D26854F828550838551F0E5521219
:107C7C007846AA82AB8374082AF582E43BF583E04C
:107C8C00F54FA3E0F550A3E0F551A3E0F552027CCB
:107C9C001022901310E0FAA3E0FBA3E0FCA3E0FD9C
:107CAC0090130CEAF0A3EBF0A3ECF0A3EDF090131F
:107CBC000CE0FAA3E0FBA3E0FCA3E0FDBA000CBBD4
:107CCC000009BC0006BD0003027DB190130CE0FA64
:107CDC00A3E0FBA3E0FCA3E0FD8A828B838CF01273
:107CEC007846AE82AF83907DCE124CA28E828F836B
:107CFC00E0F547A3E0F548A3E0F549A3E0F54A8594
:107D0C0047828548838549F0E54A12785FA882A9A5
:107D1C0083124CAD8E828F83E0FEA3E0FFA3E0F8CC
:107D2C00A3E0F98E828F8388F012785FAE82AF83E6
:107D3C007801C002C003C004C005C006C007C00063
:107D4C0074DAC0E0747DC0E01249AAE58124FBF529
:107D5C0081D005D004D003D002124D26C002C0033E
:107D6C00C004C005127BDDD005D004D003D00212B4
:107D7C004D268A828B838CF0ED127846AA82AB83D7
:107D8C0074082AF582E43BF583E0FAA3E0FBA3E058
:107D9C00FCA3E0FD90130CEAF0A3EBF0A3ECF0A332
:107DAC00EDF0027CBA901310E0FAA3E0FBA3E0FC28
:107DBC00A3E0FD90130CEAF0A3EBF0A3ECF0A3ED21
:107DCC00F0220D0A506C61796C69737420002825BF
:037DDC0073290008
:10A0E400901435E4F0A3F0A3F0A3F0901435901489
:0CA0F40039E4F0A3F0A3F0A3F0901439BD
:107DDF00C06B85816BAA82AB83ACF0FD901428E059
:107DEF002401FE901428F0C374049E50109092F951
:107DFF00124CA2901428E0FE14F0027EDF8A828BD0
:107E0F00838CF0ED12782DAE82AF83C002C003C019
:107E1F0004C005127EE5D005D004D003D0028A82BB
:107E2F008B838CF0ED12782DAA82AB8374112AF517
:107E3F0082E43BF583E0FAA3E0FBA3E0FCA3E0FDC3
:107E4F00BA000CBB0009BC0006BD0003027ED88A35
:107E5F00828B838CF0ED12782DAE82AF83740D2E52
:107E6F00F582E43FF583E0FEA3E0FFA3E0F8A3E093
:107E7F00F98E828F8388F0C002C003C004C0051240
:107E8F0078BDD005D004D003D0028A828B838CF0CA
:107E9F00EDC002C003C004C005127DDFD005D004C1
:107EAF00D003D0028A828B838CF0ED12782DAE82B4
:107EBF00AF8374222EF582E43FF583E0FAA3E0FB53
:107ECF00A3E0FCA3E0FD027E4F901428E0FA14F02B
:107EDF00856B81D06B22C083E582901441F0D0E096
:107EEF00A3F0C20B901433E0FA2401F0A3E0FB34AB
:107EFF0000F0901441E02405FAA3E03400F5838AE2
:107F0F0082E0FAA3E0FBA3E0FCA3E0FD8A828B836F
:107F1F008CF0124629AA82901444EAF09010B1E432
:107F2F00F0A3F0A3F0A3F09010B574FFF0A3F0A3AB
:107F3F00F0A3F08A82124636D20CD20D901444E090
:107F4F00FAF58212465BAA82901443EAF0BA020352
:107F5F00124515758204124535901443E0FA60DC22
:107F6F00758208124535901444E0FA9010C1E4F080
:107F7F00A3F0A3F0A3F09010C18A82124663300BD6
:107F8F001690143DE0F54FA3E0F550A3E0F551A393
:107F9F00E0F552C20B801590001A12759CAA82ABA5
:107FAF0083ACF0FD8A4F8B508C51F552854F8285F3
:107FBF0050838551F0E55212785FAA82AB838A4DC8
:107FCF008B4E901444E0FA9010CEE54DF0A3E54EA1
:107FDF00F08A821246E1AA82901443EAF0BA0109AC
:107FEF00758204124535027F8D901443E0FA6003C9
:107FFF00028529854D82854E83E0FABA1709909341
:10800F0018124CA2027F8D854D82854E83E0540C51
:10801F00FA6009909336124CA2027F8D740D254D94
:10802F00FAE4354EFB7401254DF582E4354EF583A8
:10803F00E0FC7D00F5828D83C002C00312759CACFD
:10804F0082AD83AEF0FFD003D0028A828B83ECF037
:10805F00A3EDF0A3EEF0A3EFF0740D254DF582E440
:10806F00354EF583E0FAA3E0FBA3E0FCA3E0FD8A25
:10807F00828B838CF0127846AA82AB83901445EAE8
:10808F00F0A3EBF08A828B831246F1854D82854EE9
:10809F0083E0FA20E4030282A6901445E0FAA3E0FD
:1080AF00FB8A82F583E0FABA2E03027F8D90143D8E
:1080BF00E54FF0A3E550F0A3E551F0A3E552F0D260
:1080CF000B90002A12759CAA82AB83ACF0FD8A4FED
:1080DF008B508C51F552127846AA82AB838A4B8B08
:1080EF004C7C0190149BE54DF0A3E54EF0A3740179
:1080FF00F090149E7411F0A3E4F090149E8A828B7A
:10810F00838CF0129D2B901441E02411FAA3E034DC
:10811F0000F5838A82E0FAA3E0FBA3E0FCA3E0FD75
:10812F00BA000BBB0008BC0005BD00028003028132
:10813F00A2901441E0FAA3E0FB74112AF582E43B0C
:10814F00F583E54FF0A3E550F0A3E551F0A3E55219
:10815F00F074152AF582E43BF583E54FF0A3E55063
:10816F00F0A3E551F0A3E552F0854F82855083854A
:10817F0051F0127846AA82AB838A4B8B4C7426251A
:10818F004BF582E4354CF583E4F0A3F0A3F0A3F0B4
:10819F00028236901441E02415FAA3E03400FB8AE2
:1081AF0082F583E0FCA3E0FDA3E0FEA3E0FF8C8259
:1081BF008D838EF0127846AC82AD838C4B8D4C74D0
:1081CF0022254BF582E4354CF583E54FF0A3E550BE
:1081DF00F0A3E551F0A3E552F0854F8285508385DA
:1081EF0051F0127846AC82AD838C4B8D4C742625A2
:1081FF004BFCE4354CFD8A828B83E0FEA3E0FFA3AA
:10820F00E0F8A3E0F98C828D83EEF0A3EFF0A3E802
:10821F00F0A3E9F08A828B83E54FF0A3E550F0A33A
:10822F00E551F0A3E552F07422254BF582E4354C6D
:10823F00F583E4F0A3F0A3F0A3F07411254BF582BE
:10824F00E4354CF583E4F0A3F0A3F0A3F074152507
:10825F004BF582E4354CF583E4F0A3F0A3F0A3F0E3
:10826F00741A254BF582E4354CF583E4F0A3F0A3A3
:10827F00F0A3F0741E254BF582E4354CF583E4F042
:10828F00A3F0A3F0A3F07419254BF582E4354CF558
:10829F00837401F0027F8D901431E0FA2401F0A372
:1082AF00E0FB3400F01292CEAA82BA01028009BA22
:1082BF00020302840602850E901441E0241AFAA3E9
:1082CF00E03400F5838A82E0FAA3E0FBA3E0FCA38D
:1082DF00E0FDBA000BBB0008BC0005BD0002800327
:1082EF00028340901441E0FAA3E0FB741A2AF5824E
:1082FF00E43BF583E54FF0A3E550F0A3E551F0A380
:10830F00E552F0741E2AF582E43BF583E54FF0A3A6
:10831F00E550F0A3E551F0A3E552F07412254DF5A9
:10832F0082E4354EF583E4F0A3F0A3F0A3F00283CB
:10833F00D4901441E0241EFAA3E03400FB8A82F5A6
:10834F0083E0FCA3E0FDA3E0FEA3E0FF8C828D831E
:10835F008EF012785FAC82AD838C4D8D4E741625E6
:10836F004DF582E4354EF583E54FF0A3E550F0A3CC
:10837F00E551F0A3E552F0854F828550838551F08A
:10838F0012785FAC82AD838C4D8D4E7412254DFCEF
:10839F00E4354EFD8A828B83E0FEA3E0FFA3E0F875
:1083AF00A3E0F98C828D83EEF0A3EFF0A3E8F0A3A6
:1083BF00E9F08A828B83E54FF0A3E550F0A3E551F6
:1083CF00F0A3E552F07416254DF582E4354EF58392
:1083DF00E4F0A3F0A3F0A3F0854F8285508385517D
:1083EF00F0E552127A3590142DE0FA2401F0A3E053
:1083FF00FB3400F0027F8D901435E0FAA3E0FBA36D
:10840F00E0FCA3E0FDBA0043BB0040BC003DBD0053
:10841F003A901435E54FF0A3E550F0A3E551F0A3E2
:10842F00E552F0901439E54FF0A3E550F0A3E55174
:10843F00F0A3E552F07412254DF582E4354EF58325
:10844F00E4F0A3F0A3F0A3F00284CF901439E0FA84
:10845F00A3E0FBA3E0FCA3E0FD8A828B838CF012E8
:10846F00785FAE82AF838E4D8F4E7416254DF58299
:10847F00E4354EF583E54FF0A3E550F0A3E551F059
:10848F00A3E552F0854F828550838551F012785FB6
:10849F00AE82AF838E4D8F4E7412254DF582E4352B
:1084AF004EF583EAF0A3EBF0A3ECF0A3EDF09014FC
:1084BF0039E54FF0A3E550F0A3E551F0A3E552F0F5
:1084CF007416254DF582E4354EF583E4F0A3F0A341
:1084DF00F0A3F0909354124CA2901445E0FAA3E04D
:1084EF00FB8A82F583124CAD909372124CA29014BA
:1084FF002FE0FA2401F0A3E0FB3400F0027F8D900F
:10850F009389124CA2901445E0FAA3E0FB8A82F5FE
:10851F0083124CAD124D26027F8D901444E0FAF574
:10852F008212469E1246CB22901435E0F54FA3E0FF
:10853F00F550A3E0F551A3E0F5529093AC124CA285
:10854F00E54F700FE550700BE5517007E552700362
:10855F00028643854F828550838551F0E55212780C
:10856F0046AA82AB838A4D8B4E740D254DF582E45E
:10857F00354EF583E0FAA3E0FBA3E0FCA3E0FD8A10
:10858F00828B838CF012785FAA82AB83124CAD90F2
:10859F0093BF124CA27405254DF582E4354EF58339
:1085AF00E0FAA3E0FBA3E0FCA3E0FD8A828B838CBF
:1085BF00F0124CBC9093C8124CA27409254DF58251
:1085CF00E4354EF583E0FAA3E0FBA3E0FCA3E0FD66
:1085DF008A828B838CF0124CBC7404254DF582E497
:1085EF00354EF583E0FA7403254DF582E4354EF5EB
:1085FF0083E0FB7402254DF582E4354EF583E0FCF4
:10860F00C002C003C00474CEC0E07493C0E012492E
:10861F00AAE58124FBF5817416254DF582E4354ECC
:10862F00F583E0F54FA3E0F550A3E0F551A3E0F596
:10863F005202854F22E582901458F07AFF7B4FC388
:10864F00EA9553EB64808554F063F08095F0400316
:10865F000286BC90FF0AE0FAA3E0FB90FF08EAF065
:10866F00A3EBF0901447E0FAA3E0FBA3E0FCA3E038
:10867F00FDEB24F0FBEC34FFFCED34FFFD901447D1
:10868F00EAF0A3EBF0A3ECF0A3EDF0C3E49A7410BF
:10869F009BE49CE49D5010901458E0FA9010D27413
:1086AF0005F08A82124775E55424F0F5549014575B
:1086BF00E4F090144BE553F0A3E554F0901447E029
:1086CF00FAA3E0FBA3E0FCA3E0FDE42AFA74403B2D
:1086DF00FBE43CFCE43DFDAE53AF54C3EE9AEF9B7D
:1086EF0040030287AB855382855483E0FABA0A03AD
:1086FF0002875EBA0D0302875EBA2F028008BA5C4A
:10870F000280030287A0855382855483E4F090147E
:10871F0057E02401F0FABA06005024901457E07580
:10872F00F002A4FAABF0244BF582EB3414F583740A
:10873F00012553FAE43554FBEAF0A3EBF080529095
:10874F0093DB124CA2901457E0FAF5820287B6859C
:10875F005382855483E4F00553E4B55302055485E1
:10876F005382855483E0FABA0A02800B85538285BF
:10877F005483E0FABA0D10855382855483E4F005D3
:10878F0053E4B553020554901457E004FAF5828070
:10879F00160553E4B5530205540286CB85538285E3
:1087AF005483E4F075820022901459E4F09013265C
:1087BF00E0F54FA3E0F550A3E0F551A3E0F552909B
:1087CF001459E0F558E54F700FE550700BE55170F7
:1087DF0007E55270030289FE854F828550838551CC
:1087EF00F0E55212785FAB82AC838B4B8C4C9014BC
:1087FF0057E0FBE558B5030280030288ED9093FD27
:10880F00124CA275F002E558A4FBACF0244BF58294
:10881F00EC3414F583E0FBA3E0FC8B82F583124C60
:10882F00AD124D26741A254BF582E4354CF583E0D5
:10883F00FBA3E0FCA3E0FDA3E0FE90145AEBF0A332
:10884F00ECF0A3EDF0A3EEF090145AE0FBA3E0FCE4
:10885F00A3E0FDA3E0FEBB000DBC000ABD0007BEF8
:10886F00000474018001E4F55770188B828C838D9E
:10887F00F0EE127846A882A983880789028F4D8A65
:10888F004E80D37A01EA602A90942A124CA275F096
:10889F0002E558A4FAABF0244BF582EB3414F583C0
:1088AF00E0FAA3E0FB8A82F583124CAD124D26024B
:1088BF0089F3909431124CA2901459E075F002A4F0
:1088CF00FAABF0244BF582EB3414F583E0FAA3E016
:1088DF00FB8A82F583124CAD124D260289FE9094CD
:1088EF003E124CA275F002E558A4FAABF0244BF5FA
:1088FF0082EB3414F583E0FAA3E0FB8A82F583124E
:10890F004CAD90944D124CA2124D267411254BF57F
:10891F0082E4354CF583E0FAA3E0FBA3E0FCA3E08F
:10892F00FD90145AEAF0A3EBF0A3ECF0A3EDF09056
:10893F00145AE0FAA3E0FBA3E0FCA3E0FDBA000D9C
:10894F00BB000ABC0007BD000474018001E4F557A9
:10895F0060030289BD8A828B838CF0ED127846AF5B
:10896F0082A8838F018806894B8E4C909457124CA6
:10897F00A2854B55854C56740D2555F582E4355619
:10898F00F583E0F559A3E0F55AA3E0F55BA3E0F515
:10899F005C855982855A83855BF0E55C12785F852B
:1089AF00825D85835E124CAD124D2602894C7A0191
:1089BF00EA7031909462124CA2901459E075F00253
:1089CF00A4FAABF0244BF582EB3414F583E0FAA351
:1089DF00E0FB8A82F583124CAD90946F124CA21279
:1089EF004D26800B0558901459E558F00287D42274
:1089FF00901435E0FAA3E0FBA3E0FCA3E0FD901494
:108A0F0061EAF0A3EBF0A3ECF0A3EDF090947912F0
:108A1F004CA2901461E0FAA3E0FBA3E0FCA3E0FDFD
:108A2F00BA000CBB0009BC0006BD0003028D3190DB
:108A3F001461E0FAA3E0FBA3E0FCA3E0FD8A828BC4
:108A4F00838CF012785FAA82AB838A4D8B4E740DA4
:108A5F00254DF582E4354EF583E0FAA3E0FBA3E064
:108A6F00FCA3E0FD8A828B838CF0127846AA82AB3E
:108A7F0083124CAD909491124CA27405254DF58242
:108A8F00E4354EF583E0FAA3E0FBA3E0FCA3E0FDA1
:108A9F008A828B838CF0124CBC90949A124CA274E5
:108AAF0009254DF582E4354EF583E0FAA3E0FBA3EB
:108ABF00E0FCA3E0FD8A828B838CF0124CBC124D3C
:108ACF00267405254DF582E4354EF583E0FAA3E0D3
:108ADF00FBA3E0FCA3E0FD8A828B838CF012462976
:108AEF00AA8290145FEAF09010B1E4F0A3F0A3F023
:108AFF00A3F09010B574FFF0A3F0A3F0A3F08A8257
:108B0F0012463675820412453590145FE0FAF582ED
:108B1F00C00212465BAB82D00290145EEBF0BB0238
:108B2F000474018001E4FC600312451590145EE0AB
:108B3F00FD60D075820812453590145FE0FA9010F1
:108B4F00C1E4F0A3F0A3F0A3F09010C18A82C00299
:108B5F00124663D0027409254DF582E4354EF58334
:108B6F00E0FBA3E0FCA3E0FDA3E0FE901447EBF0D5
:108B7F00A3ECF0A3EDF0A3EEF09010D27404F08A02
:108B8F0082124775901447E0FAA3E0FBA3E0FCA321
:108B9F00E0FDC3E49A74109BE49CE49D5010901484
:108BAF005FE0FA9010D27405F08A82124775755300
:108BBF000075544074022553F582E43554F583E073
:108BCF00FA74012553F582E43554F583E0FB8553A0
:108BDF0082855483E0FCC002C003C00474A0C0E0CF
:108BEF007494C0E01249AAE58124FBF5819094B7F3
:108BFF00124CA2740D254DF582E4354EF583E0FA43
:108C0F00A3E0FBA3E0FCA3E0FD8A828B838CF01230
:108C1F0078BD9094CB124CA290145FE0FAF582C00D
:108C2F0002128644AB82D002EB7003028CE19014E7
:108C3F004BE0FCA3E0FD8C82F583E0FEBE230474C1
:108C4F00018001E4FF70D1901460E4F0901460E0B3
:108C5F00F8901457E0F92401F5618862C3E5629535
:108C6F0061E433F56360469094F3124CA2C2D5E8E9
:108C7F0030E704D2D5F40475F002A430D50AF424F9
:108C8F0001C5F0F43400C5F0F56485F065E56424A2
:108C9F004BF582E5653414F583E0F55FA3E0F560ED
:108CAF00855F82856083124CAD08028C60124D2661
:108CBF00C002C003C004C005C006C007C0011287B0
:108CCF00B7D001D007D006D005D004D003D0020210
:108CDF008C2790145FE0FAF58212469E901461E0A3
:108CEF00FAA3E0FBA3E0FCA3E0FD8A828B838CF068
:108CFF0012785FAA82AB838A4D8B4E7416254DF581
:108D0F0082E4354EF583E0FAA3E0FBA3E0FCA3E099
:108D1F00FD901461EAF0A3EBF0A3ECF0A3EDF002E9
:108D2F008A219094F8124CA222901435E4F0A3F00B
:108D3F00A3F0A3F0901439E4F0A3F0A3F0A3F09004
:108D4F00142DE4F0A3F090142FE4F0A3F09014315D
:108D5F00E4F0A3F0901433E4F0A3F090143312472F
:108D6F006CAA82AB83ACF0FD901429EAF0A3EBF070
:108D7F00A3ECF0A3EDF090000212759CAA82AB83D6
:108D8F00ACF0FD8A4F8B508C51F552127846AA8267
:108D9F00AB837C01901488740EF0A37495F0A374C8
:108DAF0002F08A828B838CF0129BA4854F828550B0
:108DBF00838551F0E552127846AA82AB837C01C0BD
:108DCF0002C003C0047410C0E07495C0E01249AA39
:108DDF00E58124FBF581901428E4F090002A1275A8
:108DEF009CAA82AB83ACF0FD901326EAF0A3EBF0C4
:108DFF00A3ECF0A3EDF08A828B838CF0127846AA55
:108E0F0082AB838A4B8B4C7411254BF582E4354C26
:108E1F00F583E4F0A3F0A3F0A3F07415254BF582CE
:108E2F00E4354CF583E4F0A3F0A3F0A3F0741A2516
:108E3F004BF582E4354CF583E4F0A3F0A3F0A3F0F7
:108E4F00741E254BF582E4354CF583E4F0A3F0A3B3
:108E5F00F0A3F07405254BFAE4354CFB124623AC16
:108E6F0082AD83AEF0FF8A828B83ECF0A3EDF0A38B
:108E7F00EEF0A3EFF07422254BF582E4354CF58329
:108E8F00E4F0A3F0A3F0A3F07426254BF582E435AC
:108E9F004CF583E4F0A3F0A3F0A3F0740D254BF58C
:108EAF0082E4354CF583E54FF0A3E550F0A3E5518F
:108EBF00F0A3E552F0740D254BF582E4354CF583A4
:108ECF00E0FAA3E0FBA3E0FCA3E0FD8A828B838C96
:108EDF00F01278BD901326E0FAA3E0FBA3E0FCA309
:108EEF00E0FD8A828B838CF0127DDF12476CAA82A1
:108EFF00AB83ACF0FD901429E0FEA3E0FFA3E0F8F4
:108F0F00A3E0F9C3EA9EFAEB9FFBEC98FCED99FD09
:108F1F00C002C003901433E0C0E0A3E0C0E090149F
:108F2F002FE0C0E0A3E0C0E090142DE0C0E0A3E08C
:108F3F00C0E0901431E0C0E0A3E0C0E07432C0E0C4
:108F4F007495C0E01249AAE58124F6F581D003D0CB
:108F5F00029014B1740AF0A3E4F09014B18A828BDA
:108F6F0083C002C003129F31AC82AD83D003D00205
:108F7F00901481740AF0A3E4F09014818A828B8399
:108F8F00C004C005129B01AA82AB83D005D004C0D8
:108F9F0004C005C002C003746BC0E07495C0E0123A
:108FAF0049AAE58124FAF58122C0E0C0F0C083E52B
:108FBF0082901465F0D0E0A3F0D0E0A3F0D0E0A34E
:108FCF00F0901465E0FAA3E0FBA3E0FCA3E0FD8AB8
:108FDF00828B838CF0127846AA82AB83741A2AF59F
:108FEF0082E43BF583E0F54FA3E0F550A3E0F551A4
:108FFF00A3E0F552E54F700FE550700BE551700788
:10900F00E5527003029085854F828550838551F01C
:10901F00E552127846AA82AB838A4D8B4E740D258A
:10902F004DF582E4354EF583E0FAA3E0FBA3E0FCB7
:10903F00A3E0FD8A828B838CF012785FAA82AB83C8
:10904F007C01C002C003C0047485C0E07495C0E009
:10905F001249AAE58124FBF5817416254DF582E4AA
:10906F00354EF583E0F54FA3E0F550A3E0F551A39E
:10907F00E0F55202900322C06B85816B058105815B
:10908F000581058105810581AA82AB83ACF0FD8A3C
:10909F00828B838CF0127846AE82AF83901426EECB
:1090AF00F0A3EFF0741A2EF582E43FF583E0F54F4D
:1090BF00A3E0F550A3E0F551A3E0F552E54F700F93
:1090CF00E550700BE5517007E552700302917590F2
:1090DF001469E4F0901469E0FEE56B24FDF8C3EE2B
:1090EF0096E433FF601490958A124CA2901469E0B5
:1090FF00F5662401901469F080DAC002C003C00441
:10910F00C005854F828550838551F0E55212784610
:10911F00AE82AF838E4D8F4E740D254DF582E435A3
:10912F004EF583E0FEA3E0FFA3E0FAA3E0FB8E82FF
:10913F008F838AF012785FAA82AB83124CAD124DE7
:10914F00267416254DF582E4354EF583E0F54FA3D1
:10915F00E0F550A3E0F551A3E0F552D005D004D0CF
:10916F0003D0020290CB8A828B838CF0ED1278466B
:10917F00AA82AB8374112AF582E43BF583E0FAA34C
:10918F00E0FBA3E0FCA3E0FDE56B24FDF8740126F2
:10919F00FEBA000CBB0009BC0006BD00030292A47E
:1091AF00901469E4F0901469E0FFE56B24FDF8C3B7
:1091BF00EF96E433F566601490958C124CA29014E0
:1091CF0069E0F5672401901469F080D98A828B8356
:1091DF008CF0ED127846C0E0A86B08D0E0A68208AC
:1091EF00A683A86B08864B08864C90958E124CA2CE
:1091FF00740D254BF582E4354CF583E56B2403F8AC
:10920F00E0F6A3E008F6A3E008F6A3E008F6E56BA6
:10921F002403F886820886830886F008E612785FB2
:10922F00C0E0E56B2403F8D0E0A68208A683E56BC7
:10923F002403F88682088683124CAD124D26C00295
:10924F00C003C004C005C006C0068A828B838CF0A1
:10925F00ED1290861581D006D005D004D003D00230
:10926F008A828B838CF0ED127846C0E0E56B240385
:10927F00F8D0E0A68208A683E56B2403F8742226B3
:10928F00F582E40836F583E0FAA3E0FBA3E0FCA344
:10929F00E0FD0291A0856B81D06B22909595124CC9
:1092AF00A2901326E0FAA3E0FBA3E0FCA3E0FDE409
:1092BF00C0E08A828B838CF0ED1290861581228517
:1092CF004D82854E83A3A3E0B44D1AA3E0B4500999
:1092DF00A3E0B4331075820122B43309A3E0B4556F
:1092EF00047582022275820022224D6178696D75A4
:1092FF006D20737562646972206465707468207282
:10930F006561636865640D0A00536B697070696EFF
:10931F00672052454359434C454420646972656345
:10932F00746F72790D0A00536B697070696E6720E4
:10933F0073797374656D2F68696464656E206669EF
:10934F006C650D0A004465746563746564202E6D49
:10935F00337520706C61796C6973742066696C6504
:10936F002028002920616E64206164646564207484
:10937F006F2071756575650D0A00556E6B6E6F7791
:10938F006E2066696C6520657874656E73696F6EA3
:10939F002C2069676E6F72696E673A20004D3355E6
:1093AF002066696C657320666F756E643A0D0A00EE
:1093BF00636C75737465723D0073697A653D006502
:1093CF0078743D2563256325630D0A00546F6F2064
:1093DF006D616E7920706172747320696E206D33C8
:1093EF00752070617468206E616D650D0A00666F7F
:1093FF00756E6420636F7272656374206469726541
:10940F0063746F72792C20736561726368696E671C
:10941F0020666F722066696C652000666F756E64DA
:10942F00200063616E6E6F742066696E6420007336
:10943F006561726368696E6720666F722000646988
:10944F00726563746F727900636F6D706172696EAC
:10945F0067200063616E6E6F742066696E64200012
:10946F006469726563746F72790070726F6365738C
:10947F0073696E67206D33752066696C65733A0D7D
:10948F000A00636C75737465723D0073697A653D8C
:10949F00006D33752066696C653A205B25632C255A
:1094AF00632C25635D0D0A006372656174696E67D5
:1094BF0020706C61796C6973740D0A006372656159
:1094CF0074656420706C61796C6973742C206C6F97
:1094DF006164696E67206D33752066696C652069FC
:1094EF006E0D0A005B2F5D20006C656176696E67FB
:1094FF002070726F636573735F6D33750D0A002F84
:10950F0000726F6F74206C6F6E67206E616D6520D7
:10951F00696E6974616C6973656420746F2025735B
:10952F000D0A000D0A2A2A2A20466F756E6420251F
:10953F00752066696C657320282575204D50332082
:10954F0026202575204D33552920696E202575203D
:10955F006469726563746F726965730020696E2048
:10956F0025752E2575207365636F6E6473202A2A07
:10957F002A0D0A0D0A0025730D0A0020002000286D
:10958F0064697229200044756D70696E6720646983
:10959F00726563746F7279206C6973742E2E2E0D41
:1095AF000A0090146BE4F0A3F09010C87442F075A9
:1095BF00820F12472AAA8290146AEAF090146AE086
:1095CF00FB7A0090146BEAF0A3EBF09010C87413C1
:1095DF00F075821012472AAA8290146AEAF090144A
:1095EF006AE0FA90146BE0FBA3E0FC7D0090146B33
:1095FF00EA2BF0ED3CA3F09010C8745AF07582027C
:10960F0012472AAA8290146AEAF02290146AE0FAAA
:10961F007880A6029010C97480F0758202124719E3
:10962F0090146BE0FAA3E0FBFA7B007880A602901F
:10963F0010C97480F075820F12471990146BE0FAFD
:10964F00A3E0FB7B007880A6029010C97480F075B0
:10965F0082101247192290146AE07002F4F054B885
:10966F00A2D0E033F0F5822290146AE07002F4F099
:10967F00C0F0F5F05471A2D0E013F085F082D0F075
:10968F002290146BE0FAA3E0FB90146BE07006A33A
:10969F00E07002F4F090146BE05411F5F0A3E05475
:1096AF00A045F0A2D0E013F090146BE013F08A8283
:1096BF008B832290146BE07006A3E07002F4F0909D
:1096CF00146BE05408F5F0A3E054D045F0A2D0900D
:1096DF00146BE033F0F5F0A3E033F085F082F583FF
:1096EF0022E582901471F075410A75422090147230
:1096FF00126C0290146DE0FAFEA3E0FBFFA3E0FCF6
:10970F00F8A3E0FDF9901471E0F568856869339569
:10971F00E0F56AC002C003C004C005C006C007C0A0
:10972F0000C001C069C06A7427C0E0749AC0E0121B
:10973F0049AAE58124F8F581D005D004D003D002E1
:10974F00C002C003C004C0051257F3D005D004D027
:10975F0003D002856882C002C003C004C005124650
:10976F0079AE82AF83A8F0F9D005D004D003D00230
:10977F0090147DEEF0A3EFF0A3E8F0A3E9F0EA2454
:10978F0080FAEB34FFFBEC34FFFCED34FFFD90105F
:10979F00C1EAF0A3EBF0A3ECF0A3EDF08568821221
:1097AF0046639010C5740DF0A37412F09010C77437
:1097BF0003F085688212468190120DE0FABA5402C6
:1097CF00800302989690120EE0FABA4102800302CB
:1097DF00989690120FE0FABA47028003029896907B
:1097EF009A5A124CA2901471E0FA9010C57411F0AD
:1097FF00A37412F09010C7741EF08A82C002124632
:10980F0081D0029010C57430F0A37412F09010C77D
:10981F00741EF08A82C002124681D0029010C57465
:10982F004FF0A37412F09010C7741EF08A82C0021A
:10983F00124681D0029010C5746EF0A37412F0908E
:10984F0010C77404F08A82C002124681D0029010B1
:10985F00C57473F0A37412F09010C7741EF08A824F
:10986F0012468190128FE0FABA0012901290E0FA2D
:10987F00600B901290E0FA901293F0800590129383
:10988F00E4F01258088003125808901471E0FA900F
:10989F00147DE0FBA3E0FCA3E0FDA3E0FE9010C16C
:1098AF00EBF0A3ECF0A3EDF0A3EEF08A82C002126E
:1098BF004663D0028A82C002124679AB82AC83AD76
:1098CF00F0FED0029010C1E4F0A3F0A3F0A3F0904B
:1098DF0010C18A82C002C003C004C005C006124670
:1098EF0063D006D005D004D003D0029010C5747297
:1098FF00F0A37414F09010C7740AF08A82C002C0EB
:10990F0003C004C005C006124681D006D005D0049E
:10991F00D003D0029010C1EBF0A3ECF0A3EDF0A3B5
:10992F00EEF08A82124663901472E0FABA4902800E
:10993F0003029995901473E0FABA444A901474E0B4
:10994F00FABA334290147BE0FA90147AE0FB901449
:10995F0079E0FC901478E0FD901477E0FE90147697
:10996F00E0FF901475E0F8C002C003C004C005C04A
:10997F0006C007C000746CC0E0749AC0E01249AA18
:10998F00E58124F7F5817A0D7B127C01C002C003BB
:10999F00C00474A7C0E0749AC0E01249AAE58124FC
:1099AF00FBF5817A117B127C01C002C003C00474E5
:1099BF00B9C0E0749AC0E01249AAE58124FBF58191
:1099CF007A307B127C01C002C003C00474CBC0E0AC
:1099DF00749AC0E01249AAE58124FBF5817A4F7B86
:1099EF00127C01C002C003C00474DDC0E0749AC0D1
:1099FF00E01249AAE58124FBF5817A737B127C0181
:109A0F00C002C003C00474EFC0E0749AC0E01249F2
:109A1F00AAE58124FBF58122232323232320496EEA
:109A2F00736964652070726F636573735F69643304
:109A3F0020666F722066696C65202564206F662032
:109A4F0073697A6520256C640D0A00466F756E6424
:109A5F00204944337631207461670D0A00466F75D3
:109A6F006E64204944337632207461672E20766508
:109A7F007273696F6E3D256420256420666C616783
:109A8F00733D25642073697A653D257820257820FC
:109A9F0025782025780D0A005461672056616C7572
:109AAF00653A205B25735D0D0A005469746C653A45
:109ABF0020202020205B25735D0D0A004172746900
:109ACF0073743A202020205B25735D0D0A00416CD2
:109ADF0062756D3A20202020205B25735D0D0A00F2
:109AEF00436F6D6D656E743A2020205B25735D0D9D
:109AFF000A00C083C082901483D0E0F0D0E0A3F0BE
:109B0F00901485E4F0A3F09014877410F0901481F2
:109B1F00E0FAA3E0FB901483E0FCA3E0FD235401E3
:109B2F00FEFEEDCC25E0CC33FD901483ECF0A3EDDD
:109B3F00F0901485E0FFA3E0F8CF25E0CF33F89045
:109B4F001485EFF0A3E8F0EE600A90148574014FCE
:109B5F00F0A3E8F0901485E0FEA3E0FFC3EE9AEFC8
:109B6F009B4015901485C3EE9AF0EF9BA3F09014D1
:109B7F008374014CF0A3EDF0901487E014FC901463
:109B8F0087F0EC6003029B24901483E0FAA3E0FBC0
:109B9F008A828B8322C0F0C083C08290148BD0E066
:109BAF00F0D0E0A3F0D0E0A3F090148BE0FAA3E0A4
:109BBF00FBA3E0FC901488E0FDA3E0FEA3E0FF8D83
:109BCF00828E838FF012A05EF8A3AD82AE838A825D
:109BDF008B838CF0E8129E81A3AA82AB83E870DF9F
:109BEF0090148BE0FAA3E0FBA3E0FC8A828B838CBA
:109BFF00F022C0E0C0F0C083C082901492D0E0F099
:109C0F00D0E0A3F0D0E0A3F0D0E0A3F0901496E45E
:109C1F00F0A3F0A3F0A3F090149A7420F090148E98
:109C2F00E0FAA3E0FBA3E0FCA3E0FD901492E0FEBA
:109C3F00A3E0FFA3E0F8A3E0F9235401F56CC360A0
:109C4F0001B3920EEE25E0FEEF33FFE833F8E93370
:109C5F00F9901492EEF0A3EFF0A3E8F0A3E9F090DF
:109C6F001496E0F56DA3E0F56EA3E0F56FA3E0F5B4
:109C7F0070E56D25E0F56DE56E33F56EE56F33F547
:109C8F006FE57033F570901496E56DF0A3E56EF007
:109C9F00A3E56FF0A3E570F0300E149014967401E5
:109CAF00456DF0A3E56EF0A3E56FF0A3E570F090BE
:109CBF001496E0F56DA3E0F56EA3E0F56FA3E0F564
:109CCF0070C3E56D9AE56E9BE56F9CE5709D40272F
:109CDF00901496C3E56D9AF0E56E9BA3F0E56F9C2B
:109CEF00A3F0E5709DA3F090149274014EF0A3EFD2
:109CFF00F0A3E8F0A3E9F090149AE014FE90149A00
:109D0F00F0EE6003029C3A901492E0FAA3E0FBA3FA
:109D1F00E0FCA3E0FD8A828B838CF022C0F0C0832D
:109D2F00C0829014A0D0E0F0D0E0A3F0D0E0A3F078
:109D3F009014A0E0FAA3E0FBA3E0FC90149BE0FDDD
:109D4F00A3E0FEA3E0FF8A6C8B6D8C6E90149EE0F7
:109D5F00F8A3E0F9886F897018B8FF0119E56F450E
:109D6F007060278D828E838FF012A05EF56FA3AD8A
:109D7F0082AE83856C82856D83856EF0E56F129E52
:109D8F0081A385826C85836D80CA8A828B838CF0D8
:109D9F002275820022C0F0C083C0829014A6D0E04A
:109DAF00F0D0E0A3F0D0E0A3F09014A6E0FAA3E087
:109DBF00FBA3E0FC8A828B838CF012A05EFDA3AA2A
:109DCF0082AB83ED600280EC9014A3E0FDA3E0FE74
:109DDF00A3E0FF8D828E838FF012A05EF8A3AD8279
:109DEF00AE838A828B838CF0E8129E81A3AA82AB0A
:109DFF0083E870DF9014A6E0FAA3E0FBA3E0FC8AEF
:109E0F00828B838CF022A882A983AAF0FB88F09022
:109E1F0014A9E0A4FCADF089F0E0A42DFDE435F029
:109E2F00FE88F0A3E0A42DFDE5F03EFEE433FF89AC
:109E3F00F0E0A42EFEE5F03FFF88F0A3E0A42EFE95
:109E4F00E5F03FFF8AF09014A9E0A42EFEE5F03F65
:109E5F00FF8BF0E0A42FFF8AF0A3E0A42FFF89F07F
:109E6F00A3E0A42FFF88F0A3E0A42F8EF08D838CA6
:109E7F008222C8C0E0C8C0E0E5F0600D1460111484
:109E8F006013146014D0E08015D0E0A882F6800E25
:109E9F00D0E0F08009D0E08005D0E0A882F2C8D0F1
:109EAF00E0C822C083C0829014AFD0E0F0D0E0A30E
:109EBF00F09014AFE0FAA3E0FB30E709C3E49AFC9B
:109ECF00E49BFD80048A048B058C028D039014ADF6
:109EDF00E0FCA3E0FD33E433FE6009C3E49CFFE440
:109EEF009DF880048C078D009014B1EFF0A3E8F07B
:109EFF008A828B83C006129F31AA82AB83D00690D1
:109F0F0014AFE0FCA3E0FD33E433FCEE6504600D19
:109F1F00C3E49AFCE49BFD8C828D8380048A828B40
:109F2F008322C083C0829014B3D0E0F0D0E0A3F0BE
:109F3F009014B5E4F09014B3E0FAA3E0FB7C00902A
:109F4F0014B1E0FDA3E0FE235401FF7030EECD25E8
:109F5F00E0CD33FE9014B1EDF0A3EEF0C3EA9DEB2C
:109F6F009E5011EEC313CD13CDFE9014B1EDF0A39F
:109F7F00EEF080090C9014B5ECF0029F4E9014B5E2
:109F8F00E0FA9014B1E0FBA3E0FC9014B3E0FDA362
:109F9F00E0FEC3ED9BEE9C400B9014B3C3ED9BF022
:109FAF00EE9CA3F09014B1E0FBA3E0FCC313CB1322
:109FBF00CBFC9014B1EBF0A3ECF08A031AEB600327
:109FCF00029F919014B3E0FAA3E0FB8A828B832265
:109FDF00C083C0829014B8D0E0F0D0E0A3F090140A
:109FEF00B8E0FAA3E0FB30E709C3E49AFCE49BFD79
:109FFF0080048A048B058C028D039014B6E0FCA3B9
:10A00F00E0FD33E433FE6009C3E49CFFE49DF88078
:10A01F00048C078D00901481EFF0A3E8F08A828BF7
:10A02F0083C006129B01AA82AB83D0069014B8E0BE
:10A03F00FCA3E0FD33E433FCEE6504600DC3E49A4A
:10A04F00FCE49BFD8C828D8380048A828B8322C8E3
:10A05F00C0E0E5F0600D14600F14600F1460107411
:10A06F00FF800FA882E6800AE08007E4938003A8B0
:07A07F0082E2F8D0E0C822E4
:10D00000A5E5E0A5FE5400000000000000000000BF
:10D01000000000000000000000000000FFFFFFFF14
:0AD0200054657374204452414D0022
:10D040007521007130900000513D518290000051D7
:10D050003D51BB500890D90F12003880389008001D
:10D06000513D5182900000513D51BBB3E492E1FC2F
:10D07000900400513D5182900400513D51BBB3ECEE
:10D0800092E0FC90D925120038EC513612005090F5
:10D09000D92C12003890000071099003FF7109909B
:10D0A000015571099002AA71099003D57109900088
:10D0B0009A710990010071099002007109900002B3
:10D0C0007109900049710990000171099000047183
:10D0D0000990022B710990001071099003F67109F3
:10D0E00090000871099000887109900020710990E2
:10D0F00003097109900080710990001F7109900067
:10D1000040710990005971099000E0710990007B0D
:10D1100071099002FD7109900309711590009A71CF
:10D12000159001007115900001711590000871159E
:10D1300090000271159002AA71159000047115906B
:10D140000155711590001071159000007115900334
:10D15000FF711590D9AE120038903043120FE040A5
:10D160007490D90112003890FF127422F0A3E4F0F9
:10D1700031DC90DA0412003890FF28E4F0A37490B8
:10D18000F090FF2A7416F0A37404F0E490FF59F0B5
:10D190007F007E0090FF50E020E106DEF70FBF70B9
:10D1A000F390DA58120038EF120034742012003075
:10D1B000120030EF24B8500CEF24A3400790D9019F
:10D1C0001200382290D9061200380521E52124CE1C
:10D1D000500122014390D906120038229090007429
:10D1E0005578D2F0A3F0A3F0A3F0A3F0A3D8F49065
:10D1F000DA83E581F8F92410F581097A0A7B0FE9D1
:10D20000F8E493A3F608DBF9C083C082E9F8E608E6
:10D21000F582E608F5837B0DE608F0A3DBFAD08201
:10D22000D083DAD9E58124F0F5812253494D4D2090
:10D23000706167653D0004832204081020C082C02D
:10D240008390D22B120038D083D082120036743AE9
:10D25000120030F192E582644D658364B2FDE5828F
:10D260008583F090FF00F0A3E5F0F02257522042B2
:10D27000797465733A200052442042797465733A98
:10D28000200090D26C12003890FF00E0647590008E
:10D2900000F0120034F19290FF01E064DB90000195
:10D2A000F0120034F1929000027123F0120034F178
:10D2B00092A3E582B410F21200482290D2771200B5
:10D2C0003890FF00E06475F5F0900000E012003443
:10D2D000F192B5F02F90FF01E064DBF5F0900001D2
:10D2E000E0120034F192B5F01B9000027123F5F0CA
:10D2F000E0120034F192B5F00BA3E582B410ED1208
:10D300000048C322120048D322C082C083513D513D
:10D3100082D083D082513D51BB40012290DA5B1212
:10D32000003822ED7002F4FD54B8A2D0ED33FD2296
:10D3300090D8DA120038903049120FE0400790D9A7
:0ED34000011200382290D906120038020000B7
:10D40000A5E5E0A523FF00000000000000000000EB
:10D41000000000000000000000000000FFFFFFFF10
:10D42000494445204469736B2044726976652054F1
:04D4300065737400AC
:10D4400012D33090D7BB120038B1D4B1B290D7DB31
:10D4500012003890003C7828D1BA12004890D7E3E7
:10D460001200389000147814D1BA12004890D7EB0B
:10D47000120038900002D1AE90D7F7120038900019
:10D4800006D1AE90D80112003890000CD1AE120037
:10D4900048120048900006E014F57090000CE0F58A
:10D4A0007112D597E4F570F571F572F57390D82285
:10D4B000120038E573120034E572120034E571127F
:10D4C0000034E57012003490D8291200381200326E
:10D4D000120040B4521EB15C6012C0E090D8BF127E
:10D4E0000038D0E012003412004881AD90D89C1270
:10D4F000003881ADB4572D90D85F12003812003239
:10D50000120040B4591CB17C6012C0E090D8BF1228
:10D510000038D0E012003412004881AD90D8AD122E
:10D52000003881ADB44C1890D80D12003812D6C412
:10D5300040088B708C718D728E7312004881ADB46F
:10D540005504B1C281ADB44404B1CA81ADB4510334
:10D55000020000B44804F14081AD81ADD17BD158C7
:10D5600090FF6E7420F0D18520E007900000B1F8A4
:10D57000E42290FF62E060012274FF22D17BD15847
:10D5800090FF6E7430F0D18520E0E7900000D13B31
:10D59000D17B20E0DDE422D17BE570540F44A090E4
:10D5A000FF6CF0E57190FF64F0749190FF6EF0D124
:10D5B0007B22D17B90FF6E74ECF0D185900000B19E
:10D5C000F82290FF6E74E1F0C17BD17B90FF6E7406
:10D5D000E6F0C17BD19290FF6C74A0F0F19C742AAC
:10D5E00012003090FF6EE030E6EC20E7E9120048D0
:10D5F00090FF6E7410F0C17BE5828583F090FF226E
:10D60000F0A3E5F0F090FF24E4F0A37401F090FFA4
:10D610005CF090FF58F090FF50E030E0FC227D007D
:10D62000C083C08290FF60E0FA90FF43E0FBD082AD
:10D63000D083EAF0A3EBF0A3DDE6227D00E0FAA3BD
:10D64000E0FBA3C083C08290FF43EBF090FF60EA51
:10D65000F0D082D083DDE622E573540F44E090FFE2
:10D660006CF0E57290FF6AF0E57190FF68F0E5708C
:10D6700090FF66F0740190FF64F022F19C90FF6EC1
:10D68000E020E7F722F19C90FF6EE020E7F730E31F
:10D69000F42290FF40E4F0D1A3D1A3D1A37401F010
:10D6A000D1A3227800790AD9FE00D8F90022E0C07F
:10D6B000E0A3E0F583D082020053E0600612003060
:10D6C000A3D8F7227A087B007C007D007E00120040
:10D6D00062120040B41B02D322B408028003B47F5C
:10D6E0001CBA080280E81200307804C3EE13FEED85
:10D6F00013FDEC13FCEB13FBD8F10A80D1B40D023F
:10D70000C322FFF12540C7CF120030EFC4FF7804D9
:10D71000EF33FFEB33FBEC33FCED33FDEE33FED8A0
:10D72000EFDAABC322C324D0501424F64004240AF9
:10D73000C32224F9500824FA40042410C322D3221F
:10D740001200487A20900000E583FDC39400120087
:10D7500034E582FC120034743A120030F1927B10EE
:10D76000E0A3120034F192DBF7F192F192F1928C86
:10D77000828D837B10E0A3547FB47F01E424E040DA
:10D7800001E42420120030DBEC120048DABA120067
:10D790004822C0E07420120030D0E02220980122FC
:10D7A000120032B41BF9020000540F232400F5824A
:10D7B000E434FFF583EAF0A3EBF02249444520442A
:10D7C00069736B20447269766520546573742050C8
:10D7D000726F6772616D0D0A0D0A004D6F64656CA2
:10D7E0003A2000532F4E3A2020200043796C696E76
:10D7F000646572733A20002C2048656164733A2096
:10D80000002C20536563746F72733A2000456E7468
:10D810006572204C42412028696E20686578293A5B
:10D8200020004C42413D3078002C2028522965616F
:10D8300064202857297269746520284C29424120A8
:10D8400028552970202844296F776E20284829659B
:10D850007864756D70202851297569740D0A005718
:10D8600061726E696E673A20746869732077696CBB
:10D870006C206368616E67652064617461206F6EFF
:10D88000207468652064726976652C206172652059
:10D89000796F7520737572653F0D0A005365637467
:10D8A0006F722052656164204F4B0D0A005365630F
:10D8B000746F72205772697465204F4B0D0A0045D2
:10D8C00072726F722C20636F6465203D2000445299
:10D8D000414D20546573740D0A00436F6E6669678D
:10D8E0007572696E672058696C696E782058435369
:10D8F0003130584C204650474120436869703A20E7
:10D90000004F6B0D0A004572726F72210D0A0042C2
:10D910006164206F72204D697373696E672053498B
:10D920004D4D0D0A00466F756E642000206D6567D1
:10D930002053494D4D0D0A0046696C6C696E672095
:10D940004452414D20776974682074657374206473
:10D950006174610D0A00436865636B696E672044FA
:10D9600052414D207061676520000D0A444D4120F1
:10D97000746F204D5033206465636F64657220744A
:10D980006573743A200D0A000D0A52656164696E70
:10D990006720696E2036306B206F66206461746189
:10D9A0002066726F6D2064726976650D0A000D0A3B
:10D9B000436F6E6669677572696E672053544130B4
:10D9C0003133204D5033204465636F6465722043CA
:10D9D0006869703A2000506C6179696E6720363052
:10D9E0006B206F66204D5033206461746120757325
:10D9F000696E6720444D412E2E2E0D0A00446F6E35
:10DA0000650D0A004E6F74653A205468697320747E
:10DA10006573742072657175697265732061207712
:10DA20006F726B696E672073696D6D0D0A54657353
:10DA300074696E6720535441303133202874207349
:10DA4000686F756C6420626520617070726F7820F9
:10DA50003532292E2E2E2000743D005741524E495A
:10DA60004E473A2073696D6D206469646E27742097
:10DA7000726573706F6E642070726F7065726C790E
:10DA80000D0A000090FFE320C4000000034801805D
:10DA900000006890FFE322C45B0000034801C0005F
:10DAA00000D190FFE320C4B700000348000000004D
:10DAB0003991FFE322C4FF0000034800000000A2E8
:10DAC00091FFE320C4FF00000348000000000A9219
:10DAD000FFE322C4FF00000348000000007392FF30
:10DAE000E320C4FF0000034800000000DB92FFE3D6
:10DAF00022C4FF00000348000000004493FFE3201D
:10DB0000C4FF0000034800000000AC93FFE322C400
:09DB1000FF0000034800000000C2
:10FD0000A5E5E0A5FE510000000000000000000095
:10FD1000000000000000000000000000FFFFFFFFE7
:10FD2000517569742C2053687574204F6666205095
:05FD30006F7765720011
:07FD4000903046120FE02293
:10FE0000A5E5E0A5FE58000000000000000000008D
:10FE1000000000000000000000000000FFFFFFFFE6
:10FE20004572617365204320436F6465204F6E6C9B
:0FFE300079202020202020202020202758270064
:10FE40009030007424120067904000742412006700
:10FE500090500074241200679060007424120067B0
:10FE60009070007424120067908000742412006760
:10FE7000909000742412006790A000742412006710
:10FE800090B000742412006790C0007424120067C0
:10FE9000903000E493F47011A3E58270F6E583B42A
:10FEA000D0F190FEB01200382290FEB51200382238
:0EFEB0004F6B0D0A004661696C65640D0A0017
:10FF0000A5E5E0A5FE59000000000000000000008B
:10FF1000000000000000000000000000FFFFFFFFE5
:10FF20004572617365204320436F646520616E6490
:0FFF3000204472697665727320202027592700BC
:10FF400090FF40120FE09020007424120067902070
:10FF500000E493F4700CA3E58270F6E583B430F10D
:04FF6000C140C1A932
:10E80000A5E5E0A5FE4600000000000000000000B5
:10E81000000000000000000000000000FFFFFFFFFC
:10E820004D656D6F727920456469746F722028564A
:06E83000543130302900D4
:10E840007C0051C4ECC2E3FCB1573112B41B02612D
:10E850008AB40B024126B40A02414DB40802416851
:10E86000B415024197B40C0451C40144B4110261BF
:10E870008AB4030FEC54FEFC71CC90ED4DD1EA51FB
:10E88000DF0144B4040FEC4401FC71CC90ED52D193
:10E89000EA51DF0144B4070221E4B4050221D8B4EF
:10E8A0000602214EB4010FEC30E199D2E2FC915006
:10E8B0009160711E0144B4180FEC30E187C2E2FC94
:10E8C00091509160711E0144B419024143B41A027F
:10E8D0004148F5F0EC20E102014430E20EE5F07130
:10E8E00095B5F0F48F838E82F04197E5F0B1D2D1E7
:10E8F0005B40E5F88F838E82EC20E30AE8FDECD2E2
:10E90000E3FC711E0148EDC454F028F0ECC2E3FCB6
:10E910004197C0E0EC20E106C2E3FCD0E02230E306
:10E92000F9D0E0C0E0B1D2D15B50F0D0E0C0E0B4AB
:10E930001B0EECC2E3FC711ED0E0D0E0D0E001443D
:10E940008F838E82EDF0ECC2E3FC711E80CDEC541F
:10E9500002700201449150ECC0E090E9B2D1EAB1FA
:10E96000DF404420D541A882A98390E9C7D1EAB10C
:10E97000DF403420D531AC82AD8390E9D0D1EAD1EB
:10E9800075402420D521FAECFEEDFFD0E0FC888212
:10E990008983EAF0EEB5820CEFB58308915091605F
:10E9A00051DF0144A380EBD0E0FC91509160711ED7
:10E9B000014446696C6C204D656D6F72793B204651
:10E9C000697273743A200020204C6173743A2000FD
:10E9D00020776974683A20009150EC6402FC9160E1
:10E9E000711E0144915090EA14D1EAECC0E0B1DF0D
:10E9F000D0E0FC401320D510AE82AF8371CC7414EC
:10EA000071D2916051DF014471CC741471D2916064
:10EA1000711E01444D656D6F7279204C6F63617496
:10EA2000696F6E3A2000714AEEC39410FEEF9400B5
:10EA3000FFEEF454F06008740171DA71660144511C
:10EA4000DF01441F51DF01440F51DF0144714AEEE1
:10EA50002410FEEF3400FFEE54F06008740171D210
:10EA60007166014451DF0144714A740371E2EEC3DF
:10EA70009401FEEF9400FFEE44F0F460047166012F
:10EA800044EEF454F0600C743071EA740171DA7180
:10EA900066014451DF0144714A740371EA8E828F2A
:10EAA00083A3AE82AF83EE540F600471660144EE1F
:10EAB00054F0600C743071E2740171D271660144DB
:10EAC00051DF014490ECF8D1EA9137D1FE9115D194
:10EAD000FE912ED1FE741071D2912ED1FE916071F3
:10EAE000CC740271D27582008F837810D1FED1CBA5
:10EAF000743AD1C3AA82AB83D1C171A7D1D8A3E59F
:10EB000082540F70F38A828B83D1C1D1C1D1C1717C
:10EB1000A77195D1C3A3E582540F70F3D8CE71CC01
:10EB2000EEC4540F240371D2EE540F243871EA71ED
:10EB3000F271B07195D1C371FEEE540F23F42434F9
:10EB400071E271F271B0D1D861FEEE540F23F4245A
:10EB50003171EA71B07195D1C3EE540F23F42434AE
:10EB600071E271B0C1D8EE540F23F4243171EA710F
:10EB7000B0719571F2D1C371FEEE540F23F42434B9
:10EB800071E271B071F2D1D861FEEE54F0C4F42498
:10EB90001371D2C1FE547FB47F03742022C394202A
:10EBA00050027400242022EC20E003E49322E022AF
:10EBB000C083C0828F838E82EC20E30D20E004E4CA
:10EBC000938001E0D082D08322ED80F891087448D0
:10EBD000C1C39108F1117442C1C39108F11174418C
:10EBE000C1C39108F1117444C1C39108F111744378
:10EBF000C1C390EBF7C1EA1B5B303B376D0090EC73
:10EC000003C1EA1B5B306D00C0E0741BD1C3745BB1
:10EC1000D1C3D0E02290ED00D1EA7800D1C1742BAD
:10EC2000D1C3E8D1DB08B810F390ED06C1EA78480B
:10EC3000742DD1C3D8FA22EC20E00590ED4D80036D
:10EC400090ED52D1EA7808D1C1D8FC90ED1AC1EA12
:10EC500071CC741471D27A48D1C1DAFC744861E283
:10EC6000EC30E11290ECB820E20390ECD3D1EA90C2
:10EC7000ECEED1EA800590ECB0D1EA90EC80C1EAEC
:10EC800020205E473D476F746F20205E433D436FF9
:10EC9000646520205E443D4461746120205E4C3DEB
:10ECA00052656472617720205E513D517569740030
:10ECB0005E452D45646974005E413D1B5B303B370A
:10ECC0006D41534349491B5B306D20205E583D48E0
:10ECD0006578005E413D415343494920205E583DDF
:10ECE0001B5B303B376D4865781B5B306D00202027
:10ECF0005E463D46696C6C001B5B481B5B324A00FC
:10ED0000414444523A002020204153434949204580
:10ED100051554956494C414E540038303531204503
:10ED2000787465726E616C204D656D6F72792045E7
:10ED30006469746F722C205061756C2053746F6617
:10ED400066726567656E2C203139393600434F4451
:10ED500045004441544100309805D1B9B41B4DD110
:10ED6000B9B41B48B1BF209803741B22D1B9B45B5E
:10ED700042B1BF3098E1D1B9B44103740B22B4421F
:10ED800003740A22B44303741522B44403740822A2
:10ED9000B435028007B4360280028017C0E0B1BFEC
:10EDA00030980AD1B9B47E09D0E024E422D0E080C2
:10EDB000A6D0E0B1BF30989FD1B9B41BF680A5EAC8
:10EDC000C0E07A14E58C2098050470FADAF6D0E0F9
:10EDD000FA22B461004007B47B00500224E0227A9A
:10EDE000007B007C04C2D5B157B1D2B41B07D3E479
:10EDF000F583F58222B408028003B47F0CBC0402C0
:10EE000080E5D1C3D14A0C80DEB40D108B838A8299
:10EE1000BC0407E4F583F582D2D5C322FDD15B4063
:10EE2000C6CD12EEC3EDC0E0D139D0E02AFAE43B02
:10EE3000FBDCB4C38A828B8322EBC454F0FBEAC4AC
:10EE4000540F4BFBEAC454F0FA22EAC4540FFAEB15
:10EE5000C454F04AFAEBC4540FFB2224D0501424BB
:10EE6000F64004240AC32224F9500824FA4004245A
:10EE700010C322D322C2D5B157B1D2B41B03D3E4FD
:10EE800022B40D05D2D5C3E422FAD15B40E9CAD140
:10EE9000C3B157B1D2B41B0280E4B40D03EAC3225C
:10EEA000B40804D1C380D0B4150280F7FBD15B4015
:10EEB000E0CBD1C3EAC44BC3223098FDC298E59998
:10EEC0002274203099FDC299F59922C0E0E583D1E2
:10EED000D8E582D1D8D0E022D1DAC4C0E0540F24E2
:10EEE00090D43440D4D1C3D0E022C0E0E493A360F6
:10EEF0000AA2E7547FD1C3400280F1D0E022C0E0F3
:10EF0000740DD1C3740AD1C3D0E022C0F0C0E08038
:10EF100013C0F0C0E030E70C742D12EEC3D0E0C097
:10EF2000E0F4240175F06484D2D56007C2D52430A2
:10EF300012EEC3E5F075F00A8430D5026005243086
:0FEF400012EEC3E5F0243012EEC3D0E0D0F02281
:10F00000A5E5E0A523FF00000000000000000000CF
:10F01000000000000000000000000000FFFFFFFFF4
:10F020004D503320506C617965722C2056657220EA
:10F03000302E312E3220284E6F2053494D4D29005D
:10F0400075815090FB09120038E4F521F50BF54469
:10F05000F542F54371E34510F50A90FBC7120038FD
:10F06000903040120FE0403190FBEE12003890FBE0
:10F07000FC120038F1E690FC131200389030431275
:10F080000FE0401590FBEE120038D20D90FC3912C3
:10F090000038F1FE12004801A190FBF31200386124
:10F0A000BC750F00750E00750D00750C0090F99D74
:10F0B000120038F19C12F82A12F89490FDFEE0B488
:10F0C000553DA3E0B4AA3890FDC2E011F150523191
:10F0D0000D90FDD2E011F15048310D90FDE2E011AC
:10F0E000F1503E310D90FDF2E011F15034310D61DF
:10F0F000BC24F5600824FF6004240CD322C3221230
:10F10000F83C12004890F9BA12003861BCC0E09097
:10F11000F9D4120038D0E012003412004822E0A3E3
:10F1200022A3A3A3A3311EF514311EF515311EF53C
:10F1300016311EF517311EF518311EF519311EF561
:10F140001A311EF51B90F9ED120038781491D41283
:10F150000048216212F83C90FA2712003812F83C5D
:10F1600061BC90FA0D12003885140C85150D8516BA
:10F170000E85170FF19C12F82A12F89490FDFEE00C
:10F18000B455D1A3E0B4AACC90FC0BE070C6A3E0C8
:10F19000B402C190FC10E0B402BA90FA62120038D6
:10F1A000C390FC24E033FAA3E033FBA3E033FCA3D9
:10F1B000E033FD90FAB1120038780291D412004881
:10F1C00090FC0EE0F53CA3E0F53D90FACF1200383C
:10F1D000E53D120034E53C120034120048EA253CBB
:10F1E000F51CEB353DF51DEC3400F51EED3400F556
:10F1F0001FE51C2514F51CE51D3515F51DE51E350F
:10F2000016F51EE51F3517F51F90FA3D12003878E8
:10F210001C91D412004890FC0DE0F50990FA771289
:10F220000038E50912003412004890FC2CE0F52863
:10F23000A3E0F529A3E0F52AA3E0F52B90FA8D12BF
:10F240000038782891D4120048414B90FBA8120056
:10F2500038C20AC20BC209852824852925852A2699
:10F26000852B27752200752300D16BE530600ED108
:10F27000E750065186400251A8517F50EC414B2087
:10F280000B02A1AFA1E9200E02C3221546E546609C
:10F2900002D322E5457003F4F54554B8A2D0E54504
:10F2A00033F54514F546C32290FA59120038F1108F
:10F2B000C20AC20BC209D208AA2CAB2DAC2EAD2FAC
:10F2C000B150F15FF19C712812F82A12F89490FF66
:10F2D00031F090FF37F090FF33F0300D0271627122
:10F2E000414020200A1D200B1A20092AF19C712878
:10F2F0009112750808717D20B2F875080990FF37E2
:10F30000F080C575080A717D20B2F875080B90FF72
:10F3100037F0120048229112200AD1200BCE20088B
:10F32000CB3009C8717D80EEE50C2401F50CE50DAC
:10F330003400F50DE50E3400F50EE50F3400F50F41
:10F3400022C3E5109401F510E5119400F511E512C2
:10F350009400F512700AE5107006E5117002D322D0
:10F36000C3227864D8FE7C147B0090304F120FE0EB
:10F370007C727B0190304F120FE0C20D2220980169
:10F3800022120032120040120030FA90FCCA780BB0
:10F3900071CC500361BC2290FCD4784271CC5003F4
:10F3A000915B2290FCD9784371CC500391642290F8
:10F3B000FCCF784471CC500391422222F1DB120041
:10F3C00048E50812003412004802006DE60493C3B9
:10F3D0009A700C06E493C3966002C322F6D3227699
:10F3E00000C322C29400D29474FFA296C29533D275
:10F3F00095A296C29533D295A296C29533D295A284
:10F4000096C29533D295A296C29533D295A29633E1
:10F41000F42271E3B50A0122850AF0F50A30E4030B
:10F4200030F41F30E10330F13230E50330F5353090
:10F43000E30330F33830E00330F05030E20330F2D1
:10F440006B2220080B90FC82120038D208C20922DD
:10F4500090FC89120038D209C2082290FC91120057
:10F4600038D20A2290FC9D120038D20B2290FCADBB
:10F47000120038B20E200E0B7466120030120030EB
:10F48000020048746E12003002004890FCB6120070
:10F49000387C4690304C120FE0EB60011B90304FEF
:10F4A000120FE07C4890304F120FE02290FCBF1208
:10F4B00000387C4690304C120FE0EB249E40010B4C
:10F4C00090304F120FE07C4890304F120FE02274C2
:10F4D00020020030080808E612003418E612003452
:10F4E00018E612003418E612003422EAC0E033EBCA
:10F4F00033FAEC33FBED540F33FCE433FDEA253CE7
:10F50000FAEB353DFBEC3400FCED3400FDEA25144C
:10F51000FAEB3515FBEC3516FCED3517FD8A0C8B37
:10F520000D8C0E8D0FF19C12F82A12F894D0E05435
:10F530007FC33333FAE433FB74002AF58274FC3B57
:10F54000F583E0FAA3E0FBA3E0FCA3E0540FFD2267
:10F55000C3EA9402F50CEB9400F50DEC9400F50E63
:10F56000ED540F9400F50FA809E8C313F86017C312
:10F57000E50C33F50CE50D33F50DE50E33F50EE531
:10F580000F33F50F80E3E50C251CF50CE50D351D5B
:10F59000F50DE50E351EF50EE50F351FF50F22C3EF
:10F5A000EA94F8EB94FFEC94FFED540F940F22E5EE
:10F5B0002304540FF5237021AA091AE522045AF5F1
:10F5C000227016AA24AB25AC26AD2791EBB19F5033
:10F5D0000A8A248B258C268D27C3228528248529F9
:10F5E00025852A26852B27D322E52314540FF523BE
:10F5F00044F0F47010AA091AEAF4FBE522145AF553
:10F60000224BF46002C32285FF3E85FF3F85FF4009
:10F61000850F41AA28AB29AC2AAD2BEAB5240EEB05
:10F62000B5250AECB52606EDB5270280108A3E8B7B
:10F630003F8C408D4191EBB19F501C80DEAA3EABC8
:10F640003FAC40AD41B19F500E853E24853F25859E
:10F65000402685412780AE852824852925852A26B0
:10F66000852B27752200752300D322AA24AB25AC55
:10F6700026AD27B150E50C2522F50CE50D3400F53B
:10F680000DE50E3400F50EE50F3400F50FF19C1278
:10F69000F82A12F894E523540FC4C333FAE433FB79
:10F6A00074002AF58274FC3BF5837830E0A3F608F9
:10F6B000B83BF9E0F53BE5822409F582E5833400A7
:10F6C000F583E0A3F52EE0A3F52FA3A3A3A3E0A366
:10F6D000F52CE0A3F52DE0A3F510E0A3F511E0A3D0
:10F6E000F512E0A3F51322E5306023241B601FE52B
:10F6F0003B20E11A20E21720E31420E411E538B49E
:10F700004D0CE539B45007E53AB43302D322C32295
:10F710007830E612003008B838F8742E120030E65F
:10F7200012003008B83BF890FAE2120038E53B12BC
:10F73000003490FAF0120038782C91D490FB01122A
:10F740000038781091D4120048782491D491CFE5F4
:10F750002212003491CFE52312003412004822AA6D
:10F7600010E5115401FBC3E51313F513E51213F56E
:10F7700012E51113F51185111085121185131275FB
:10F780001300EA7004EB700122E5102401F510E586
:10F79000113400F511E5123400F5122212F81B9015
:10F7A000FF16E50F540F44E0F090FF15E50EF090C2
:10F7B000FF14E50DF090FF13E50CF090FF127401BB
:10F7C000F090FF177420F02290FF11749AF090FFD0
:10F7D000127401F090FF1774EFF02290FF1774E697
:10F7E000F090FF17E02290FF3274FFF07800D8FE0F
:10F7F000D8FED8FE7400F0D8FED8FED8FE2290FFC6
:10F800001674A0F090FF17E0C0E0742E12003012C2
:10F81000F37DD0E030E6E720E7E42290FF17E0C078
:10F82000E012F37DD0E020E7F22290FF17E0C0E085
:10F8300012F37DD0E020E7F230E3EF22C0E0C08297
:10F84000C083E8C0E0E9C0E090FC5E120038782098
:10F8500090FC007910E0A312003412F4CFD9F6C363
:10F86000E5829410F582E5839400F5837910E0A396
:10F87000547F24E0400274002420120030D9EF129B
:10F880000048D8CF120048D0E0F9D0E0F8D083D0BB
:10F8900082D0E022E490FF31F090FF30E0E0E0E041
:10F8A000E0E0E0E0E0E0E0E0E0E0E0E0E0E0E0E058
:10F8B000E0E0E0E0E0E0E0E0E0E0E0E0E0E0E0E048
:10F8C000E0E0E0E0E0E0E0E0E0E0E0E0E0E0E0E038
:10F8D000E0E0E0E0E0E0E0E0E0E0E0E0E0E0E0E028
:10F8E000E0E0E0E0E0E0E0E0E0E0E0E0E0E0E0E018
:10F8F000E0E0E0E0E0E0E0E0E0E0E0E0E0E0E0E008
:10F90000E0E0E0E0E0E0E0E0E0E0E0E0E0E0E0E0F7
:10F91000E0E0E0E0E0E0E0E0E0E0E0E0E0E0E0E0E7
:10F92000E0E0E0E0E0E0E0E0E0E0E0E0E0E0E0E0D7
:10F93000E0E0E0E0E0E0E0E0E0E0E0E0E0E0E0E0C7
:10F94000E0E0E0E0E0E0E0E0E0E0E0E0E0E0E0E0B7
:10F95000E0E0E0E0E0E0E0E0E0E0E0E0E0E0E0E0A7
:10F96000E0E0E0E0E0E0E0E0E0E0E0E0E0E0E0E097
:10F97000E0E0E0E0E0E0E0E0E0E0E0E0E0E0E0E087
:10F98000E0E0E0E0E0E0E0E0E0E0E0E0E0E0E0E077
:10F99000E0E0E0E0E0E0E0E0E0E0E0E022526561AD
:10F9A00064696E67204D617374657220426F6F7475
:10F9B000205265636F72640D0A004D4252205369F4
:10F9C000676E6174757265204E6F7420466F756E38
:10F9D000640D0A00556E6B6E6F776E205061727405
:10F9E0006974696F6E20547970653A2000466F75AE
:10F9F0006E642046415433322050617274697469D8
:10FA00006F6E206174204C4241203D2000526561A0
:10FA100064696E6720464154333220566F6C756DB1
:10FA2000652049440D0A0042616420464154333246
:10FA300020566F6C756D652049440D0A0046697249
:10FA40007374204461746120536563746F72206124
:10FA500074204C4241203D20005C5B506C61793A3F
:10FA60002000566F6C756D65204944206C6F6F6B7C
:10FA700073206F6B0D0A00536563746F727320708F
:10FA8000657220636C75737465723A2000526F6FF3
:10FA900074206469726563746F7279207374617223
:10FAA000747320617420636C7573746572202320F5
:10FAB00000536563746F7273207573656420666F9D
:10FAC0007220464154207461626C65733A20005282
:10FAD0006573657276656420536563746F72733AFB
:10FAE00020000D0A5C5D20204174747269623D0043
:10FAF000202046697273745F436C75737465723D40
:10FB000000202053697A653D000D0A0D0A0D0A5C3C
:10FB10005B5C4020304D503320506C617965722C15
:10FB20002056657273696F6E20302E312E325C5D07
:10FB30000D0A4D503320506C617965722C2056654A
:10FB40007273696F6E20302E312E322C204D617908
:10FB500020322C20323030310D0A436F70797269B7
:10FB60006768742028432920323030302C20504AD6
:10FB700052432E434F4D2C204C4C430A0D0A0D543A
:10FB80007970652027515549542720746F2072657C
:10FB90007475726E20746F20746865206D6F6E6965
:10FBA000746F720D0A0D0A000D0A4D503320506C0F
:10FBB000617965722C20426567696E20506C6179AD
:10FBC0006261636B0D0A00436F6E666967757269E7
:10FBD0006E672058696C696E7820584353313058ED
:10FBE0004C204650474120436869703A20004F6BD3
:10FBF0000D0A004572726F72210D0A00526573651D
:10FC000074696E672049444520446576696365736D
:10FC10000D0A00436F6E6669677572696E672053DF
:10FC20005441303133204D5033204465636F646557
:10FC30007220436869703A200057616974696E6781
:10FC400020666F7220486172642044726976652074
:10FC5000746F2062652072656164790D0A000D0A77
:10FC600043757272656E7420536563746F722042BF
:10FC7000756666657220436F6E74656E74733A0DB7
:10FC80000A00506C61790D0A0050617573650D0AA8
:10FC9000004E6578742046696C650D0A00507265E7
:10FCA00076696F75732046696C650D0A0052616E46
:10FCB000646F6D204F00566F6C2055700D0A005612
:10FCC0006F6C20446F776E0D0A000451554954043F
:10FCD000504C4159044E4558540850524556494FCE
:02FCE00055537A
:020000021000EC
:032000000230406B
:032003000221D5E2
:01200B0032A2
:032013000221FDAA
:01201B003292
:0320230002204454
:03202B0002223757
:10202E00210901A101E52106212721342118213F93
:10203E004113617501E1C0D0C0E020980820992BB2
:10204E00D0E0D0D032C298E51604B51707E599D086
:10205E00E0D0D032F516C082C083758381F582E55B
:10206E0099F0D083D082D0E0D0D032C299E528B595
:10207E002707C21DD0E0D0D03204F528C082C0831D
:10208E00758382F582E0F599D083D082D21DD0E09F
:10209E00D0D032C0D0C8C0E0752B00C2AF201D0911
:1020AE00D299E4F527F528D21DE52704B5280AD2E2
:1020BE00AF052BE52B70E480E7F527C083C0827552
:1020CE008382F582C8F0D082D083D2AFC8D0E0C868
:1020DE00D0D022201DFD22C2ACE517B51605E4D2E4
:1020EE00ACD32204F517C082C083F582758381E0DC
:1020FE00D083D082D2ACC3223108C4C0E0540F24A6
:10210E0090D43440D411A1D0E022C0E0740D12203E
:10211E00A1740A1220A1D0E022C0E0E5833106E5C9
:10212E00823106D0E022E493A360051220A180F64E
:10213E00227800D8FED8FEC2AF43878053890F4362
:10214E008920C28EC28F74FEF58DF58B75985075F1
:10215E002700752800C21DD28ED2ACD2AF22E490D9
:10216E00FF5DF0E51EB51D0F74FFF51EF51DD0E0E9
:10217E00D083D082D0D03204B43C01E4F51E2323A8
:10218E002400F582E43483F583E0FAA3E0FBA3E0B8
:10219E00FCA3E0FD90FF12EAF0A3EBF090FF28E421
:1021AE00F0A37490F090FF2AECF0A3EDF0E490FF12
:1021BE0059F0908004E02401F0A3E03400F0D0E068
:1021CE00D083D082D0D032C0D0C082C083C0E07560
:1021DE00D00890FF50E020E185D0E0D083D082D0AF
:1021EE00D03290FF5CF0D0E0D083D082D0D032C01D
:1021FE00D0C082C08375D008FF90FF6EE0EFD08311
:10220E00D082D0D032C2AD75C80075CA0075CBD0A1
:10221E0075CC0075CDD0C215C216C217C21875295D
:10222E0000752A00D2ADD2CA22C0D075D008FFAE3A
:10223E0082AD83C2CFC29400D2940020960D301787
:10224E0002800AD217740371758002C217C295D22A
:10225E009520960D301602800AD216740271758082
:10226E0002C216C295D29520960D301802800AD25F
:10227E0018740471758002C218C295D295209614F6
:10228E00052AE52A14600724F4500C752A017406F9
:10229E0071758003752A00C295D29520960D301562
:1022AE0002800AD215740171758002C215C295D2D0
:1022BE00952096140529E52914600724F4500C7511
:1022CE002901740571758003752900908023E0241F
:1022DE00FC40062405F002236DE4F03019189080BE
:1022EE0024E024FFF0F8A3E034FFF07009E8700654
:1022FE00C219740A7175301A18908026E024FFF006
:10230E00F8A3E034FFF07009E87006C21A740B717E
:10231E0075301B18908028E024FFF0F8A3E034FFFE
:10232E00F07009E87006C21B740C7175301C1890A1
:10233E00802AE024FFF0F8A3E034FFF07009E87083
:10234E0006C21C740D717590802CE02401F0500FA4
:10235E00A3E03400F0A3E03400F0A3E03400F08DED
:10236E00838E82EFD0D032F8E51004B44001E4B58C
:0F237E00110122F51024C0F582758380E8F0224A
:10300000A5E5E0A500FF00000000000000000000B2
:10301000000000000000000000000000FFFFFFFFB4
:103020004861726477617265204472697665727373
:01303000009F
:103040000231F50232FF02349402327D0233AD02C6
:1030500033B502501A024F60024E8D026540024E97
:10306000CA024E77024EA40250EE02528C02545B0A
:103070000200000252ED0254EB0256360234F10215
:1030800036940236870235C6023631023657023789
:103090007102377B0236B20237A5023A06023A5A6B
:1030A000023B700242EE0244DC024A99024B2602C5
:1030B00042140248B80234E502349F0234C4024488
:1030C00010024B6002659B02654E0000000230EE6C
:1030D00002360C0239D502312802317802319002D1
:1030E00031DC0233EE0245DF0247A5024474E4F509
:1030F000A875B81075B800F522F510F51191E845DE
:1031000010F5129080247808E4F0A3D8FC90802C6D
:103110007804E4F0A3D8FC908023F0C219C21AC24C
:103120001BC21CD21F020FF0EC7011908024EAC267
:10313000AFF0A3EBF0D219D2AF020FF0B4011190AF
:103140008026EAC2AFF0A3EBF0D21AD2AF020FF0A2
:10315000B40211908028EAC2AFF0A3EBF0D21BD2E8
:10316000AF020FF0B4030E90802AEAC2AFF0A3EBD7
:10317000F0D21CD2AF020FF0EC232424F582758329
:1031800080C2AFE0A3FBE0D2AF8B82F583020FF0E9
:10319000EC7010908024E4C2AFF0A3F0C219D2AF5B
:1031A000020FF0B40110908026E4C2AFF0A3F0C289
:1031B0001AD2AF020FF0B40210908028E4C2AFF030
:1031C000A3F0C21BD2AF020FF0B4030D90802AE42B
:1031D000C2AFF0A3F0C21CD2AF020FF090802CC29D
:1031E000AFE0A3F8E0A3F9E0A3F5F0E0D2AF898364
:1031F0008882020FF090CFFF5172B4FF795172B400
:1032000004745172B4E86F5172B4FA6A5172B4F92D
:103210006512006AD8FED8FED8FE7899D8FED297FB
:10322000D29590D000E493A3139297C295D29513B0
:103230009297C295D295139297C295D29513929771
:10324000C295D295139297C295D295139297C29533
:10325000D295139297C295D295139297C295D29513
:10326000E582B4C0C0E583B4FEBBD297758200028C
:103270000FF0A3E49322D3758201020FF0909FFF19
:103280005172B4FFF15172B404EC5172B4E8E751D9
:1032900072B4FAE25172B4F9DD12006AD8FED8FEB7
:1032A000D8FE7899D8FED297D29590A000E493A347
:1032B000139297C295D295139297C295D295139275
:1032C00097C295D295139297C295D295139297C2B1
:1032D00095D295139297C295D295139297C295D293
:1032E00095139297C295D295E582B4C0C0E583B498
:1032F000CEBBD297758200020FF0742E022030519F
:10330000FA7C0171BF4009BBAC028012EB1256740B
:10331000742A1200307C0171BF402FBBAC2C51FAD3
:103320009090007174402351FA51FA715151FA7C16
:10333000147B0171DC4013D21E51FA7C727B017147
:10334000DC4007C3758200020FF0D3758201020FC3
:10335000F090900071A6EE54FEFE71A2FC71A2FBEB
:1033600071DCEC24FA70047DC8DDFEEEB582EBEF73
:10337000B583E72271A6E4F8F971A228F8E439F9D7
:10338000EEB582F5EFB583F171A288F0B5F0097161
:10339000A289F0B5F002C322D374211220300200BA
:1033A0000022E493A32271A2FE71A2FF2271BFE466
:1033B0003400020FF071DCE43400F582020FF0916A
:1033C000687486914F4013EC914F400E917591684F
:1033D0007487914F4004913BFBC38175916874865B
:1033E000914F4008EC914F4003EB914F81757E0166
:1033F00091687486914F40360E7440914F402F0E65
:10340000917591687487914F40240E913B9180F99A
:10341000913B9180913B9180913B9180F5F0913B64
:103420009180F583913BF5829175E9020FF09175DA
:1034300074FFF5F0F5838E82020FF0337D08D29190
:103440000000D2900000A2913300C290DDF3227DF3
:103450000833929100D29000C290DDF533D29100F2
:10346000D29000A291C29022D291D2900000C2913B
:103470000000C29022C2910000D2900000D291229E
:10348000C2910000D2900000C29022000000000013
:103490000000002278FAC2B5D2B5D8FA020FF0C205
:1034A000AFE511B51008D2AF758200020FF004B479
:1034B0004001E4F51124C0F582758380E0D2AFF5B8
:1034C00082020FF0C2AFE51004B44001E4B511056B
:1034D000D2AF020FF0F51024C0F582758380ECF0B6
:1034E000D2AF020FF0020FF0E42291E8F582020F52
:1034F000F0C02290623E12569AEB125671EA1256B2
:10350000711256F9125640A3A3A3A3E0A3C0E0E0B2
:10351000A3C0E0E0A3125671D0E0125671D0E012C1
:1035200056711256F9A3A3A3A3A3E0A3C0E0E0A39E
:10353000C0E0E0A3C0E0E0125671D0E0125671D0B6
:10354000E0125671D0E012567112565FD022C3EDD0
:1035500013FDEC133400FCED3400FDC2A8E51DB4EE
:10356000FF34E4F51DF51E1235E1D2A8201E0675C4
:103570008200020FF07C147B001233DC7864D8FEEA
:103580007C147B001233DC7C727B011233DCC21EA4
:10359000758200020FF004B43C01E4B51E08D2A805
:1035A000758201020FF0F51D23232400F582E43417
:1035B00083F583EAF0A3EBF0A3ECF0A3EDF0D2A83F
:1035C000758200020FF0C2A890FF2BE4F090FF2A52
:1035D00004F0E51DF46005E4F51EF51DD2A8020F08
:1035E000F090FF12EAF0A3EBF090FF28E4F0A37450
:1035F00090F090FF2AECF0A3EDF0E490FF59F090EA
:103600008004E02401F0A3E03400F022E490FF5CA9
:10361000F090FF5DF090FF5EF090FF517402F07546
:103620001DFF751EFF5388F0D2A8C2ACD2AF020FA7
:10363000F0C2A8A81EE51DD2A8B4FF07743BF5820E
:10364000020FF0C3985002243CF8743CC398600207
:1036500024FFF582020FF090642E12569AC2A8A899
:103660001DA91ED2A8E8125671742D125659E912DE
:10367000567112565FE8F46007C3758200020FF0BE
:10368000D3758201020FF0C2AF90FF517400F0D2E7
:10369000AF020FF0C2AF90FF517402F0D2AF020F31
:1036A000F0908004C2A8E0FCE4F0A3E0FDE4F0D2D6
:1036B000A8227A227B0074091252DBF122906469FD
:1036C00012003890FF28E4F0A37490F090FF2A7461
:1036D00008F0A37402F0E490FF59F07F007E0090A0
:1036E000FF50E020E106DEF70FBF50F390647C123C
:1036F0000038EF12003474201200307420120030B1
:10370000EF24D85011EF24C3400C905DC81200384C
:10371000758200020FF0905DD412003875820102AC
:103720000FF0909000745578D2F0A3F0A3F0A3F0BE
:10373000A3F0A3D8F490647FE581F8F92410F58113
:10374000097A0A7B0FE9F8E493A3F608DBF9C08352
:10375000C082E9F8E608F582E608F5837B0DE60805
:10376000F0A3DBFAD082D083DAD9E58124F0F581A9
:10377000227C461233BF8B82020FF0EB24C0500232
:103780007B407C461233DC7C481233DC020FF05362
:10379000544130313320617474656E756174696FA2
:1037A0006E203D200074011252FF74071252DB7527
:1037B0003700753600753500753400905AE712569B
:1037C0009D907000124F079071FEE0B45539A3E050
:1037D000B4AA349071C2E01239B3503B1239C1908F
:1037E00071D2E01239B3502F1239C19071E2E01258
:1037F00039B350231239C19071F2E01239B3501726
:103800001239C1E40239A1125087125662905B044A
:1038100012569DE40239A1A3A3A3A31239D2F53411
:103820001239D2F5351239D2F5361239D2F5379030
:103830008042E534F0A3E535F0A3E536F0A3E537A3
:10384000F0905B3712569D7834C022D21F12570178
:10385000D022125662023868125087905B7112565D
:103860009D125087E40239A1C022D21F905B5712EB
:10387000569D908042E0F534A3E0F535A3E0F5369F
:10388000A3E0F537907000124F079071FEE0B45539
:10389000C7A3E0B4AAC290700BE070BCA3E0B4026E
:1038A000B7907010E0B402B0905BB212569DC39016
:1038B0007024E033FAA3E033FBA3E033FCA3E0334E
:1038C000FD905CC312569D78021257011256629009
:1038D000700EE0FEA3E0FF908042E02EF534A3E0FE
:1038E0003FF535A3E03400F536A3E03400F537901A
:1038F000803CE534F0A3E535F0A3E536F0A3E537E9
:10390000F0E5342AF534E5353BF535E5363CF5365A
:10391000E5373DF537908038E534F0A3E535F0A381
:10392000E536F0A3E537F0905B8712569D783412A8
:10393000570112566290700DE0F53B54F8C423F520
:103940001FE53B54076008051F905C4512569D908B
:103950005BC712569DE53B1256B5905BD812569D3B
:10396000E51F1256B5905C1A12569D90702CE0F52A
:1039700030A3E0F531A3E0F532A3E0F533908032D7
:10398000E530F0A3E531F0A3E532F0A3E533F090A4
:103990005CA112569D7830125701125662D02274E3
:1039A00001C0E090FF0EE0FAA3E0FB1254F1D082D8
:1039B000020FF024F5600824FF6004240CD322C316
:1039C00022C0E0905B1E12569DD0E0125674125633
:1039D0006222E0A322908032E0C0E0A3E0C0E0A336
:1039E000E0F5F0A3E0D083D082020FF0543F75F0F1
:1039F00018A42400F582748A35F0F583222582F517
:103A0000825002058322905FE012569A7900E912F3
:103A100039ECE05401600E09B940F3905DD41256C0
:103A20009A7582FF227401F0E47E17A3F0DEFCE9B0
:103A30001239EC740C1239FDEAF0A3EBF0A3ECF0B0
:103A4000A3EDF0E91256B29061B212569A780212C2
:103A5000570112565F8982020FF0883089318A320D
:103A60008B338C348D358E368F377830793485F0C2
:103A700026905FEB12569AE5261256B2905FFB1223
:103A8000569A12570190600412569AE627FA0809CE
:103A9000E6F53837FD0809E6F53937FE0809E6F599
:103AA0003A37FFEA24FFFAED34FFFDEE34FFFEEF74
:103AB00034FFFF780512571BEA12567112565FAA9F
:103AC0003BC3E53A13F53AE53913F539E53813F513
:103AD00038C3EF13FFEE13FEED13FDEAC313FA70C4
:103AE000E090600912569A783812571B90600412C1
:103AF000569A780512571B12565FE5261239ECE0EC
:103B00004402F0A3A3E538F0A3E539F0A3E53AF0C9
:103B1000A3EDF0A3EEF0A3EFF0A3E0FAA3E0FB7EA9
:103B2000007F00EB7003EA6025125640A3A3A3A315
:103B3000C3E09538A3E09539A3E0953A5010EAFE2A
:103B4000EBFFA3A3E0FAA3E0FB70DEEA70DB906179
:103B50002612569A780612572212565FE526123917
:103B6000EC740A1239FDEEF0A3EFF0C214020FF06C
:103B700090616E12569AEC125671742C125659ECD2
:103B8000F526A81F08AC1AAD1BECF46017F404B4BA
:103B90007801E4B5050C90637912569A758200029B
:103BA0000FF0D8EAE5261239ECE020E10675820133
:103BB000020FF0740A1239FDE0F52CA3E0F52D7028
:103BC0003EE52C703AA3E0F530A3E0F531A3E0F533
:103BD00032A3E0F533E4F538F539F53AE526123944
:103BE000EC74081239FDE0F52EA3E0F52F90617812
:103BF00012569A90617C12569A12565F023C43907C
:103C0000617C12569A743D125659782C1257221222
:103C1000565FAA2CAB2D125640A3A3A3A3E0F53800
:103C2000A3E0F539A3E0F53AA3A3E0F52EA3E0F570
:103C30002FA3A3A3E0F530A3E0F531A3E0F532A371
:103C4000E0F53390618112569A78301257019061F5
:103C50008E12569A783812571B90619A12569AE52E
:103C6000261239ECA3A3E0C0E0A3E0C0E0A3E01279
:103C70005671D0E0125671D0E012567112565FE5BF
:103C800033B40F0FE5261239ECE054FDF0758201D4
:103C9000020FF0E5261239ECA3A3AE82AF83E0B5A4
:103CA000380CA3E0B53907A3E0B53A02A1208E8213
:103CB0008F83C3E0A39538E0A39539E0A3953A50EC
:103CC00009903CEE12569D02576EE5382401F538F6
:103CD000E5393400F539E53A3400F53A123F0BB4D2
:103CE00001028143B402028060F582020FF00D0AE6
:103CF0004572726F723A20436C7573746572206FEF
:103D00006666736574203E20746172676574206313
:103D10006C7573746572206F66667365740D0A0046
:103D20009060BA12569A78301257019060C21256BB
:103D30009A783812571B742912565912565FE51F8C
:103D40001252FF8A068B0750159063AE12569DE5FE
:103D5000261239ECE054FDF0758202020FF0C3E543
:103D6000309402F534E5319400F535E5329400F5F0
:103D700036E533540F9400F537A83BE8C313F860D9
:103D800017C3E53433F534E53533F535E53633F52A
:103D900036E53733F53780E3908038E02534F53465
:103DA000A3E03535F535A3E03536F536A3E03537F4
:103DB000F537E52C7015E52D7011E5261239EC74F8
:103DC000081239FDEEF0A3EFF0801AAA2CAB2D12E9
:103DD000564074081239FDEEF0A3EFF012562BEAAC
:103DE00070EDEB70EAAA06AB07A91F9061A212560C
:103DF0009A78021257229061B212569A783012576E
:103E0000019061B712569A783812571B9061BC1214
:103E1000569A782E12572212565F125640A3A37458
:103E200083F0A3A3E538F0A3E539F0A3E53AF0A3C6
:103E3000E51FC399F0A3E52EF0A3E52FF0A3E4F06E
:103E4000A37410F0A3E530F0A3E531F0A3E532F060
:103E5000A3E533F0E51AB4FF05E4F51AF51B04B445
:103E60007801E4F51A75F008A42400F582E5F03431
:103E700084F583E534F0A3E535F0A3E536F0A3E55A
:103E800037F0A3EAF0A3EBF0A3E4F0A3F019E960A4
:103E90001E12562BE5342408F534E5353400F5358B
:103EA000E5363400F536E5373400F537023DEBE50D
:103EB000261239ECA3A3A3A3A3E0A3B53818E0B559
:103EC0003914A3E0B53A0FE5261239ECE054FDF0C1
:103ED000758201020FF0E5382401F538E539340028
:103EE000F539E53A3400F53AE5261239ECA3A3E5B5
:103EF00038F0A3E539F0A3E53AF0A3A3A3A3A3A365
:103F0000EEF0A3EFF0758200020FF090601B1256E6
:103F10009A783012570112565FE5313354F8F53470
:103F2000E53233F535E53333F536E433F537908054
:103F300006E0B53421A3E0B5351CA3E0B53617A3E0
:103F4000E0B5371290800CE0B5260B90800AE0FABD
:103F5000A3E0FB023FE690602A12569A783412578B
:103F60000112565F12425F500302401590603A12F0
:103F7000569A7802125722C3EA33F582EB3324D0E3
:103F8000F583E0FAA3E0FB90605312569A78021290
:103F9000572212565F125640A3A3E030E704D21412
:103FA000E422A3A3A3A3A3A3E5265438C423123970
:103FB000FDE526540724028380080102040810202E
:103FC0004080F9E049F0908006E534F0A3E535F053
:103FD000A3E536F0A3E537F090800AEAF0A3EBF012
:103FE00090800CE526F0740B1252DBC3E53033FAF7
:103FF000E531540333FBC3EA33F582EB3324B0F5E8
:1040000083E0F530A3E0F531A3E0F532A3E0540FEF
:10401000F53374012290605A12569AA818A919E82B
:10402000F4600C08B818027800E9B50002E42290A8
:104030008002E0FD2401A3E0FE340054F860037424
:104040000222C002C003C005C00674011252FF8ADA
:10405000148B15D006D005D003D002500374022271
:104060009060CC12569A780512572212565F9060D3
:10407000F912569A780212572212565F90607D12FA
:10408000569AC3ED33F582EE3324D0F583E58224CE
:10409000FEF582E58334FFF583C3ED9AFDEE9BFECA
:1040A000ED7003EE6026742E125659E0F8A3E0F985
:1040B000A3E8F0A3E9F0E58224FBF582E58334FF71
:1040C000F583ED24FFFDEE34FFFE80D412565FC36E
:1040D000EA33F582EB3324D0F583E514F0A3E5153C
:1040E000F0908002E02401F0A3E03400F0AA14ABC9
:1040F00015125640A3A37482F0A3E4F0A3E534F0B4
:10410000A3E535F0A3E536F0A3E537F0A3E4F0A38B
:10411000F0A3F0A3F0A3F0A3F0A3F0A3F090803CF1
:10412000E02534F534A3E03535F535A3E03536F533
:1041300036A3E03537F537D214E518B4FF05E4F5BA
:1041400018F51904B41801E4B51902E422F518C4ED
:10415000032400F582E43489F583E534F0A3E535E2
:10416000F0A3E536F0A3E537F0A3E514F0A3E515D9
:10417000F0A3E4F0A3F0E422201F0122908002E0EB
:10418000FDA3E0FE90D000ED7003EE6060E0FAA3C6
:10419000E0FBA31256FC1256FC1256FC1256FC7899
:1041A000021257221256FC742D122030743E122037
:1041B00030C083C08212564074021241EE74011264
:1041C00041EE74011241EE74041241EE7408124182
:1041D000EED082D083ED24FFFDEE34FFFE1256FCBC
:1041E000EE125674ED125674125662809A22F8F945
:1041F0001256FCE0A3C0E0D8FAD0E0125674D9F908
:1042000022667265655F6661745F6D656D6F727958
:104210003A0D0A00908002E0F514E4F0A3E0F515F1
:10422000E4F090D000E5147004E515601FE0FAA3F7
:10423000E0FBA3C082C0831254F1D083D082E51486
:1042400024FFF514E51534FFF51580D99080067428
:10425000FFF0A3F0A3F0A3F090800CF0020FF09019
:104260008002E0FEA3E0FF7008EE7005E4FAFBD3E5
:1042700022EE24FFFEEF34FFFFE4FCFDC3EE9CFAC8
:10428000EF9DFBC3EB13FBEA132CFAEB3DFBC3EAF8
:10429000F51433F582EBF5153324D0F583E0FAA35A
:1042A000E0FB125640AA14AB15438207E0B5371A5B
:1042B0005382FEE0B536135382FC438201E0B535EC
:1042C000095382FEE0B53402C322500CEA2401FCFB
:1042D000FAEB3400FDFB800AEA24FFFEEB34FFFF1B
:1042E000500AC3EE9CEF9D400302427CD3228E26EF
:1042F0009061C312569A780212570112565F8A14BF
:10430000EBF51554F0C4F538EC540FC44238EC54B6
:10431000F0C4F539ED540FC44239ED54F0C4F53A08
:10432000E53B20E71220E61320E51720E41B20E3FD
:104330001F758201020FF07904801A53157F7903EB
:10434000801353153F7902800C53151F79018005A6
:1043500053150F8012C3E53A13F53AE53913F539D1
:10436000E53813F538D9EEE5261239ECA3A3A3A35B
:10437000A3A3A3A3E0FAFEA3E0FBFFEA7006EB70A1
:1043800003024404125640A3A3A3A3E0B5380CA330
:10439000E0B53908A3E0B53A04800DA3A3A3A3E0D8
:1043A000FAFEA3E0FBFF80D3E51553150F54F06030
:1043B00007C4F912562BD9FB9061DD12569A783852
:1043C00012571B9061EF12569A780612572290618D
:1043D000FE12569A780212572290620B12569A7861
:1043E0001412572212565FE5261239EC7410123956
:1043F000FDEAF0A3EBF0A3E514F0A3E515F0758258
:1044000000020FF090621712569A758201020FF0A7
:10441000EC1239EC74101239FDE0A3FAE0A3FBE0D2
:10442000A3F8E0540FFD125640A3A3A3A3E0F9A301
:10443000E0FAA3E0FB7E04E53B20E70F20E60D2039
:10444000E50B20E40920E307020FF00E0E0E0EC369
:10445000E933F9EA33FAEB33FBDEF4A3E0540FC39C
:10446000333333334D29F950010AEB8AF0898388BD
:1044700082020FF0ECF5261239EC74101239FD852A
:104480008232858333E0A3FAE0FB7009EA70067597
:104490008202020FF0125640A3A3E030E7067582B5
:1044A00001020FF0EE1252DB8A308B3112562BEAEA
:1044B0007014EB7011AA30AB3112564074081239E7
:1044C000FDE0FAA3E0FB853282853383EAF0A3EBBB
:1044D000F0A3E4F0A3F0758200020FF0C00191EAAE
:1044E000D0825003758200020FF0ECF5261239ECF1
:1044F00074101239FD858232858333E0A3FAE0A37C
:10450000FBE0A3FCE0540F44B0FD740B1252DB122D
:10451000564074021239FDE054806002D3228C822E
:104520008D83E0A3AC82AD838E828F83F0A3AE82B5
:10453000AF83ED54F024507004D9E380448A308B6B
:104540003112562BEA7019EB7016AA30AB311256A5
:104550004074081239FDE0FAA3E0FB7003EA60360C
:10456000740B1252DB7C007DB090630F12569A7868
:1045700002125722780412572212565F196002A1C4
:104580000F853282853383EAF0A3EBF0A3ECF0A32E
:10459000ED540FF0C322853282853383E4F0A3F01B
:1045A000A3F0A3F090644812569AD322C0D0E4340A
:1045B00030F974461256597463125659743D1256A6
:1045C00059E91256597420125659852C82852D832B
:1045D0007920E0125671A3D9F912565FD0D0220586
:1045E000A28E828F8305A2ECF5261239EC7410128C
:1045F00039FD85822E85832FE0A3FAE0A3FB7009A5
:10460000EA7006758202020FF0E0A3FCE0540F444A
:10461000B0FD740B1252DB125640A3A3E05480602D
:1046200006758201020FF08C828D837E00E060D3DC
:10463000241B601943820BE0543FB40F52A3E07077
:104640000CA3E0BE0003FF8006C39F60027EFF0E46
:10465000E58254E02420F582E5833400F58330D6EA
:10466000CCE58354F02430500912476E7582010264
:104670000FF012476E740C1252DB125640A3A3E0E7
:1046800054806006758201020FF090C000809E0584
:10469000A2F0A305A2BE000D752500740D05A2F0C1
:1046A000A305A280275382E0780BE403F9E029A355
:1046B000D8F9B507E3EE24EC500274FF2414F52575
:1046C000EE75F00DA40405A2F0A305A25382E04309
:1046D0008208E0A305A2F0A305A2E0A305A2F0A32F
:1046E00005A2E0A305A2F0A305A25382E043821A2B
:1046F000E0A305A2F0A305A2E0A305A2F0A305A2F2
:104700005382E0438214E0A305A2F0A305A2E0A334
:1047100005A2F0A305A25382E043821CE0A305A2F8
:10472000F0A305A2E0A305A2F0A305A2E0A305A2C1
:10473000F0A305A2E005A2F005A25382E0AE82AF8D
:1047400083908036EEF0A3EFF0EE2420FEEF3400ED
:10475000FF30D60712476E7E007F00852E82852FA0
:1047600083A3A3EEF0A3EFF0758200020FF0852E75
:1047700082852F83E0FAFCA3E0FBFD12562B701418
:10478000EA7011AA04AB0512564074081239FDE014
:10479000FAA3E0FB852E82852F83EAF0A3EBF0A33A
:1047A000E4F0A3F022AF25BF006F908036E0F8A3BD
:1047B000E0F5838882E0F530A3E0F531A3E0F5323F
:1047C000A3E0F533A3E0F534A3E0F535A3E0F53637
:1047D000A3E0F537A3E0F538A3E0F539A3E0F53918
:1047E0008C828D83E530F0A3E531F0A3E532F0A3B0
:1047F000E533F0A3E534F0A3E535F0A3E536F0A307
:10480000E537F0A3742EF0A3E538F0A3E539F0A363
:10481000E53AF0A3E4F0020FF0908036E0FAA3E06E
:10482000FBEA24E0FAF582EB34FFFBF583A3E0F525
:1048300030A3A3E0F531A3A3E0F532A3A3E0F53361
:10484000A3A3E0F534A3A3A3A3A3E0F535A3A3E0BA
:10485000F536A3A3E0F537A3A3E0F52CA3A3E0F579
:104860002DA3A3E0F538A3A3A3A3E0F539A3A3E008
:10487000F53A8C828D83E530F0A3E531F0A3E53283
:10488000F0A3E533F0A3E534F0A3E535F0A3E53676
:10489000F0A3E537F0A3E52CF0A3E52DF0A3E53870
:1048A000F0A3E539F0A3E53AF0A3AC82AD83DF05D0
:1048B000E4F0020FF00248218C268E2E8F2F752CEB
:1048C00000752DC0AC267920AE2CAF2D1244EA7FA6
:1048D000014048852C82852D837F02E0603DF924CC
:1048E0001B60E1E52C440BF582E0543FB40F29A393
:1048F000E070D1E954407035A3E0B52530E52C24B3
:1049000020F52CE52D3400F52D54F0B4C00280B410
:10491000904A7912569A80A602496A852E82852F7E
:1049200083E47932F0A3D9FC8F82020FF0E5825440
:10493000E0440DF582E0F525AC2CAD2DBC0006BDA4
:10494000C0030248FD7E007FC079208C828D83E009
:10495000A3AC82AD838E828F83F0A3AE82AF83D966
:10496000EA85822C85832D0248C4852E82852F837B
:10497000F0A3790BAA82AB83852C82852D83E0A3DB
:1049800085822C85832D8A828B83F0A3B9040474DD
:104990002EF0A3D9DFE4F0A3AA82AB83852D83E5B3
:1049A0002C54E04414F582E0A3F532E0A3F533A3E0
:1049B000A3A3A3E0A3F530E0A3F531E0A3F534E031
:1049C000A3F535E0A3F536E0A3F5378A828B83E5BE
:1049D00030F0A3E531F0A3E532F0A3E533F0A3E531
:1049E00034F0A3E535F0A3E536F0A3E537F0A3AA4C
:1049F00082AB83852C82852D83E58254E0F5827914
:104A00000BE403F5F0E025F0A3D9F7B52547852C95
:104A100082852D837901E58254E0C39420F582E5F7
:104A2000839400F58354F0B4C02BE0F5F0543FC3F9
:104A3000997022A37805124A63A3A3A3A3A37806BF
:104A4000124A63A3A3A3A37802124A63E5F020E607
:104A50000409B911C18A828B83E4F0758200020FC8
:104A6000F0A3A3E0AE82AF838A828B83F0A3AA82F5
:104A7000AB838E828F83D8E9226469725F7265612D
:104A80006420746D7020627566666572206F76654D
:104A900072666C6F77210D0A0090631D12569AECB6
:104AA000F5261239ECE05402FD74101239FDAE8285
:104AB000AF83E0A3FAF514E0A3FBF5157011EA70DB
:104AC0000E742412565912565F90FFFF020FF01217
:104AD0005640A3A3E0335006900000020FF0125698
:104AE0002B781412572212565FEB7023EA7020AA1B
:104AF00014AB1512564074081239FDE0FAA3E0FB1E
:104B0000BD020CEA7009EB7006900000020FF08EF7
:104B1000828F83EAF0A3EBF0A3E4F0A3F085148284
:104B2000851583020FF0ECF5261239EC7408123962
:104B3000FDE0A3FAE0A3FBEA7003EB601912564014
:104B400074081239FDE0A3F530E0A3F5311254F1F9
:104B5000AA30AB3180E1E5261239ECE4F0020FF027
:104B600085F026124C8D5002D322C3EB13FBEA13BF
:104B7000FAE913F950027801C3EF13FFEE13FEEDCB
:104B800013FDD5F0E5B80002800CE92401F9EA3400
:104B900000FAEB3400FBC3ED9401FDEE9400FEEF50
:104BA0009400FF8D308E318F32E9FDEAFEEBFFE598
:104BB000261239EC74081239FDE0A3FAE0A3FBC217
:104BC000F0753301EAF8EBF912564074041239FD1E
:104BD000E5F07029E0C39D703DA3E0C39E7038A34B
:104BE000E0C39F703375F001E533B40108752C0004
:104BF000752D008023882C892D801D80CBE0C395E6
:104C0000307013A3E0C39531700DA3E0C3953270EB
:104C10000775F0028002A3A3A3A3E4F533E5F060D7
:104C20000F8583148582151254F1851483851582AE
:104C3000EAF8EBF9E0FAA3E0FB7003EA6009E5F0BB
:104C4000B402B87F0080027F01E52C701EE52D7054
:104C50001AE5261239EC74081239FDBF0106E4F09A
:104C6000A3F08025EAF0A3EBF0801EEAFCEBFDAA9E
:104C70002CAB2D12564074081239FDBF0106E4F02A
:104C8000A3F08005ECF0A3EDF0C3020FF075F00483
:104C9000E53B20E70E20E60D20E50C20E40B20E3A9
:104CA0000AD32205F005F005F005F0C322905F3A23
:104CB00012569AE51CB40608905F7D12569AC322DC
:104CC000B40109905F4012569A024D26B402129028
:104CD0005F4712569A90FF6EE020E302D322024D06
:104CE000E6B40312905F5212569A90FF50E020E013
:104CF00002D322024E4DB40414905F5D12569A9076
:104D0000FF6EE030E702D322751C01C322B4050B0D
:104D1000905F6A12569A751C06C322905F881256DD
:104D20009D751C01C322E519B5181374FFF518F51C
:104D300019E51BB51A1C74FFF51AF51BC32204B440
:104D40001801E4F519C4032400F582E43489F583DD
:104D5000801504B47801E4F51B75F008A42400F56F
:104D600082E5F03484F583E0A3FCE0A3FDE0A3FE3C
:104D7000E0A3FFE0A3FAE0A3FBE0B40111904F54DD
:104D800012569A90FF6E74E6F0751C05D32290605F
:104D9000A012569AEF125671EE125671ED1256711C
:104DA000EC1256719060B112569AEB125671EA12DB
:104DB000567112565FEF540F452490FF6CF0EE9041
:104DC000FF6AF0ED90FF68F0EC90FF66F0740890D9
:104DD000FF64F090FF6E74C4F0751C0290FF14EA3B
:104DE000F0A3EBF0D32290FF22E4F0A374A0F090A4
:104DF000FF24E4F0A37408F090FF5CF090FF58F0FB
:104E0000751C03C322F890FF23E0F9B4B0047513B6
:104E1000002254F0B4A00475130022E513600122AF
:104E2000904E3812569DE91256741256FCE81256EE
:104E3000741256627513012249444520444D4120A5
:104E40004572726F722C20416464723D0090FF14B1
:104E5000E0FAA3E0FBE4F090FF14EBF0EAC454F0B6
:104E60004402F582EAC4540F44A0F583E0547FF075
:104E7000C214751C04D322E51C24FB600A24FF60C5
:104E800006758200020FF0758201020FF0E51AF438
:104E90006005E4F51AF51BE518F46005E4F518F56E
:104EA00019020FF0E51CB40606758201020FF0E549
:104EB0001AF47010E518F4700BE51CB40106758245
:104EC00001020FF0758200020FF0E51AB4FF05E44D
:104ED000F51AF51B04B47801E4F51A75F008A4245A
:104EE00000F582E5F03484F583E4F0A3E535F0A322
:104EF000E536F0A3E537F0A3EAF0A3EBF0A37401E5
:104F0000F0E4A3F0020FF0C083C082125062124F8F
:104F10003090FF6E7420F012507320E009D082D0E0
:104F2000831250D1E42290FF62E060012274FF22DC
:104F3000E537540F452490FF6CF0E53690FF6AF09A
:104F4000E53590FF68F0E53490FF66F0740190FF5E
:104F500064F022226964655F736C6565700D0A00F8
:104F60007524E0F17820E70320E6237524F0F1783A
:104F700020E71020E618800B90FF6CE524F090FFEE
:104F80006EE022742E122030758200020FF012564D
:104F900062905EDD12569D12569D905EF5E52430BE
:104FA000E403905EFE12569D74011252FF740712C4
:104FB00052DB12506290FF6E74ECF01250739070DE
:104FC000001250D1125062907006E014452454BF74
:104FD00090FF6CF090700CE090FF64F090FF6E74A6
:104FE00091F012506290632712569DE52490FF6C59
:104FF000F0740890FF64F090FF6E74C6F012506277
:10500000125674125662751C0490FF0EE0FAA3E06B
:10501000FB1254F1758201020FF090FF40E4F01191
:10502000451145114511457401F01145114590FF99
:105030006C74E0F090FF6EE090FF6C74F0F090FF05
:105040006EE0020FF07800790AD9FE00D8F900224C
:105050006964653A20686172642072657365740DD5
:105060000A0090FF6EE0C0E0742A122030D0E020E9
:10507000E7F02290FF6EE0C0E0745F122030D0E0D5
:1050800020E7F030E3ED227A209070001256621291
:10509000568B743A12203074201220307B10E0A31B
:1050A0001256741256FCDBF6C3E5829410F582E5C5
:1050B000839400F5837B10E0A3547FB47F01E42444
:1050C000E04001E42420122030DBEC125662DABF0B
:1050D000227D00C083C08290FF60E0FA90FF43E031
:1050E000FBD082D083EAF0A3EBF0A3DDE6221252DC
:1050F00046700C905EC7120038758201020FF0FFF7
:10510000905EDD120038EF120050905EE912003818
:105110007A007B0074021252DB90200012521F0AA8
:10512000BA20F17D00EDFAE4FB74021252DBED12BD
:10513000522B6033ED6008901FF0E4F0A3EDF0799E
:105140000090200009E9F0A3EDF0E582240FF5823C
:10515000E5833400F58354F024E060E8EDFA7B0049
:1051600074011252DB8018902002740FF0E5822443
:1051700010F582E5833400F58354F024E060EB0DF4
:10518000BD20A2901FF0E4F0A3F0E4FAFB74021239
:1051900052DB902200E4F0A3F07A207B0074081226
:1051A00052DB90800012521F9080167421F0A3E40D
:1051B000F0908018E4F0A3F090800D74DFF0A3EF7E
:1051C00014F074061252FF74001252DB12562B7444
:1051D000011252DB12562B74021252DB12562B7440
:1051E000031252DB12562B74041252DB12562B742C
:1051F0000D1252DB90D00012521F74FFF518F519F2
:10520000F51AF51BF51DF51E908006F0A3F0A3F02E
:10521000A3F090800CF0751C04758200020FF0E47E
:1052200078107900F0A3D9FCD8F82203035407F8CA
:10523000EC54032402838004010355FFB800035497
:105240000122031880F6E4FAFB1252DB1252931289
:1052500052AE5003E4FC227A007B08E41252DB12C7
:105260005293E4FAFB1252DB1252AE92E1C0E07AA2
:10527000007B04E41252DB1252931252AED0E09241
:10528000E0F45403FC048322040810205146F58204
:10529000020FF090FF00E0F5F0A3E0900000645AE8
:1052A000F0A3F4F0A3E5F0649CF0A3F4F02290FFE7
:1052B00000E0F8A3E0F5F0900000E0645AB5F019C2
:1052C000A3E064A5B5F012A388F0E0649CB5F009F2
:1052D000A3E06463B5F002C322D322540F23240059
:1052E000F582E434FFF583EAF0A3EBF022EA51FF04
:1052F00040078A828B83020FF0900000020FF0F8C3
:10530000F9905FD212569AE81256B2905FDA1256AE
:105310009A908016E0FAFEA3E0FBFF8A04EBFD7092
:1053200006EA7003025397EB125671EA1256717433
:1053300020125659EB7024EA24DF401F9053F112DB
:10534000569DEB125674EA1256741256FCEF125622
:1053500074EE12567412566202576E125640E0FAFC
:10536000A3E0FBA3E0600312541F7401F0D8AC1259
:10537000565F90800DE0C399F0A3E09400F0908018
:1053800016EAF0A3EBF0AA04AB05125640E4F0A332
:10539000F0AA06AB07C3229053CA12569A90801601
:1053A000E0FAA3E0FBEA7003EB601AEB125671EA35
:1053B0001256717420125659125640E0FAA3E0FBBF
:1053C000A3E4F080E012565FD3226D616C6C6F63D2
:1053D0005F626C6F636B2C206F7574206F66206D3D
:1053E000656D6F72792C2066726565696E673A200B
:1053F000005741524E494E473A206D616C6C6F63C5
:105400005F626C6F636B73207573696E6720726582
:10541000736572766564206D656D6F72792000C06A
:1054200082C083905F9C12569DED125674EC12560A
:10543000741256FC742D1220301256FCEB12567466
:10544000EA1256741256FC742D1220301256FCD0FB
:1054500083D082E0125674125662229054AC1256D7
:105460009D90800DE0FEC0E0A3E0FF125674D0E0F6
:105470001256741256FC743D1220301256FC12540F
:10548000CBEFB50112EEB5000EE9125674E81256D4
:1054900074125662020FF0C2AFD299E9120034E8DA
:1054A0001200341200483099FD02576E4D656D6F41
:1054B000727920417661696C61626C652028346B79
:1054C00020626C6F636B73293A2000908016E0FABB
:1054D000A3E0FB78007900EA7004EB700122125619
:1054E0002BE82401F8E93400F980EC1254F1020FA2
:1054F000F0908016E0FEA3E0FF9062E912569A8ACF
:10550000048B0579007800BB0008EA24DF40030221
:1055100055E6EB54E06019C082C0839062BF12561A
:105520009DEB125674EA125674125662D083D082E2
:10553000097420125659EB125671EA12567112561E
:1055400040E0FAA3E0FBA3E07014C082C083906245
:105550006412569D90628112569DD083D08230E7AE
:10556000079055AF12569A08E4F0BA009ABB00971C
:10557000E8701F12565F5382F0EEF0A3EFF09080B8
:1055800016ECF0A3EDF090800DE029F0A3E03400DC
:10559000F0225382F0AA82AB83908018E0FEECF0F8
:1055A000A3E0FFEDF08A828B83EEF0A3EFF022669A
:1055B00072656520626C6F636B20772F2070656E5B
:1055C00064696E6720786665722C20707574206F30
:1055D0006E2070656E64696E672066726565206C0A
:1055E0006973740D0A0012566290629412569DEB14
:1055F000125674EA1256741256FCED125674EC12DE
:1056000056741256FCEF125674EE1256741256FC73
:10561000E91256741256FCA881E612567418E61266
:10562000567412566212566202576E125640E0E0ED
:10563000FAA3E0E0FB2212562BF5838A82020FF0D8
:10564000EB541F90FF1CF0A3E4F0EA540FC4F58262
:10565000EA54F0C444E0F58322301F2B022030309E
:105660001F25C0E0740D122030740A122030D0E0E3
:1056700022301F13D176C4C0E0540F2490D434409C
:10568000D4122030D0E02222301FFCC0E0E583128B
:105690005674E582125674D0E022301FEAC0E0E46E
:1056A00093A3600BA2E7547F122030400280F0D019
:1056B000E022301FD2C0F0C0E08013C0F0C0E03064
:1056C000E70C742D122030D0E0C0E0F4240175F016
:1056D0006484D2D56007C2D52430122030E5F0753D
:1056E000F00A8430D50260052430122030E5F02421
:1056F00030122030D0E0D0F022301F8B74200220F6
:1057000030301F16080808E612567418E612567153
:1057100018E612567418E612567422301FFC080858
:1057200080EA301FF50880E9D21F124CAD12566294
:10573000742012203090FF28E0C0E0A3E0125674DD
:10574000D0E0125674742012203090FF2AE0C0E09E
:10575000A3E0125674D0E0125674742012203090D8
:10576000FF50E0125674C2AF12566202006DC2AF13
:10577000D2997A007B0074071252DB9057C0120056
:1057800038EB120034EA1200341200489070001214
:105790005ABF0ABA20E09057C81200389080001211
:1057A0005ABF125A9D9030201200389057DF1200D5
:1057B0003890FF6E74E6F0751C0512004802006D0B
:1057C000426C6F636B2023004D656D6F72792C20E6
:1057D0003830303020746F20384646460D0A000DB0
:1057E0000A4120736572696F7573206572726F72FA
:1057F000207761732064657465637465642C207719
:10580000686963682070726F6261626C7920776189
:1058100073207468650D0A726573756C74206F6609
:10582000206D656D6F727920736F6D65686F77207D
:1058300067657474696E6720636F727275707465E2
:10584000642E2020497420636F756C642062650D9E
:105850000A7468617420796F75722053494D4D2028
:105860006973206261642E20204974277320616C63
:10587000736F20706F737369626C652074686174F4
:10588000207468657265277320610D0A70726F62FB
:105890006C656D2077697468207468652061646444
:1058A0007265737320636F6E6E656374696F6E7378
:1058B00020746F207468652053494D4D206F6E2011
:1058C000796F75720D0A6369726375697420626F0E
:1058D0006172642C206F7220746865726520636F3A
:1058E000756C6420626520612062756720696E2096
:1058F00074686973206669726D776172652E0D0A2E
:105900000D0A496620746869732069732061202735
:10591000756E737461626C652720646576656C6F63
:105920007065722072656C65617365206F662074A6
:1059300068650D0A6669726D6172652C2074686510
:105940006E2074686973206973206D6F7374206CA6
:10595000696B6520612062756720696E20746865D7
:1059600020636F64652E0D0A0D0A506C65617365C6
:1059700020747279207573696E672061206469668E
:10598000666572656E792053494D4D2C20616E64B9
:105990002069662070726F626C656D0D0A646F65B8
:1059A000736E277420676F20617761792C20747281
:1059B0007920747970696E67204445425547207795
:1059C00068696C652074686520706C617965722007
:1059D00069730D0A72756E6E696E672C20746F2084
:1059E000656E61626C65206164646974696F6E6183
:1059F0006C20646562756767696E6720696E666FA3
:105A00002C20616E64207468656E0D0A656D616995
:105A10006C206120636F7079206F662074686174F8
:105A200020646562756720696E666F20616E642010
:105A30007468657365206D656D6F72792064756D2E
:105A400070730D0A746F207061756C40706A7263B8
:105A50002E636F6D2E2020486F706566756C6C79B3
:105A60002049276C6C2062652061626C6520746F30
:105A700020666967757265206F75740D0A776861B5
:105A80007420636175736564207468697320746F32
:105A90002068617070656E2E0D0A0D0A007800791D
:105AA000087A20E8120034743A120030125AE2E602
:105AB00008120034DAF9120048D9E61200482278B8
:105AC00000E583540F120034E582120034125AE2CA
:105AD0007910E0A3120034D9F9120048D8E312007B
:105AE0004822742002003052656164696E67204D5F
:105AF000617374657220426F6F74205265636F72B8
:105B0000640D0A004D4252205369676E61747572CC
:105B100065204E6F7420466F756E640D0A00556ED9
:105B20006B6E6F776E20506172746974696F6E204E
:105B3000547970653A2000466F756E642046415472
:105B4000333220506172746974696F6E2061742001
:105B50004C4241203D200052656164696E672046D9
:105B60004154333220566F6C756D652049440D0ADF
:105B70000042616420464154333220566F6C756D8B
:105B8000652049440D0A00466972737420446174AB
:105B90006120536563746F72206174204C42412010
:105BA0003D2000506C6179696E672066696C653ACA
:105BB0002000566F6C756D65204944206C6F6F6BCB
:105BC00073206F6B0D0A00436C75737465722073DC
:105BD000697A65206973200020736563746F72733E
:105BE00020286561636820736563746F7220697330
:105BF00020353132206279746573292C0D0A436C8B
:105C00007573746572732077696C6C2062652063AC
:105C1000616368656420696E200020626C6F636B4D
:105C20002067726F75707320286561636820626CED
:105C30006F636B2069732034303936206279746564
:105C400073290D0A00436C75737465722073697A49
:105C50006520646F65736E277420666974206E69B1
:105C600063656C7920696E746F20346B20626C6F91
:105C7000636B730D0A4341434845204D454D4F52D8
:105C8000592055534147452057494C4C204E4F54BD
:105C900020424520454646494349454E54210D0A78
:105CA00000526F6F74206469726563746F7279203B
:105CB00073746172747320617420636C757374659E
:105CC000722000536563746F72732075736564206E
:105CD000666F7220464154207461626C65733A208D
:105CE0000020204174747269623D00202046697270
:105CF00073745F436C75737465723D002020536943
:105D00007A653D000D0A0D0A0D0A4D503320506C86
:105D1000617965722C2056657273696F6E20302E22
:105D2000362E322E322C204D617920342C20323008
:105D300030310D0A436F70797269676874202843A7
:105D40002920323030302C20504A52432E434F4DC0
:105D50002C204C4C430D0A0D0A54797065202751B4
:105D60005549542720746F2072657475726E2074C3
:105D70006F20746865206D6F6E69746F720D0A0D07
:105D80000A000D0A4D503320506C617965722C2049
:105D9000426567696E20506C61796261636B0D0AC0
:105DA00000436F6E6669677572696E672058696C2B
:105DB000696E78205843533130584C204650474143
:105DC00020436869703A20004F6B0D0A00666169D4
:105DD0006C0D0A004572726F72210D0A00526573D4
:105DE0006574696E6720494445204465766963653A
:105DF000730D0A00436F6E6669677572696E67207E
:105E0000535441303133204D5033204465636F6427
:105E1000657220436869703A200057616974696E41
:105E20006720666F722048617264204472697665EB
:105E300020746F2062652072656164790D0A000D1F
:105E40000A43757272656E7420536563746F7220B5
:105E500042756666657220436F6E74656E74733A40
:105E60000D0A00506C61790D0A0050617573650D63
:105E70000A004E6578742046696C650D0A00507200
:105E80006576696F75732046696C650D0A0052610D
:105E90006E646F6D204F00566F6C2055700D0A00B8
:105EA000566F6C20446F776E0D0A00496E697469F5
:105EB000616C697A65204D656D6F7279204D616EF8
:105EC000616765720D0A00426164206F72204D693E
:105ED0007373696E672053494D4D0D0A00466F7507
:105EE0006E6420004944452000206D6567205349B9
:105EF0004D4D0D0A004D61737465720D0A00536CAF
:105F00006176650D0A0052756E6E696E67204F6C82
:105F100064204669726D776172652C2074686174C3
:105F200020646F65736E27742075736520746865CF
:105F30002053494D4D0D0A0D0A006964653A200051
:105F400069646C650D0A0077616974204452510DD3
:105F50000A007761697420444D410D0A0077616938
:105F600074206E627573790D0A0077616974696EC9
:105F70006720746F20736C6565700D0A00736C6523
:105F80006570696E670D0A00696C6C6567616C20ED
:105F9000286F682073686974290D0A005741524EB2
:105FA000494E473A206D616C6C6F635F626C6F6342
:105FB0006B732C20626C6F636B20697320616C7251
:105FC0006561647920616C6C6F6361746564202D18
:105FD00020006D616C6C6F63200020626C6B3A0076
:105FE000666F70656E2C2066643D0066696C655F47
:105FF00063616368652C2066643D002C20627974BF
:106000006573200020746F20002020526571276482
:1060100020635F6F66667365742000202066696E7A
:106020006420632C206375723D002020202073655E
:1060300061726368204641542000202020204641A0
:106040005420736563746F7220666F756E642C20C4
:10605000693D002C20626C6B3D00202020204641D1
:106060005420736563746F72206E6F7420666F7551
:106070006E6420696E206C6973740D0A0020202004
:10608000206D6F76696E6720666174207365637436
:106090006F72206C6F6F6B75702061727261790026
:1060A0006964653A20726420346B2C206C62613D17
:1060B0000020746F20626C6B2000202072642063CB
:1060C000200020286F666673657420002020202041
:1060D00063757272656E746C792063616368656460
:1060E00020626C6F636B7320772F204641542073BE
:1060F0006563746F72733A2000202020206E6577EC
:1061000020626C6F636B20746F20696E73657274AC
:1061100020696E746F2061727261792061742069E8
:106120006E6465783D00202070726576696F7573C6
:1061300020636C757374657220696E20626C6F6386
:106140006B3A200020202020202062696E5F73655A
:10615000617263683A20626567696E3D002C206554
:106160006E643D002C206D6964646C653D00665F63
:10617000635F772C66643D006E6F200070726576F9
:106180000020206663616368652C20633D002C203D
:10619000635F6F66667365743D002C20746172677F
:1061A0003D0020206D6B20727265712C20626C6B3B
:1061B0003D002C20633D002C206F3D002C206E788C
:1061C000743D0066696C655F7365656B20746F2054
:1061D00062797465206F66667365743D0020206384
:1061E0006C75737465725F6F66667365743D002CC1
:1061F00020706F735F636C75737465723D002C2043
:10620000706F735F626C6F636B3D002C20706F73F7
:106210005F627974653D00656E64206F6620666913
:106220006C6520726561636865642C20756E6162BF
:106230006C6520746F20667365656B0D0A00506C89
:10624000617920626C6B20000D0A46696E69736883
:1062500065642C20707265737320616E64206B65B9
:10626000793A20005741524E494E473A20667265AE
:10627000655F626C6F636B732C20626C6F636B2065
:106280000020697320616C726561647920667265B3
:10629000650D0A005741524E494E473A20667265D5
:1062A000655F626C6F636B732C20626C6F636B2035
:1062B0006973207265736572766564202D200057BE
:1062C00041524E494E473A20667265655F626C6F77
:1062D000636B732C20626C6F636B20697320696E33
:1062E00076616C6964202D20006672656520626CA1
:1062F0006F636B733A002C2066697273743D002CD7
:10630000206C6173743D002C206C6973743D002017
:10631000206E65787420626C6F636B3A00667262FF
:106320002C706F73623D00536574206D756C7469D9
:10633000706C65206D6F64652C2073746174757367
:106340003D004465627567204D65737361676573D1
:10635000205475726E6564204F4E0D0A00446562CC
:106360007567204D65737361676573205475726E30
:106370006564204F46460D0A00202069646520723E
:1063800072657120717565756520746F6F20667513
:106390006C6C20746F20666F7220636C757374650B
:1063A00072207269676874206E6F770D0A00202072
:1063B0004F7574206F66206D656D6F7279210D0ABF
:1063C00000735F72656164696E675F6469720D0A6C
:1063D00000735F63616368696E67310D0A00735F04
:1063E00063616368696E67320D0A00735F6361639E
:1063F00068696E67330D0A00735F63616368696E75
:1064000067340D0A00735F632D6E2D700D0A0073E3
:106410005F706C6179696E670D0A00735F66696E03
:106420006973685F706C6179696E670D0A00706CE2
:1064300061795F71756575655F656D7074792C2024
:1064400071756575653A2000202066696C655F721C
:1064500065616420666F756E64206C61737420637F
:106460006C75737465720D0A0054657374696E6798
:10647000205354413031332E2E2E2000743D000025
:1064800090FFE320C40000000348018000006890F2
:10649000FFE322C45B0000034801C00000D190FF6D
:1064A000E320C4B700000348000000003991FFE377
:1064B00022C4FF0000034800000000A291FFE32077
:1064C000C4FF00000348000000000A92FFE322C45A
:1064D000FF00000348000000007392FFE320C4FFA8
:1064E0000000034800000000DB92FFE322C4FF002D
:1064F000000348000000004493FFE320C4FF0000B5
:10650000034800000000AC93FFE322C4FF00000337
:106510004800000000E0A3C0E0E0A3C0E0E0A3C0AA
:10652000E0E0A3125674D0E0125674D0E012567414
:10653000D0E012567422E06006A312203080F722C9
:10654000C002124CADD00240F7DAF5020FF0EAB10A
:10655000606008A3E493F582020FF08882020FF0D6
:10656000F5F0B1870C908000E4936009B5F001224A
:10657000B4FF02E422E5822CF58250EC0583E5832A
:1065800054F0B480EE80E170037C0022B4FF037C01
:10659000002220E7037C01227C0B228A148815E567
:1065A00014B160605CAE82AF83A3E514B187ECFBED
:1065B000C2D5A815E6F5F0E493B5F002800755F0D2
:1065C000B5F00FD2D5A308DCEB20D51A75820002F6
:1065D0000FF08E828F830BE4C2AF120059D2AF400E
:1065E00056A3DBF380B98E828F83A3A815E6C2AFD2
:1065F000120059D2AF404008A3DBF2758200020FAF
:10660000F0E5141265870CE5822CE583340054F024
:1066100024807029E514C2AF120059D2AF4018A3EC
:106620001CA815E6C2AF120059D2AF400AA308DC7D
:10663000F2758200020FF0758201020FF0740112F0
:1066400052FF401DEAC0E0EBC0E0740C1252DB9038
:10665000800078C07900801ED0E0FBD0E0FA1254B0
:10666000F1758201020FF0A3E583550FB40F07E522
:1066700082B4FF02802FE493B4000280EAB4FF02E8
:1066800080231265870C8002E493AE83AF828883F7
:106690008982F0A3A883A9828E838F82DC0280C7BF
:1066A000E493A380E39080007424C2AF120067D209
:1066B000AF40A588F0908000AA83AB8290C000E034
:1066C000AE83AF828A838B82C2AF120059D2AF40B1
:1066D00087A3AA83AB828E838F82A3E583C395F0C1
:1066E00070DDE582C39970D7D0E0FBD0E0FA125498
:0466F000F102659FAF
:020000021000EC
:20900000CA9F10013A012A04280029002000210022002300240025002600270028012802AD
:20902000218F28032100280428052806280728082809280A280B280C20802190280D2000DE
:209040002100280E20812191280F2000219228102100281121932812210028132814281507
:209060002082281620002817281828192194281A2195281B2196281C2100281D2083281EF6
:209080002000281F219728202100282128222823282428252826282728282829282A20849D
:2090A000282B2000282C282D282E282F283028312832208528332000283428352836283746
:2090C0002198283821002839283A283B283C283D283E283F2840284128422843284428451B
:2090E0002846284728482849284A284B284C284D284E284F28502851285228532854285518
:209100002856285728582859285A285B285C285D285E285F28602861286221992863210035
:20912000286428652866286728682869286A286B286C286D286E286F2870287128722873F7
:20914000287428752876287728782879287A287B287C287D287E287F2880288128822883D7
:20916000288428852886288728882889288A288B288C288D288E288F2890289120862892CC
:20918000208728932000289428952896289728982899289A289B289C289D289E289F219A80
:2091A00028A0210028A128A228A328A428A528A628A728A828A928AA28AB28AC28AD28AE6D
:2091C00028AF28B028B128B228B328B428B528B628B728B828B9208828BA200028BB2089E5
:2091E00028BC200028BD28BE28BF28C028C128C228C3219B28C4210028C528C628C728C890
:2092000028C928CA28CB28CC28CD28CE28CF28D028D128D228D328D428D528D628D728D8C6
:2092200028D928DA28DB28DC28DD28DE28DF28E028E1208A28E2208B28E3200028E428E55E
:2092400028E628E728E828E928EA28EB28EC28ED28EE28EF28F028F128F228F328F428F5B6
:2092600028F628F728F8208C28F92000219C28FA219D28FB208D219E28FC208E219F28FDC1
:209280002000210028FE28FF2A012800220123952489250726A42707280121C7220023806B
:2092A00026C4270C28022009211C220426AA270A280320002100220023A626A02707280463
:2092C00028052005238426B427092806200022032300248125C026AB270A280721AE220049
:2092E00023952489250726A42700280821482201238026C4270C280920092104220426AAFB
:20930000270A280A20002100220023A826A42707280B280C21402220238026C4270C280DC5
:20932000222426C6280E219E220026C8280F20092102221426AA270A28102005210022009C
:20934000238426B427092811200021012300240125C026AB270A281221C323952489250703
:20936000262027002813200321C223832626270D281421B322082815200021C622002395C1
:20938000260027082816210023002496250326AA270A2817204221B62380248925072818DF
:2093A000200021002394260E2819200F238426B42709281A2000239326A82703281B2628BF
:2093C0002700281C21012300240125C026AB270A281D21C523952489250726202700281E62
:2093E000210023942600270A281F260E282020032179220123832626270D2821213228228F
:209400002000210422002380240025FC26AA270A2823210023002500282421A3220D238066
:20942000249E253B282520422157220124892507282620002143220D2400253828272108ED
:209440002298239524892507262427002828204221932201238026AA270A28292003217E10
:20946000220423832626270D282A200021B02200239526A02707282B21002300240C25049F
:2094800026AA270A282C21022380248625C326AB282D2042219722012489250726AA282EBD
:2094A000200021002200241F2504282F21B22395248925072620270428302042218B220425
:2094C000238026AA270A2831200021B12200239526A02707283220032175220423832626A4
:2094E000270D2833200521002200238426B427092834200021602300240125C026AB270A98
:2095000028352108229823952489250726242700283621BC2200283721A3220D2300240112
:2095200025C026AB270A28382160220023802400253826AA2839210622982395248925077A
:2095400026242700283A21BE2200283B20052100238426B42709283C200021602300240190
:2095600025C026AB270A283D2142220123952489250726242700283E210C229826A42707D2
:20958000283F21082840216022002300240125C026AB270A2841210C229823952489250720
:2095A000262427002842200521002200238426B427092843200023802400251026AB270A2E
:2095C0002844212222012395248925072624270028452100220023002404251226AA270A84
:2095E0002846200321D422052383248925072626270D28472000216022002300240125C060
:2096000026AB270A284821B3239524892507260027082849210023002409250026AA270A16
:20962000284A210223802486253B284B204221DD220524892507284C200021002200241FFB
:209640002500284D21B323952489250726202700284E210023002497250326AA270A284F89
:20966000204221E2220523802489250728502000211022002300248025CC26AB28512100D4
:20968000224023B42489250726AA27042852220023B02692270928532114220123952600B5
:2096A00027082854214823A4262A270028552100220023002409250026AA270A285621087B
:2096C00023802486253B2857204221112207248925072858200021002200241F25002859FC
:2096E0002114220123952489250726202700285A211626022709285B210022002300248076
:20970000254826AA270A285C23A02489250726142709285D2480255026A42704285E211601
:2097200022012395248925072700285F210422002300249C257826AA270A28602143220DE4
:20974000240125C426AB2861210322002415286221002400250026AA2863215E23952489EF
:20976000250726102709286421032300241525C426AB270A2865210023802400250626AAF0
:209780002866248F25E326AB2867204221CD22072489250726AA2868200021602200230088
:2097A000240125C026AB286921002380248F250326AA286A204221DD220724892507286B47
:2097C00020002143220D2300240125C026AB286C210022002400250426AA286D2003217F8C
:2097E00022012383248925072626270D286E2162286F200521002200238426B427092870E6
:20980000200021062395260027082871210123002497253B26AA270A28722042210E2208A5
:2098200023802489250728732003213C220B23832626270D2874200021032200239526025C
:209840002708287521272300248125C426AB270A2876210023802409254826AA287721585D
:20986000223423A324892507262A270028782100220023A0260027092879210723802403ED
:20988000253926AA270A287A21042300241C2538287B2107238024832539287C21032395EF
:2098A0002489250726022708287D21272300248125C426AB270A287E2100238024092548D4
:2098C00026AA287F2158223423A324892507262A27002880210622002300248125C02693D5
:2098E00027012881210023802489254826AA270A28822002216622082300240025662883BE
:209900002000210022002380241F2502288421062489250726DC270C2885210023AA26AA8B
:20992000270A288623B626002708288723802486253B26AA270A288821052489250726DC0C
:20994000270C2889210023AA26AA270A288A23B626002708288B23802486253B26AA270AF3
:20996000288C2042217B220824892507288D200021002200230024012582288E21052481AA
:2099800025C226AB288F2003219322082383248925072626270D2890200021052200230015
:2099A000248125C0261327012891210023802489254826AA270A28922002217E220823005C
:2099C0002400256628932000210022002380241F2502289421052489250726DC270C289500
:2099E000210023AA26AA270A289623B626002708289723802486253B26AA270A2898210539
:209A00002489250726DC270C2899210023AA26AA270A289A2380241F2502289B21012300B1
:209A2000248125C226AB289C2003219322082383248925072626270D289D200021042200D9
:209A4000239526122708289E216023C426AA2704289F210023C02600270928A0204221CB87
:209A60002208238026AA270A28A12070215422B823952612270828A2200221CC22082380AB
:209A800026AA270A28A3200321CA220F23832626270D28A42000210022002300248C250C62
:209AA00026AA270A28A521042482257828A621002380248925482612270428A7200321DE70
:209AC000220F238325072626270D28A82000210122002300249C257826AA270A28A921005C
:209AE00023802481254028AA200321CF220F2383248925072626270D28AB2070210822B83E
:209B0000239526A0270428AC200321D4220F23832626270D28AD2127220B28AE2070216325
:209B200022B823952612270828AF2000210122002380248625CB26AB270A28B0204221DD7A
:209B400022082489250726AA28B1200021182280239526A4270028B2200321D9220F2383E7
:209B60002626270D28B32070210A22B8239526A0270028B4200221E02208238026AA270A83
:209B800028B52070210A22B8239526A0270028B621542602270828B720002118228026A460
:209BA000270028B82100220023802480254826AA270A28B92070215E22B82395248925074B
:209BC0002612270828BA20002100220023802409254B26AA270A28BB2070215F22B8239513
:209BE000248925072610270828BC2000210022002300241C258326AB270A28BD2003213278
:209C000022092383248925072626270D28BE20002100220023002482258C26AB270A28BF6E
:209C20002003212522092383248925072626270D28C0204221BC238026AA270A28C12000BD
:209C4000210122002300240125C026AB28C22070210F22B82395248925072620270028C355
:209C6000200321E3220F23832626270D28C4200521002200238426B4270928C52000210330
:209C800023952614270828C621A623A4262A270528C7210023A02644270928C82118226D86
:209CA0002380249E257B26AA270A28C920422113220B2489250728CA200021AE2200239556
:209CC0002624270028CB2100220323802487257B26AA270A28CC20422116220B2489250758
:209CE00028CD200021AE220023952624270028CE20052100238426B4270928CF2003210D00
:209D0000220B23832626270D28D0200021002200230024802602270028D123802409254849
:209D2000261E28D221582234233324802507262A28D32100220023002680271028D4211035
:209D40002363262A270028D52100236026A8271228D621AF224C230026C8270C28D72100BE
:209D600022002680270528D823802486253B261E270028D92042211C220E23002480250714
:209D800028DA20002135222926C4270C28DB2002211D220E261E270028DC2000217F2234CB
:209DA00026C4270C28DD210022002390249F25042610270A28DE2300248425002680271065
:209DC00028DF2106236324802507262A270028E021002380248926AA270A28E12005238439
:209DE00026B4270928E22070216122B823952612270828E32000210122002380248625C3A0
:209E000026AB270A28E4204221CE220F2489250726AA28E52070215022B823952612270802
:209E200028E6200521002200238426B4270928E72070216422B823952612270828E82000AE
:209E4000210122002380248625C326AB270A28E9204221D3220F2489250726AA28EA2070A4
:209E6000215122B823952612270828EB200521002200238426B4270928EC2070216522B847
:209E800023952612270828ED2000210122002380248625C326AB270A28EE204221D8220F51
:209EA0002489250726AA28EF2070215222B823952612270828F0200521002200238426B4E5
:209EC000270928F12070216122B823952602270828F22000210122002380248625C326ABBA
:209EE000270A28F3204221DD220F2489250726AA28F42070215022B823952602270828F5B9
:209F0000200521002200238426B4270928F6200021012380248625CB26AB270A28F7204208
:209F200021E1220F2489250726AA28F82000210222002300248125C426AB28F92100238059
:209F40002489254826AA28FA20052384250726B4270928FB2070214E22B8239526102708DA
:209F600028FC2000210022002380248625C326AB270A28FD204221E7220F2489250726AABA
:209F800028FE200021BB220023952620270028FF20052100238426B427092A0810013A00BD
:209FA000540155210700060C0B03501051005204610F645565550855095505A10D04180437
:0C9FC0000C0177B8780B79A07A0072B021
:020000021000EC
:10D00000FF04E8FAF9DAFF57FDFDD7DF7E5DEFF7A1
:10D010007EFA6DA7DF77FDF5F737FFDF7FFFFDF7BE
:10D02000DF7DF7DDDFFDF7DD7FDF7DF7FDFFABFFA8
:10D03000FFFEFFEFFFFFFD7FDFFFFDFFFFFFFFFFB5
:10D04000FFFFFFCBFFDF7FFFFDF7DF7FFFFDDF7F10
:10D05000FFFDF7C77FFFFDFFE6FBFFF9F7DF7FF777
:10D06000FD67DFF7DD77DF7DF3FDF7DFFFF0FEFF24
:10D07000FFFFFFFFFFFFFFFFFFFFFFFFFFFDFFFFC2
:10D08000FFFFEAFEFFFFFFFFFFFFFFFFFFFFFFFFC6
:10D09000FFFFFFFFFFFFFFFCFFFFFFFFFFFFFFFFA3
:10D0A000FFFFFFFFFFFFFFFFFFFFFFAFFEFFFFBF21
:10D0B000FFFEFBFFFFFFFFFFBFFFFFDBFFBFFF7EAA
:10D0C00027FFFFFFFFFFFFFFFFFFFFFFFFFFFFFF48
:10D0D000FFFFFFFFFF8FF6FFFFFFFFFFDF7FFFFF79
:10D0E000FF3FFFFFF7FFFFFFFFDFCFFFFFFFFFFF68
:10D0F000FFFFFFFFFFFDDFFFFFFFFBFFFFFFFFED78
:10D10000DF7FFFFDFFFFFFFFFFFD5E7FFFFDF7FEFF
:10D11000FFFFFFFDF1FFEFBFFFFEBBEFBFFFFEEE26
:10D12000BFFFFE7BEFBFFFFE7FFAFFF7DF7FFFFD54
:10D13000F7DF7FDFF75F77FFFDF7DF7FFF9FFC7F84
:10D14000FEF9E79F7FFEF9E75FFEF9E79B7FFEF9B7
:10D15000E7FFBF3EFFBDF7DF7FFFDCF7CFCFFCF778
:10D16000CF7FFFFCD7DFEF679F9F7FFED9E79F7FD1
:10D17000FED98F7FFEF9E79F7FFEF9BFA3CFBFFEE9
:10D18000FEFBEFFFFFFEFFFBFFFEFFEFFFFFFEFBDF
:10D19000FFD3F7D7D77FFFFDF7DF7FFFF5DF7FFFF7
:10D1A000FDF7DF7FFFFF63FDDB6FBFFDF6DB6FBFCA
:10D1B000FDDA65BFFDF6DB6FBFFDFF72FBBFFFFF52
:10D1C000FFFFFFFFFFAFFFFFFEFFFFFFFFFFFF2F90
:10D1D00078FFFFFFFFFFFFFFFFFFFE7FFFFFFFFF67
:10D1E000FFFFFFFF97BDFFFBFFFEFFFFFDFFDFFF20
:10D1F000FDDFDFFFFBFDFFFFFFFFCEFFF7FFFFFFC0
:10D20000FFBFBFFF1FCFDDF3DF7FEFFCFFFF17FF87
:10D21000FFFEFBEFBFFFFEFBCFBFFEFBEBBFFFFE42
:10D22000EAEFFFBFFF6FFFFFFFFEFF7FFD7FFFFF06
:10D23000FFFFFFFFFFFF7FFFCF7FEFFFFFFFFFFF3E
:10D24000FFFFFFFFFFFFFFFFFFFFFFFFFFECFFFB05
:10D25000FFFFFFFFFFFFFFFFFDFFFFFFFFFFFFEFF0
:10D26000BF7FF1FFFFFFFFFFFFFFFFFFFCFFFBFFA3
:10D27000FFFFFFBFFFFF3FB8FFFFFDFFFFFFFFFF07
:10D28000FFFFFFFFFFFFFFFFFFFF7F5FDCFFFFFFF1
:10D29000FFFFFEFBEFD7FDFDF1FF5FFFFBEFFFFEA2
:10D2A000EFFEFFFFFFFFFFFFFFFFE77BFFDEFDAFAE
:10D2B000FFFFFFBFFF47F7FFFFFFFFFF77FFFDF710
:10D2C0006FFFFDF7DF7FFFFDF7FF93FFFFEFFFFF2E
:10D2D000FFEFBFFFFEEDBFFF7EFBCE1FFBFCF5C1E6
:10D2E000FFFFFFFFFFFFB7D7FE9FFFFFFFFFFFF727
:10D2F000DB77BFFFE3FFFFFFFFFDFFFFFF3FFB719A
:10D30000CF3FFFFCF3CFFEFFFFD1FFFFFEFFFFBFCC
:10D31000FFFFBFFFFAEFBFFFFEFBEFFF7FFEFAF755
:10D32000AFFFBFFFF77BEF9EFFF9E79F7FFEF9E3BB
:10D33000AF7F3FFCFFFBFF57FF7FFDF3DFBEFDF735
:10D340005F7FFFFDBFFFFEBFFEF7FF7F7BFEBFF7E6
:10D35000FBDFFFFDF7DF77D7FDFFFDFF3FFCFFFFA2
:10D36000FFFDFFFFFFFFFBAFFFFEFBECB3FFBEFACD
:10D37000FFA2F5FFFFFFFEFFFF3DFFFFFFFFFF7F67
:10D38000FEFFFFCFFFAFD5FBFFFF7FFFFFDCF9E71D
:10D390003BBFF3CE3BEFBCF3CEFBF76DFFFFFFBF10
:10D3A000FFFFEFFFE7FFFFFFFF9D7FDEFFE79DEF42
:10D3B000F2FFFFFFDFFFFF77B3EFACCE3AEBBEB378
:10D3C000EE3AEBAEFFDBFFFFFFEFFEFFEFD9F3D747
:10D3D0007FFDF5CF5F7FFDF5D77BF8FFFFFFF7FF00
:10D3E000FF7DFFEDFB9EFBEAB3AFFE7BEEEB67F646
:10D3F000FFFFFFFBFFFFFFF7DFDB5D77DF79F3FD6B
:10D4000037DFFF47FDFFFFFFFFFFFFB7DB777EE75B
:10D410001D77DD79E79D77FEADFFFFFFFFFFFFFF83
:10D42000E77F7FF7F7DF7FFCFDF7DF7FFF80FFDF20
:10D430007FFFFDF7DB6FBEDBBEEDB6FB6FBFEDF62A
:10D44000DB7F68FFFFFFFFFFFFFCFEDB3FFFF3CF4B
:10D45000FFFFFFF3FFFFEFF5FFFFFFFFFF7FFFFF82
:10D460007DF777DF7DFFFD77DF7FFF7FFBFFFFFF2E
:10D47000BFFFFFFACD7FFEE79F7FFEF9E79F7FFEAC
:10D48000BFFCFFFFFF9FFFFFF9FD7FFFF7DF7FFF7F
:10D49000FDF7DF7FFFCFFEFFFFFFEFFFFFFEFBDFAC
:10D4A000F7FDF7DF7FFFFDF7BFFF1FFFFF977FF659
:10D4B000F9E79F7FFEF99F5FFEF9E79F7FFEF98BFB
:10D4C000FFFFFFFFFBFFFFFFFFF77FFFEDE7FF7FA2
:10D4D000FFFDF7FFDFFFFFF7FFFDFFFFFFFFF77F18
:10D4E000FFDDF7DF7FFFFDF7FFC7FFFFFEFFFEFF5A
:10D4F000FFBFFFFDDD7FFFFFFFDF7FFFFD7F76FFCB
:10D500007FFF7FFFFFFFFFFFFFFFFFFDFFFFFFFF2D
:10D51000FFFFBFF9FFFFFF2BF7FFF2FB6FFFF6DB0B
:10D520006FB7FDF6DB6FFF3FFCFF575F7FFD555781
:10D530005F5CBD55575F75F555475FFD8EFEFFFF7C
:10D54000FFF5FFFFEFFDCFFFFCF3FFF7DFFCF3CEAE
:10D55000FF47DEEFFFFFDFFEFFFDFFF5DF7FFDFF93
:10D56000FFDF7FFDFDFF89EFFFFFFFFFFFFFFDFFF7
:10D57000FFBBFFB7FFBDBDFFFFFB7FDCFFFFFFFF72
:10D58000FFFFD75A7DFDD75D7FFDF5D75F7EFDFF9D
:10D59000E5FFFFFFFFFFFFA75FFFBFFFFFEFFFFFFD
:10D5A000FFFFEFFF3FF6FFFFFFFFFFFDFFDF6F7B9A
:10D5B000E6DF7FFBFDBEDF7FFF9FFBFFFFFFFFBBC3
:10D5C000FEFAFBADBF7AABA7BFF6FEF3CFFF6FFC51
:10D5D000FF7FFFFFFFEEFFEDBEFBFB6FBEFBFEBD5F
:10D5E000FDF7FFAFFEFFFFFFFF5FFFEFFFF7C9FF94
:10D5F000FFF7FFFEFFF7B7FB57FFFFFFFFFFDFFF60
:10D60000FFFFCFF7FFFFFBFFFFFDF7EFFFB3FFF8D3
:10D61000FBEEFFEFAFBFFEFBB5FFFEFBAFBFBFFAF8
:10D62000FAFF87FFFF7FFFFFF5FFFF7FFDD75F7FDB
:10D63000FDF5D7FFFFEFFF6FFFFF7FFFFFFEFFFF4F
:10D64000BFFFF9EF9FFFFEFBFFFFFFFFC3FFFFBF21
:10D65000FFFFFEFFFF3FAAF2CA3FFF3CF3CA2BFFCA
:10D660008F5BFFFFFFFFFFFFFCFFFFE77F7EFFD722
:10D670009F7FFEFCFF7ABCFFFFFFFFFF7E9F77BE10
:10D68000F99B6FBEF3E69B6FBE7FBFF6FFFFFFFF08
:10D69000FDBFFF7EFFFDDF7FDFFFF7DD7FDFFF06E2
:10D6A000FFFFFBFFFF3D4BAE5FCEE99C73EE3AE31D
:10D6B0009E73EFF3ABFDFFFFFFFFFFA5FF5BFFFCDA
:10D6C000CF3FFFFFFFCF5FFFBE83FF7FFFE7FFFB83
:10D6D000F7DFFF3EEBB18FFEFBEAA3E7BE7EEDFF77
:10D6E000FFFFD7FFF7DBEFFFBDDF75F7FD37DF7D0E
:10D6F000F3FD7FF1FFFFFFFFFF9D7FFB7DF777DFEE
:10D7000075FFFD77DD6DF77FF9FFEFFFFFFFDF7F2F
:10D71000FFF7477FFCF1FFFF7FFCFDD71FF9FFFDFF
:10D72000F7DFEFA679F7BAEBBBEEBAEFAEBB6EBA96
:10D73000F7B7F6FFFFFFFFF6FF7FFFFDF77FFFFD67
:10D74000F3DF7FFFFDFF2EFFFFFDFFFFDEFFF7BFD3
:10D75000F77EEFBD77DF7BEFBDF7FFBFFEFDFFFE7E
:10D76000FF9F2FFEFFF777FFFDF7DF7FFFFDE77FCE
:10D77000D5FF7F7FFEFBDFD7CFFEF77FFFFDF7DF13
:10D780007FFFFDF7FFECFF7FBEFBFFF7EFEFFFFF33
:10D79000FDFFFFFFFFFFFFFFFB7FF3FFBFD9E79F09
:10D7A0007FE4F1E79FFFF9E79F7FFEF9E79FFFFB2B
:10D7B000FFF7EFFFFFFDF6FF7FFFFFFF7FFFFFE7B4
:10D7C000FF7FFFDFFDFFF7F7FFFFFBFDFDBFBEEFB4
:10D7D000BFBFFEFBEFBFBFFE0FFEFFFDFBFF7FFFE6
:10D7E000FDFFFFFFFFFFFFFFFFFFFFFFFF67FFFFE3
:10D7F000FFFDFFFF7FFEFFFFFFFFFFFFFFFFFFFFBC
:10D80000FFFF87FFFFFFFFFFDBEFBEFCE66FBEDD24
:10D81000F6DB6FBFFDF6FF51FF7FF1D557477FFD68
:10D82000C5155B7DD5D5575B7DF5D5BF66FFCFFBB5
:10D83000FFFFB3C7DCFFFCCF3FFFFCF3CD3FFFFF93
:10D840007FE7FFFAFFFF7FFFF3FBFFBFFFFBFFFF59
:10D850007FDFFFFFFD9FBBFFFBFFFFFFF6DFBDAFDD
:10D86000DFFA69A79FFEFAE9F7FF1FFCDFF7FFFF6A
:10D870005BFBFFF5D755FDF5D75F3BFDF597FF4FF8
:10D88000FEFFFFFFBFFFFFF7F7FFFFFFFFFFFFDF19
:10D89000FFFFFFFE3FFFFFFFFD7FFF7F7FFDB763C1
:10D8A000FFFDF7DF7FFFFDF7FFBBFF7FBFE7F7FF60
:10D8B000C7BFFD7E6BBEFFF67B6FBF7FFEFFD3FF52
:10D8C000FFDFFCFFFFF77FCEFFFFFDFF7FFFFFFFC6
:10D8D000FFFFFFABFFFFAFFEF3FFFFFF3FFEA28F97
:10D8E0003BEAB8E38F2FFE7FF5FFFFFFFFBFF7DFB7
:10D8F000FFBF7DFBEFBFFFFEEF6EBFFFFFF8FFFB3B
:10D900002FFDF7DFFFEFBD5FFBAFBFFEFEFBEFBFFD
:10D91000FF3FF8FFFDFFFBFFBFF7F7DFFFEDF7DF8E
:10D920007FFFFDF7DFFFD7FEBFFEFEFFFFFFFBBA65
:10D93000DFFEFDF7DF7FFFFDF7DFFF4FFDFFCF3F8E
:10D94000F7F4EBFC3FCFFCACFFFFFFF3FFBFFEFFA4
:10D95000AED5FFF3CF3CFBF53FCF7FFEE7FFFFFFE8
:10D96000F5FFCFFFAFD5EBD4EB6EBBE77FF9E73325
:10D970003FF3CE9B6FFEF3E6FBF7EC7FEB7DD75CCE
:10D9800073FFFFE7FFFF7FFFCD3FFFFFF3FDAFF228
:10D990003FFEFD6A2B6FFFB2FFBCCFBAEBBEB3EE0A
:10D9A0003AEBAE5FF95EEF7FE79DF7EFD9F7CB7FFC
:10D9B000FDF5CB5F7FFDF5D73BFC7FFDFFF576FBEB
:10D9C0003FFEEDFB9EFBEFBFAFFE7BEEEBF7F6BF3E
:10D9D000FEFEEFBFBFFFF7DFDB5DF7DF7FF3FD3755
:10D9E000DFFF5BFCFFFFEF3DFFFCF7DB777FE79D91
:10D9F00077DF79E79D77FE1BFDFFFFFF3FFFBCF35D
:10DA00007FFFFDF7DFFFFDFDF7DF7FFF9AFFDB5FA5
:10DA10002FBDF4DF6FBEFBBEEDB6FB6EBBEDB6DB1C
:10DA20007F6CFFFCE79F74D2FFFEDB3FFDF3CF6FFF
:10DA3000BFFDF3DBFFEFF47FFFFDF7DEFBFFFF7DB4
:10DA4000F777DF7DDF7D77DF77FFBFFBFFFBEFFF42
:10DA5000FF7FFACF7F7FF7DF7FFFFDF7DF7FFEBF1E
:10DA6000FD7FF9C57FFF7DF9FF7FFFF7DF7BFFFDBE
:10DA7000F7DF7FFF6FFEFFFE7BEBAFFFFFFBFFDFFC
:10DA8000FFFFFFFFFF7FFFBFFF0FFF5F1F5D74D230
:10DA9000E91F7FFEF99F7FFEF9E79F7FFEF9BFFF39
:10DAA000BFFFECFAEB7FFEFEF77FFFFDF7DFFFFF26
:10DAB000FDF7FFCDFFD75F5CD554FBFFFFEBBFFE4B
:10DAC000FAEBAFFFFEFAEBFFC9DFEFBFFF1F7FFCF2
:10DAD000FFFFFFFDFFFFFFFFFFFFFFFF7FF1FFF5F0
:10DAE00097FDF7DFEFFFFFFFFFFFFFFFFFFFFFFFE8
:10DAF000FFFFFBFFEFCF3F3DFDF6FA5FFF72CB2F3D
:10DB0000BFF8F2CB2FFFDFFDFF975E7FBDF1575FC0
:10DB10007F25D75D75DD75D75D75FD1FFEFFFFFFA6
:10DB2000FFFF3EEFFDCFFFFCF3CF3FFFFCF3FFFF16
:10DB300047FEEFF7DFFFBBF4BFFFDFFFFFFFFFFF95
:10DB4000FFFFFFFFFFADEFFFFFF7FFFEF7DFBBFAC1
:10DB5000A9BEFEFA6BAFBFFEFFFFC4F9FF5F6FBE49
:10DB6000F7DFDF7EFCD75F7FFDF5575F7FFDDF844A
:10DB7000FFFFAFFDFFBFF7BFB6FFE79F7FFEF9E7EF
:10DB80009F7EFEBFE5BF7FFF7D7FFFFFDF7D77B715
:10DB9000DF7FFFDD77DF7FFDDFF2FFFFFF6FFFE756
:10DBA000FFFB57FFED77DF7DFFFDF75FFFA7FCEF82
:10DBB000FFDFF9FFFFFFEDFFDBBFFFFBFBFFBFFF59
:10DBC000FFFDEFF8FFDFDFDF87FFFFFEF32FFFBC76
:10DBD000F3CE3BFFBCFFFF1FFBFFFDBFFFBFFF6F8F
:10DBE000BFEFF7FCF3EF3FFFFCFBDFFF97FFBFDF6B
:10DBF000FFF7FFA7FF7E799577DEF9E79F7FFEFBB2
:10DC0000BF1FFFFFEFEDF3DF5F1FFFFCCB2DFFF426
:10DC1000F3CF3FFFFCFFE3FFFBFFFEFBBFAFFE7F49
:10DC2000FFF7DF7FFFFDF7DF7FFF7DC4FFFFFCFF16
:10DC3000FCFFFF3C3FFFF2CA39CF38F3CF2BFFAFD9
:10DC400058FFFEFFDFBEF73CFFFFFF7FFEFCD79FC4
:10DC5000FFFFFCFF29BDCFBFF4DFD32FFF5DBEEB7D
:10DC60009B6FBEEBE69B6FBE7F0FF6B79FFAFFACD4
:10DC7000B79F7EFFFDDF77DF7DF7DD7FDFFF1AFFD8
:10DC8000577FFD75FB67AF7DCFE99C7BEEB8E39EC8
:10DC900033EEFBB9FD2F9BFA6EB9E2DEFAFFFCCF43
:10DCA0003FFFFFFFCFFFFFBE96FFFF5F7FFDFDF74A
:10DCB00057FB3EEBB1DFBE7BEEB7E7BE7EECFFFB72
:10DCC000AFBFFFFAFBAFFFBDDF75FF9D37DF7FF30F
:10DCD000FD3FF1FF7FFFF9E7DFFFFF79F777DF7D9A
:10DCE000DFFD77DF7FF7FFF9FF6FBDF9FF7FFFFFF4
:10DCF000FF477FFCF1FFFF7FFCFFD75FE8FFD1F616
:10DD0000DF6ABFFDF7BAEFBBEEBAEFAEBBEEBAF714
:10DD1000C7F6FFBFFFFDFFCFFFFFFDF37FFFFDF362
:10DD2000DF7FFFFDFF76FFFFFF77FFFFF7FFBFF706
:10DD30007DEFBDF7DD7BEFBDF7FFB7FEAFFFFFFA6D
:10DD4000EDA7FFFEE777FEF9E79F7FFEF9E7FFD734
:10DD5000FF16FF7DF9ED9F7FFEF77FFFFDF7DF7F69
:10DD6000FFFDF7DFE5FFEFFFDFDFFAEBBFFFFDDDD4
:10DD70007FFF7DF7DF77FFFBBFF4FFF5F9E6279D17
:10DD800076DAE99FFFF9E79F7FFEF9E79FFFFBFF48
:10DD9000FBEFBFF3CC3BCB7CFFF7DF7FFEFDF7DF74
:10DDA0007FFF17FD7BF5DDF7CFBEFFE4FBBEEFBFC6
:10DDB000FFFEFBEFBFFFFE1FFEBFFEFFEFF3CF3EF8
:10DDC000FFDCFFFDF7FF7FFFFDF7DFFF2FFFFFFF0A
:10DDD000FF7DBFFDEFBBFFFFFFFFFFFFFFFFFFFF6B
:10DDE000FF83FFFFFFFFCFD36D3FFDF66FBFFDF653
:10DDF000DB6FBFDDF6FF5DFF7FFDF1D75F6DDDE51A
:10DE0000955B65F5D5565F75F5D5BFEDFF7FF5FEE2
:10DE1000FCFDFBFEFF7CCF3FFF7FF3CF3FFFFC7796
:10DE2000E5FFDFFDCFDFF7FFFB4BFFFDD7FB7FFDFE
:10DE3000FC93DFFF5FFAAFFFFFDBFEEFDFFFFFFFCB
:10DE4000FBFFFFFF77FBFFBFFBBFFD67F9F6D7DFE7
:10DE50007FFDF1D65FFDF5D75F7FFDF5D7FF0FFEA4
:10DE6000BFFE7DEB7F9EFEFDFFDFFFFFFFFFFFFF9D
:10DE7000FF7FFF5FFFF7FB9FF7FFFFFFFF7773FF5A
:10DE8000FDD75D7DFFF5B7FF87FEFFFBFFFE3FFF80
:10DE9000FDFF76E1BF7FFEF9EBBB7FFEFFCFBF7ECC
:10DEA000FF5BABFFFFFBEBFFFEFBFBBFFFFFFBFFDF
:10DEB000FFFF62FFFFFF5F7FF8BCF77EFBFCFF2BDD
:10DEC000EFBCF3FFE3FFFFF69FFFFE7FFFBDFFFF09
:10DED000FF7EFF7FFFFEFBEFFFFFFDBFBBFF9ACD85
:10DEE000BAD37E4FFD37FEFBED9F7FFEF9EFBFFFFC
:10DEF000BFD8FFFFBFFF3FFDBFE7DDFFFDF7DF7FBF
:10DF0000FFFDF7DFFF57FEFFFF7EFBDFFFFFFDDFBB
:10DF1000FFFDB7DF7FFFFDB7DFFE57FDFF67FBFDAE
:10DF2000BFFFFFFBC77AAF9DE7DF73AFBDF6FF967C
:10DF3000F5CF33F6F8F3CFFFFF6FFDE7CFFFFFFF1D
:10DF4000D7CFDFAFCB7BBE597FFDF7DFFEE73BBF0F
:10DF5000F3CA9B6FBEF3E7FBF76EFFB7ACBFFEFEE5
:10DF6000FBFFE7FBFF7FFFCD3FDFFFF3FDAFF0FFE0
:10DF7000A7B7CBFADDF6D2FFAECFBAEBBEB3EEBA9F
:10DF8000EBAE9FE87F52A9E6BE5BEEABFFD77FFD0D
:10DF9000F5CB5F7FFDF5D71BFCDFBF75F67FAFBD0F
:10DFA00075EEAB9EFBEABBAFFEFBEFEB47FEFF8DD2
:10DFB000F29BEF978F3ADFF55D77DF7BF3FDF7DFBD
:10DFC000FF60FEFFFEFF7FFEF9FF9F777EE71D7774
:10DFD000DF79E79D77FE1FFFFFF6DFFFFFFFFFFF03
:10DFE0007FF7F7DFFFFDFDF7DF7FFF88FF5B679FB0
:10DFF000FDF6DF6FBFDBBEEDB6FB6EBBEDB6DB7FC4
:10E000006DFFFEF6DB6FFFFFF3DB3FFFF3CF6FBF6C
:10E01000FDF3DBFF6FF3FFFFFDFDEFFFFFFD7DF77E
:10E0200077DF7DDF7D77DF77FFBFF8FFE3BDFFFEA2
:10E03000FEFAEF7F7EE7DF7FFEF9E79F7FFEDFFCE2
:10E040007BF5FE5FFF7EF9EE7FFFF7DF7BEFFDF7ED
:10E05000DF7FFFCFFEF7FAFF5FFF9BFEBFBFDFFF53
:10E06000FFDF7EFFFDFFBFFF2FFF7F9F7B7EFC5307
:10E07000D71FFFF99E7FFEF9E79F7BFEF9AFFFBF39
:10E08000FFFFF7DE7BEEADF77FFFF9F7DF7FFFFDE8
:10E09000F7FF87BF57FFFFB7EEFAEDAFEBFBFEFBD5
:10E0A000EFBFFFFEFBEFFFCBFFEFBFFFADFFFE7B40
:10E0B000EFFFDFFFFFFDF7DF7FFFFDFF00FFF7FF53
:10E0C000FFE69B6FBEFBFFFFFFFFFFFFFFFFFFFFB2
:10E0D000BFFBFFF6D3EFFFFFFFFF2FF7F28B2DBF44
:10E0E000FCF2D34BFFDFF9DFC35D6FFDA5975F76D1
:10E0F0003DD75D77D575D75A6FFD6FF63FFFFFCEE1
:10E10000FEFF7F73CFFFFEB3EEBFFFFEFBEFFF37D7
:10E11000F6EFBFFFF4FBFB7FFDF36EDFBFF7DB7FA6
:10E12000FFFDB7FFA9FEFDFFFFFFFDF7DDFF7FFF4E
:10E13000BFFEBF7FFFFFFFFFFF80FF7F1F6DFBE57F
:10E14000C67A7FFDD15F7FFDF5D77BFEDDFFEA7FDD
:10E15000FFDFEFFEFAFADE7FDEE79D7FEEF9E7DF15
:10E160007EFFBFE1FFFFFFFFF5DFFFFF7D7757DF9A
:10E170007DFFDD77DF7EFB57F9F7DF7F7BFFFDDF7C
:10E18000DFEFBEF6F9EFBFFFF6FBEFFA8FDDFF6FB3
:10E19000FFFFFEEBAFBFFAFFFFBFFFFFFFBFFFFFB9
:10E1A000FF0FFEFFEFFFFDFAFEEFBFF30DEB3CF3B9
:10E1B000CF3BFFFCFFFF5FF7FFDFEFFEF8FFFFFF46
:10E1C0004FE7FEFBEFBFFFFCF3BFBFB7FFFFEFFF63
:10E1D000FFDFF7FFFFD99F535E79E79D77DEFBFFF7
:10E1E000C1FFBFFFFFEFFFFFEFBFDDDF7BFFBDF72D
:10E1F000DF7BFFFDDFEBFFFFFFFF7FFFFFF7FFFD93
:10E20000DF77FFDDF7DF7FFFFD7DC7FFFDFFF3CF8A
:10E21000EFFFF27EE4771E6BFC3D77DE6BFF6F5BFA
:10E22000FFFFFFCC33FF7CF97F7F3FDFF9FC9F7F4F
:10E23000FDFCFDCABC7F9FF5B6DB6EBB67BEF99BDC
:10E240006FBEF3E69B6FBE7FBFF6FFCF7ACD35D7AB
:10E250005E73BFDDDF6FDFFFF7DD7FDFFD56BF5F82
:10E26000ABFF37DB6C297FEFF99C7BEE3AE39E73C3
:10E27000EFF999FDAFDEFB5E79EF9DFFFFFCCF3F2D
:10E28000FFFDFFCF5FFFB69DFF57567FFFFDF76293
:10E29000FF6EEBB1DF7EFBEAB1E7BE78E3FFEBAFE9
:10E2A000FFFEFBEFB5FFDDDF75FFFD37DF75F3FD2B
:10E2B000FEF5FF7FFFDF73CF3DFF7CD777DF7DFF6C
:10E2C000FD77DF6DF79EE8FF7FFDFFF3CF3FBFFCDB
:10E2D000477FFCF1E7FF7FFCFDD777F9FFDDF5D342
:10E2E0005F7FFDF5BAEBBBEEBAEFAEBB6EBAE79758
:10E2F000F6FFFFBE492F9DF4D2FDF77FFFFDF3DF50
:10E300007FFFFDF32EFFFFFF7FEFBFF7FEBBF77E22
:10E31000EFBD77DF7BEFBD77FFBFFEAFFFDF7FFF96
:10E32000FFFFFFE777FEF9E79F7FFEF9E7FFCDFFED
:10E3300017FBEFF7DF7FFFF5F77FFFFDF7DF7BFFD1
:10E34000FDF7FFE6FFEBFFBFCE7AEBADDFFDDF7F32
:10E35000FFEDF7DF7FFFFB3FF0FFF5F947477D75E6
:10E36000D4F19FFFF9E79F7FFEF9E79FFFF9FFF7E1
:10E37000DFAFAFBEFAEA7B7EFFFF7FFEFDE7FD7FEA
:10E38000FF7FFDFBF7FFD74E3BEDB4FBBFFFFFFF69
:10E39000FFFFFFFFFFFFAFFEBFFCF7FFF8EF8F3F70
:10E3A000BEFFFBEFBF7FFEFBEF9FFF77FF5FFFFB33
:10E3B0007FFEF9E79FFFFFFFFBFFFFFFEFFFFFFF80
:10E3C000A3FB6FFFFFF7D37FBFBDE22FBEFCF2CBF5
:10E3D0002FBFFCF4FF48FE7FFDF5D75D7EF965D7C2
:10E3E00073DD74D75D77CDF5D6FFE17F83BFBFEBDB
:10E3F000EFBBCFFEFCFF3DFADCFBFFFDEFFE7FE64F
:10E40000FFFCFFFFDFFFFFFBCFFF7FCE6FDFFFFED5
:10E410003FFFFF5FFBFF7DF7FDDF7FFFFD3EEDFF71
:10E42000FDEFF7F6FFFFBFF7DFFC7FDCD7DF7FEC08
:10E43000F9B5D31BFDF5D35F7FB9B5DFFF87FABF11
:10E44000FF5EFFFFEFFFF6E77FBE79E79F7FFEE904
:10E45000F6FF2FFF7FFEDDF557DEF7DF7677EBED7A
:10E4600077DF7DFFEDF7FB95F78F3FFCFF7FFFFF29
:10E47000FFEEEDBF7FFEDBEFBFFFBEFFC3FFFFFF81
:10E48000FFE36FFFFCDFAFFFEFEFFFFFFFFFFFFFDB
:10E49000FFE7FFFFFE3FFEDFFF7F3BFFF2CF3BEDDD
:10E4A000BCF3CB3FFF7FF2FFDFFF7FFF7F7FFFF7F4
:10E4B00076943F5F7BB575BFFBFE7F9AFEFB7F7F47
:10E4C000FFFEF7ED1FFFFBC7B7FF7EFBE79EFFAF29
:10E4D000F9FEF46FFF2CDFF7D5DFEFDDB7DF7FEB61
:10E4E000EDB75FFDFFAE7FEFFFFFBDFFFFFEDFFF7C
:10E4F000FDF7DF7FFFF5F7DFFF5FFCFFE79FC5FF5D
:10E500005FAFF7C32AFEB0E2CF33AEBDF6FFA4F58E
:10E510009FD75FE8FFEFF3FF2FFFFF9BFFFFFFD7C2
:10E52000CFFFAFD9FBDFFF638DFFF759E43BBFF3AC
:10E53000CEFB6FBEF3CEFBF768FFEFFFA7FEFFFB3E
:10E54000AFE6FBBFFFFEDD2FDFFFE7FD6FF6FFFF4E
:10E55000D75FAEFFBDFFFFAEEFBAEB9EBBEE3AEB6F
:10E56000AE77EAFEEFABAFFE5EEEBFFF577FFDF585
:10E57000CF5F7FFDF5D7DBFCFFBFF4F7FF2EF7F58C
:10E58000EFF99EFBEEB0AFFE7BEEABCDF2FFFFFAF4
:10E59000CBFFB3FFFADFDDDD77DE75D7DD37DFFFD9
:10E5A00026FFF9FFFFFFFFF9E7FF777CC71D77DF45
:10E5B00079C79D77FE82FFFDFFFFFFDFF9F7FB7F45
:10E5C000F7F7DF7FFCFDF7DF7FFF95FFDD7FBFFD06
:10E5D000F6DF77BFDBBEEDB6FB6EBBEDF6DB7F652E
:10E5E000FFFFFFDB6FFFFFFFD93FFFF3CF6FBFFDE3
:10E5F000F3FFFFEFF2FFFFFFFDDFFFFF7F7DF77609
:10E60000DF7DEF7D77DF7FFF7FFBF7FFFFFFDEFF23
:10E61000FA6F77FEE79F77FEF9E79F7FDEB7FDFF92
:10E62000FBFFFFFF7EF9C77FBFF7DE7EFFFDF7DF51
:10E630007FFFEFFED7FFFFDFFFDFF7FBBFF7FDEF49
:10E64000DF7FFF6DFFBFFF3FFEFF9F7F76F8E58F07
:10E650005DFEF99F7FFEF9E79F7BFEF9A7FF6FFE46
:10E66000FFFF9F2FFFE6F7FFFFFDF79F7FFFFDF7FF
:10E67000EF85BFF7FFFFFF7ED36FBFF37BFFFCF794
:10E68000DF7FFFFCF3FFC0FFFBFFFF8FFFDEB9EF73
:10E69000FFFFFFFFFDFFDFFFFFFFFFC4FFEDBFFF39
:10E6A00086197ED8E1FFFFFFFFFEFFFFFFFFFF7F20
:10E6B000FBFFF2FF4DFFBCF7FF6FFF76DB6FBFFD87
:10E6C000EFBFFFFF4FD87FD75F3DFDF1D75F5CBD48
:10E6D00055575D75D5C75F3FFDCFF6DFBFBF87F9E3
:10E6E0009FFDE3CFF7FEB7CF7FEFFCFFFFFF5FFE9D
:10E6F000FFBFFF36FBBBDBDF7AFFB6DE77EB7DFFCC
:10E70000FFFFFF9DF2F7CFD7FEFFFFBFF67BB3FF02
:10E71000FFDE7FE3FFEFFF7C81FFD7FF7EFCB1FCD4
:10E72000FF6CE995537AF9E5975F7EFD7BECFFE797
:10E73000FFFF7BBFFDF7EB7F7FF7F77FFFFFAFBFEB
:10E74000BE7DE1FF7FFF5D7FFF77CE7F7777DB7D4B
:10E75000FBDD77DF75F7DFF8D7FFDF6FF3FB7ED9DF
:10E76000EFBFF6F9EFBFFDFEDBEF77DBFCDFFFFF6E
:10E77000FFFFFFE7FDFFEAB7FFFAFFEFFFFFFDBE78
:10E780005FFEFFEFFFB3FE79CFBFF33E7FBCF3CE5A
:10E790003BEBFCEBDF37FDFEFFEFFBFFBEFFFFFBBC
:10E7A000BFFFFEFB6FBFFFFEFFEFBBFFFBFFEFF9FD
:10E7B000EDBDDBEEB99F5FFEF9679777DEFBFFD516
:10E7C000FFFFFFFFFDF1DFBFBFFDDE7FFFBDF7DF16
:10E7D0007FFFFD3FA9FFFFFFFEFD7FDDFFFFFD5D2A
:10E7E0007FFFFDF7DF7FFF7D7FB1F7EEF77FFFFD56
:10E7F000DBCFFFFDD54FFF7FFFFD6F3EFEBF78B73C
:10E80000F5BFEFFEFBFDB75FFEFFD77F7FF9F7D7C0
:10E810007F7B3FF5FFFF7F1EF9CCF1EF8FBF38E321
:10E820008A33CE38E7DAFF3BD6FFFF7FBEF9FFFD24
:10E830007CFDFF9F7FFEF5E7CF3FFFBF7EEFFFFF31
:10E840003FEF7FF97E9DEFFAE69B6FBEF9E69BEF07
:10E85000DFB3FDFFFF9FF7FFFDB2DE77FEF6DB774C
:10E86000DF7DF7DD37BF977FFBFFFFBBEEBD4F9F1F
:10E87000FBBEE79E7BEEB8E7DEFB7AA9FBFDFFFF60
:10E880005FEFFFA2CA3FFDF3CF3FFFFFFBD7BF6F94
:10E89000F77FFFFFBFEBEF3BD6B8CF7BECB38FBE6C
:10E8A000FAEAABAF1FF8FFFFFF7FE3FD77E97C4794
:10E8B00037DF7BFFCDF7DF7FFFFFF8FFFFFFDFF9DB
:10E8C000FFDD7FDFFDDD77DF7DFFDD77DBFD07FE31
:10E8D000F7FFFFFFFDF77FFFFDD11F7FFCF1FF5F1B
:10E8E0007FFFF577FE7DFFFD6FDBE8AEBDEEFBAE93
:10E8F000BBEEBAEB8E9BEEFD95FDFFFFFFFFFCF735
:10E90000DF7FFFFEDF7FFFFDF7DF7FFFBFCBFFFF76
:10E91000FFFFDDFFDEF7EFFDDB7BEFBDF7DE7BEF1B
:10E92000FDFFECFFFFFFFF79FB9FB7FFF99F7FFE25
:10E93000F9E79D7FF6F97FF2FFFFFFFFFDFFDFBFE5
:10E94000FFFDDE7FFFFDF7DF7FFFFD7FF8FFFFFFAD
:10E950007FFFFFEFFF7FFFF7DF7FFBFDF7DDFFFEB0
:10E96000FFFCFF7FFEF9E39F3FFEF8E11F7EF9E326
:10E970008F5FFEF9E5DFFEFFFFFF9FFDFFDFFBDF9F
:10E98000FFFFFFDF7FFFFDF7DFFE47FEFFFFFFDF3B
:10E99000FBFFBDFFDEEBBDF7DE7BEFFDF7CFFF2713
:10E9A000FFF7FFFFFFFFFFFFDF37FEE3AF77DE7903
:10E9B000EBBDFFFE17FFFFFFFFFFFEFFEFAE3FFEC9
:10E9C000E18F1F7EF9F5D77BFFE8FFFFFF3FFDFFDB
:10E9D000D3FDBDF51B6FBEFDF6D75F3FFD7FE1FFA9
:10E9E0005F7FBDB5D35B7E79C5465F7DB5D55F7F63
:10E9F000ADF57BF9FFFFFF3FFFFCFBBD37FFF3CF1A
:10EA00003EFFFCF3CDFBFF3AF9FFFFEFF7DDBFFF61
:10EA10005FEFEC72E3EBBF3FFDBBFFFB57DAFFFF9D
:10EA2000F7EFDF5FFFFFF7EFEEFF77DDF5FFFDFFAD
:10EA3000FE3FFEF7FF7FE6917BDBBFF5566FBDE53E
:10EA4000D75D7FFCF7DFABFDFFFFFBFDD7DFFFBF2F
:10EA5000FFF7EFFF7FFEFFB7BFFDDF8CFF7FFFE714
:10EA6000F5F7DFFDF7DDDD7DF7DD77DF7DF7ED7FA6
:10EA7000E6FFDF7BAB3DF0FBEFB7FFF86FB7FDF6CE
:10EA8000DB6FB3FF3F716BFFFFFFFDFFDFF6FFEBB7
:10EA9000BFFFFFFFBFFF7FFFEFE7F8EFFEFFDFFFE6
:10EAA000EFF4FFCC7EFCF2C63BFBFCF3CFFFAFDD07
:10EAB0007EFFFFBFFFFFDEDFEFFDFEDB6FBFFFFE70
:10EAC000FBEFFF8FFEFFBFFFEFF57E7EFFE5777A5E
:10EAD000F9C59C5B5EF9A7FF5FFFFFFFFFF7FF7EB5
:10EAE00073F5377EFFF5F7DE7EF3EDF7FF97FFFF57
:10EAF000FFFFB7FF7DFFFF777DFFFDB7DF7DFFFDE8
:10EB0000F7F74FFFFFFFE7B1FE1CDFE4999F79E6BF
:10EB100031E79C73AEF9BF4CF5FFFFD7CD5EBE8FDA
:10EB2000FEFFFFFFF35BFFFFFCF3FFABF4FAFFFF19
:10EB3000F3CE9FEFF7F9CEEFBCF3CE3BEFBCF3E69D
:10EB40003DDAFFFFFFF9E6DFFFFBF9FEEFBF7FFFD6
:10EB50009D77DE79FF9BF9B7FFFFBFEB9EF3F4BF14
:10EB6000EFFBEEBAEBAEBBEEBAEBF7B6DBFFFFFFA7
:10EB7000F5CF2FEAFFFBBF7FFDF5D75F7FFDF506E1
:10EB8000FEFFFFFFFBFEB72FADFBBEAFBEFAEABB39
:10EB9000FFBEFBFFA5FFFFFFFF77FE7FBFBEF7763F
:10EBA000FFFD77DF79F78D77FD8FFFFFFFFF1D7F7B
:10EBB000DFFDFFDDDF7DE71D77DC71E79D7FE5FF92
:10EBC000FFFFFFDFFFFDF7FF5FFDF5F7DF7FFFFDD5
:10EBD000F7DFFFE7FFF7DFFFF6ADEEDAEF9EEFB905
:10EBE000EDB6DB6FBFFDF6DFD9FFFFFFFFDF7FFF75
:10EBF000FFF6CFFFFCF3CFFFFFFFFFFF1BFCFFFF84
:10EC0000FFDFFDEFFD7FDFBDDD77DF7DFFFDF7DFA0
:10EC1000FF8FFEFFFFFF9F3FFFF9FF9FFFF9E79F79
:10EC20007FDEF9679DFF67FFFBFFFFDFB3FFFDF9A5
:10EC3000DFEFFDF7DF7FFFFDF7DFFF2FFFFFFFFFB8
:10EC4000FFFF7FDF7FF77FFFFD77DD7FFFFD77FF32
:10EC5000D8FFFFE79F3BFEF9638F1FFEE3971F7E00
:10EC6000F8E5975FFEE1FFDFFFFF59FBFF75DE7FF1
:10EC7000FFF7DF69F7DD7FFFFD7FF2FFEFFFFF3D6D
:10EC8000FFDFFBEB9DDE79E79D77DE7DF7DDBFFBE8
:10EC9000FFFFFFFFFFFFFFFFFFE37FFEFAE78DB7F8
:10ECA000DE7AEBFFFDFFFBFFFFFFFEFFEFFEFD9FA8
:10ECB0007FFEFBF6FF6FBFFFFFEEFFFFFFD34F3E70
:10ECC000FDFFD33FFDF4D34F3EFDF4D3FF27FDFFFF
:10ECD000F5575F6FFDF1D75FEFF5475F7FBDF1D669
:10ECE0005AFFB2FDFFEFFFF1BF9FFFFDD11F77FD80
:10ECF000D5D73DDFBFFFFF83FFFDEF3FBF7FBBCF1A
:10ED0000BFFED7ADFFEE7CD3FFDFBF7FEBFEFFFF83
:10ED1000FDFE7FEFFF7CFF7CF7DFFFDFFFF5FFFFEE
:10ED2000FFB1FFFFBF1FFEFFF197137FF0811B7F35
:10ED3000FCE19F67FF77F8BFFFFEFBFFFF3FEBFEA5
:10ED4000F5FFFFFFEF7BFFF7DCFF9FFDFFDFAFD796
:10ED50003F7FF5FFD715DD75D75A575DF7DFFDEF1C
:10ED6000FEFDFFFF7BAFBDDF7FDBAFEDF6FB6DBFD1
:10ED7000BDFEBAFF47FFFFFFFFFFFFFFFF7F9FFFC3
:10ED8000FFAFFFFFEFFFFF7F7FBFEFFFFFFFFCF74E
:10ED9000CD3DEFBC463FEFFCF3CB3FDBF8FF45FF3B
:10EDA000FFFFFFBEFBEFFDFEBE6DBFFFFEFBEFB33F
:10EDB000FFFEFFE5FFFEFF7FFEFBE7977DFEE79787
:10EDC00047FAF9E71FFBFEFFE6DFFFFF7FFFF5F7DE
:10EDD000CF7FFBF7DD7FB3EDB7DE7FDD1FF8EDEF13
:10EDE000FF7F3FFFF7EF7FDF77DF7FDFFDF79F7F5D
:10EDF000FF7FF5FFFFFF1CFFCE3D6F1EB3F0438E7C
:10EE000033CEFCC7DCFF3BDAFFFF1FBF8FFF9F3F06
:10EE1000FFFF9F3FFFF5F3CFFFFFBF46EFFF673DCB
:10EE2000EFDFF9FE9FCFFAE4932FBEF9E6937FDE82
:10EE3000B3FDFFA79EF7EBFDFFDF7FFFF7DB77DF7B
:10EE40007DF7DDFFBF8BFFFBFFFFBBF43DEFDE7304
:10EE50003EE79E7BEEBDE7DEFB7EA37FFCFFFE5F11
:10EE6000EAFF7BFF3FFDF3CF3F7FFDFBD7BF6FF096
:10EE7000FFFFD7BF6BBDFABEBBCFFBEDB6CFFEFB2E
:10EE8000EEBBAF1FFBFFFFEB7FAFFEF7DE7947F76F
:10EE9000DF7DEFFD77DC78FFB3F8B7FFFFDFF9B771
:10EEA000DD7FDCFDDD77DD7DB7DD77DBFDA7FEE710
:10EEB000FFFFFFFDF75F77FED11F7FFCF1F75F7F5C
:10EEC000FFF51FFE7FFFFD6FDBE39EB9EEFBAEBBE0
:10EED000EEBAE98E9BEE7DB1FFFFFFFFBFFFF7CFDC
:10EEE0007FFFFCDF7FFFFDF7DF7FFFBFCBFFFFFF73
:10EEF000FFFDFFDEF7EF7DDB7BEFBDF7DE7BEFFD98
:10EF0000FFC9FFFFAFFFF9FF9FB7FEF99F77FEF93B
:10EF1000E79F7FFEF97FC2FDFF97FFFDF9DFBEFF90
:10EF2000FDDE7FFFFDF7DF7EFFFD7FF8FFFFE97F5E
:10EF3000FFFFF7DF7EFFF7DF7FFFFDF7DDFFFEBEA0
:10EF400070FF7FF4F9E39F3FFEF8E33FFEF9E38FA4
:10EF50005F7EF9E79FFEFFFFFF9F75FF5FFFDDF715
:10EF60007DE7DD77DFE9E7FFFF0FFEFFFFFFDF9BB8
:10EF7000FFBDFFDEE99D77DE79E7DD77DFFD03FF8B
:10EF8000FFFFFFFFFFFFFFDF777EE7BF77DEF9EFD1
:10EF9000AFFFFE01FCFFFFFFFFEFFFFFEE9FFFFD56
:10EFA000E7DF7FBEFFF6DFFFE6FFFFFBBFFCF38B73
:10EFB000FFBFFCDB6FBFFDF6D34F3FFD7FE5FB5F7F
:10EFC0007ED9F5D74D7DD9D5465B7DF5915B6FBD7B
:10EFD000F5AFF8EFFFFFBFFFFFFFFF3AFBF3CF37BF
:10EFE000F7FCEFFFFBDF3FF9FFFFFFFFEFBFFFFF86
:10EFF000B56DDF6DF7CDE7FFFFBBFFD7FEF7FFCFA6
:10F00000EFFFFFFFDFF54577F3F7DAFFFF7FFFFF45
:10F010005EDCFD7EFCF5FF5FFFB9F5577E3DF5D761
:10F020005FEEF9F7FF9BEFFFBFFFF9FF9F6FFFF95F
:10F03000FEEEFFFFFEFF7FFFDDFF91FFFF77B7FDD5
:10F04000FFDFF1F7DDDD7BF75D779F7EF7E5FFE022
:10F05000FBFF4FBEEF76FBFFB7FFD8EDBFFDBEFB5A
:10F06000EFBFFF7F73FFFFDFFF5FFFFFFAFFFB7F55
:10F07000FFFAFFFFDFFFFFFF3FFAF7FFFFCFDF7F62
:10F08000BEFFCC7ADCF3CE0F7BBCF0CFFFFFDDFF01
:10F09000FFFFEDFF7DFFFFEFFFF6FBEDBFEFBEFBD8
:10F0A000EBFFFFFEFFFFFFE7F7DB6EFFE77E7EB9BA
:10F0B000E79F5FFAF9E77B6FFBFFFFF7B7177FFF6B
:10F0C000F7B76ECDFDD7DD76FFFDF7BFB5FDFFFFCE
:10F0D000EFF77F7FFFFF777FFFFDF7DF7FFFFDF714
:10F0E0007F15FFFFFFE4FDED1CD3E7B91E73CE3D96
:10F0F000F79C7FE6F93F66FDFFFFFEFF7BDE8FF3A7
:10F100005FBFF5FF5F3FFFFCD7FFEBF7FEFFFFF2AE
:10F110004E9D7FF6F9CEEFBCF3CE3BEFBCF3FEBDC8
:10F12000D8FFFFFF79A7DE7FEB79FFF7DF7FFF9D39
:10F1300077DEF9FE1BFCFFFFF5BF4BDF7BF4BFEF73
:10F14000FBEEBAEBAEBBEEBAEB1FB6FFFFEAFFA5D4
:10F15000FEBF6AFDFBBF7FFDF5D75F7FFDF54EFE6D
:10F16000FF7FEDFBD7AB67FFFBBFFFEEFBEFBFFF02
:10F17000FEFBEE85FFFFBFFEF7EB7C97FE7777F790
:10F180005DF7DF7FF3CDF7FED3FFFFFFFF9D7FDB52
:10F19000FDB75DDF75E79D77DE79E79DFFE07FFFD7
:10F1A000FFFFDF7FFFF5F75FFDF5F7DF7FFFFDF77F
:10F1B000DFFFE27FF7DFFFF63DEED8ED9EEFB9ED22
:10F1C000B6DB6FBFFDB61FDAFFFFFFFFFF7FFFFD5E
:10F1D000F6CFFFFCF3CFFFFFFFFFDBDBFDFFFFFF01
:10F1E000DFFFEFBD7FDFFDDD77DF7DFFFDF7DFFBBD
:10F1F0002FFAFFFFFF9FF7FFF9FF9FDFF9E79F77E8
:10F20000DEF9E79FFF05FFFFFFFFDFBFFFBDFBDE6E
:10F21000EFFDF7DF7FFFFDF7DEFF837FFFFFFFF7E7
:10F22000EFFEB6FFF77FFFFDF7DF7FDFFDF7FFD1D2
:10F23000FFFFE79F3FFEF9638F3FFEE5875FFEF824
:10F24000E7975FFEECFFFFFFFF5DFFFFF5DF7D9FB0
:10F2500077DB7DF7DD7FFFFFFFF3FFFFFFFFBDFFE4
:10F26000DFFBEF9DDE79E79D77DE7DF7DDFFF8FFC1
:10F27000FFFF7FFFFEFFFF7DE7BFDE79EB9DF7DE3F
:10F28000FAEBBFFCF7FFFFFFFFFFFFEFFEFDBFEF55
:10F29000FEF9E6DFFFFFFF0FFCFFFFFFCBFFBFFC28
:10F2A000F3CBBFFCF2CB2F3FFD74D3FF3BFFFFF549
:10F2B000D75D7DDDB5935DCF75535D76B5F5D65BD6
:10F2C000FFAFFFFFFFFCF3FFFFF7EFF33DEFF9FBAD
:10F2D000EFBFF7BEF7FF95FFFF5FBFFCDEFBFF3F11
:10F2E0009FCFCDFEFFFEFBEFFFFE7EE3FFFFFFFFA4
:10F2F000FFBFFFFF7DFFDEFEF3F6FBEFBFFFF7FF73
:10F30000E6FDFFFF5FFFFFF5575B6FF5D75F6F7D92
:10F31000C59F7DFF9FFAFEFFFF9BEFEFF9DA9A6F23
:10F32000B9E69E5FFEF9F6DAEF7FF9FFDFEFDFFD6A
:10F33000FFFDFFDFFDF5F7DF7DF7FDF7DFFF57BED0
:10F34000FFFFFFFBFFBDD7DEDBAFFFDEDB6FBFFFE5
:10F35000FEFAFE57FFFFFFFFFFFBEB7D777FFFAB62
:10F36000FFFFFFEDE7FFFFFF877FFEFFFFFDBFCF42
:10F37000FB7FF4C33FDFBCF3CB3FFFDCDFD1BFFF3C
:10F38000FFFFFDFFEFF7FFFBB8FFF6BBEFBFFFFA94
:10F390007BFFCEFFFFFFFDFC57E7FF5DFEE79F7F92
:10F3A000EEF9E59F7FFE3DF1FFFFFF7FFBF7B7D74B
:10F3B0007DFFF6DD7DBBEDB7DD7F7F3FF9FFFFFF12
:10F3C00077FFFFF7FF7FFFF7DF7FDFF9F75F7F7FD3
:10F3D000DFF5FFFF7F9E5FCCF14D1EEB31E79A6BAF
:10F3E000CEF9C79AFF9BD6FFFF7FFD8FFE9D387F2A
:10F3F000F55B7F7DFCF35F3F7FBF46EFFFFF3FFF85
:10F40000F2F96695CFFAE69B6FBEF9E693EFDABBA9
:10F41000FDFFFF9F7FEBFDB6DE7F7FF7DD77DF7DB2
:10F42000F7DF77BF95FFFAFFFF3B74B965DF73BE67
:10F43000E78E7BEFBDE7DC7B7E6D7FFDFFFF5FEA44
:10F44000FFBFFE3FFFF3DF5F7FFDFBD7BF6FE2FF34
:10F45000FFFFBF6FFF7BD6BFCFFBEDB1FFBEFBEF62
:10F46000B9E7DFD8FFFFFF7FAFFE77E9754737DFEA
:10F4700075D79D37DF7CF79B71B7FFFFDFF9E79DFD
:10F48000FFDFFDDDF7DF6D97DD77DBF575FEE7FF6D
:10F49000FFFFFDFFFFFFFFD11F7FFEFDF75F7FFF37
:10F4A000F577FE7FFFFD6FDBEBAEBDEEFBAEBB6E17
:10F4B000BAE98E9BEEFDA5FDFFFFFFFFFCF7DF7FA6
:10F4C000FFFCDF7FFFFDF7DF7FFFBFC9FFFFFFFF0F
:10F4D0007DFFDEFBEF7DDB7BEFBDF7DE7BEFFDFF2E
:10F4E000E7FFFFFFFF79FF9FFFFFF99F7FFEF9E72F
:10F4F0009F7FFEF97FF0FFFFFFFFFDFBDFBBFFFDFE
:10F50000DE7FFFFDF7DF7FFFFDFFF8FFFFFFFF9FBF
:10F51000FFEFFD7FFFF7DF7FFFFDF7DF7FFF9FFC42
:10F52000FF7FFEB9639F3FFEF8E11F7EF8E5875F2E
:10F530007EF9E53FFEFFFFFF9FFDFFDFE7DFFFD91D
:10F54000F7DF7FFFFDF7DFFF47FFFFFFFFDFFBFF79
:10F550003DBFDEEBBDF7DE7BEFFDF7DFFF9BFFF787
:10F56000FFFFFFFFFFFFFF37FEEB8DB7DE78EBAD50
:10F57000B7FED0FFFFFFFFFFFEFFCFAE5FFEE797B6
:10F580003FFEF8F7DF7FFFC3FFFFFD7FFDF6D76F7C
:10F590007FF5D75F7FFDF5D75F36FDFFF6DF5F7F35
:10F5A000FDF5D65E6FFDF45E7DFDD5535F7DBDE557
:10F5B0007FDBFFFFFFFF9FFEF3F97BDFF3DFB5F794
:10F5C000FDFBDFBBFFFFF8FFFFFFFD7FFCBEFFF38E
:10F5D0007BF9DDFFCEFFFFDCFBFB87FEFFBFFFFFFC
:10F5E000FF5B7FD7FFEFFFFFF5FF7F7FFFF7BC7566
:10F5F000FEFFFF5FF1FE1FFF3BD11577FCB1831FBC
:10F600007E7CF7FF8BFFFFFFBFFEFFEFEF7FEEE794
:10F61000AFFFFEFBE69FEFFDFF9BFFFFFFFE7DA719
:10F62000DFFFF79D1D7BEFDDF7DD77FF5DFEE5FF7B
:10F63000FFFFBFAFFEFB7FBFFFDAEFBDFDDEDBEB01
:10F64000BF7B7F77FFFFFFFFEFBFFFFAFFEBDFFF1F
:10F65000FFBFEFFFFFFFFB7FF8FFFFFFCF1F7DBF67
:10F66000FF8F7B7FE1862FFBBCFECFFF7FFDF7FF87
:10F67000FFB77BFFEF7FEFD7DFFBEFBBFFFEFFD7CF
:10F68000FFCFFCFFFFFFEF97F7F67AEDDEF6BBEF5B
:10F690009E5FFEFBEFFF4FFFFFFFFFF7DF7FFFF7F0
:10F6A000F76FEFED97DF7FEDFDF7FF85FEF7FFFFCB
:10F6B000F75F7FF7F7F77FFFFDF7DF7DFFFDF77758
:10F6C0001FFFFFFFFF3FFFFCFFFF9BBFF3FEBBEEF3
:10F6D000BCEBA8FBBF6FFDFFFFFFCF7FFECFF3CFDB
:10F6E000FFF5FFCF3FFFF5F3FF2BF3FEFFFFF3E73F
:10F6F0009FEFDFF9CFEFBCEBE63BEF7CF3E63DDBC2
:10F70000FFFFFFF9F3DFFFFBF9FFF7DF7FF39D77E3
:10F71000FE79FFDBFCFFFFFFBFEB8ED3F6BBEFBB39
:10F72000EEBAEFAEBBEEBAEB67F6FFFFFFFFF5D721
:10F73000FFEEFEF25F7FFDF2D75F7FFDF55EFEFF1D
:10F74000FFFFFBEEBFEFBDBBAEEFFE7BEEBFEF9E5C
:10F75000FBFEBDFFFFFFFFF7DE7FA78F777EE75D34
:10F7600077DD7CE7FD77FEC1FFFFFFFF9D77DEF1D0
:10F77000F75DDB71E7DD77DE71E71D7FE7FFFFFFF8
:10F78000FFDF7FFFFFDF7FFFFDF77F7FFFFDF7DFFD
:10F79000FFE6FFF7DFFFB69BEEDFEFBE2FBBFCBE41
:10F7A000DB6FBFFDF69FD8FFFFFFFFDB7FFFFDF69E
:10F7B000CFFFFCF7DBFFFFFFFFFF5BFCFFFFFFDF7F
:10F7C00077EFBD7FDFFDDD77DF77FFFDF7DFFF4FF1
:10F7D000FAFFFFFFDF7FFFFDFBDFDFFDF7DF77FED7
:10F7E000F9F79FFF2FFFFFFFFFDF7FFFFDFBDFFF2D
:10F7F000FDF7DF7EFFFDF7DFFF83FFFFFFFFFFFF6A
:10F80000FFDFFFFFF7FFFFFFDF7FFF7FF7FFD8FF7F
:10F81000FFE79F3FFEF9E38F7FFEE78F1F7EF9E54D
:10F82000975FFEE1FFFFFFFF59FFFF75DE7FDF7788
:10F83000DF7DF7DD7FFAFDFFF6FFFFFFFFBBEFBFC8
:10F84000FBEB9BAFB9E69A6FBEFDF6DB3FF97FFF9E
:10F85000FFFFFFFFFFFFFFEFFFFEF9E3ADB7FE7B0A
:10F86000EB3FFDFFFFFFFFFFFFFFEFFEF99F7FFF75
:10F87000FBEEFFFFFFFF9FFEFFFFFFD75F7FF9FF5C
:10F88000577FFDF5D75F3FDDE4D3FF1FFDFFE59711
:10F890005F7EFDF5D75FFDF5975F7FADF5D64BFF3A
:10F8A000BAFFFFFFFFF3CF37DFFF333FFFFCF3CF9C
:10F8B0003FFFBEF3FF87FFFBFFBF7FFFFFFFB6FFEA
:10F8C000FFFFEFEFF6DFFFFFFD7FE9FFFFFF3FFFE9
:10F8D000DCF3FF3FFFF2CF3DDFBEFAB79FFBFFF047
:10F8E000FFFFFF1F7FFCF1DF1B7FE1871B7DFCE734
:10F8F0009F7DFFFFF9BFFFFFEFBFFBFE7EEB7FFEAB
:10F900007AEFB79FBDF7DBFD7FFDEFDFFFDFEDFE99
:10F91000DDD59FDBE9B7DF7FFFBDD7DFFF9FFEFFB0
:10F92000FFDFF7EF77FFF7F74FFFFDD7DF3FEFFC84
:10F93000F3FF77FFFFFFFFFFF2F7E7BBBFF7FBFF28
:10F94000FFFFDE7FF7FDFFBBFFFFFFFFFFFF8FDF46
:10F95000FF3CC73BEFBCF38FFBF7FDFFCBFFFFFF87
:10F96000F7FFDFBFFFFFFBB9FFFEFBEFBFFFEFFBC2
:10F97000FFE2FFFEFFFFFCFFEFF557FEE79F7FEE84
:10F98000B9E9AFBFDEFFE4FFFFFF3F77F5F2FF37D6
:10F99000FFF3CF3FFFFCFFFFFFFF5DFBFFFFFFDF3C
:10F9A000FFF77DFFDF7B7DF7DF7FFFFFFFFFFFFFBF
:10F9B000F4FFFFFF2ADFFFFAEFACB93AEBAFABCEB3
:10F9C000FAEBAAFFBBD6FFFF7FFD8FFF5F5FFDFC59
:10F9D00057DFFFFCF3573FFFBF6EEFFFFF9FCFD214
:10F9E000F9AE9FEFFAAE9BEFBAEBAE9BEFDFABFD4C
:10F9F000FFFFCF7FEBFDA7DF777FF7DD77DF7DF7B9
:10FA0000DD77BF9DF7FBFFFF33F43DEB9F7BBAE74C
:10FA1000DE3BEEBDE7DE7BFCAAFBFEFFFF5FEAFFFD
:10FA2000FFCA3FFFF3DBFF7FFDFBD7BF6FF4FFFF94
:10FA3000FFBFEFFDFBFEB9CFFAEDABEF9E7BEEAB68
:10FA400067DED9FFFFFF7FE3FE77FC7DC7F7DF7C32
:10FA5000E75D77DD7D975FE8F7FFFFDFF9FFFDFFEB
:10FA6000DDBDDD77DB77B7DD77D9FD87FAD7FFFF1F
:10FA7000FFFDFFFF7FFFF11FFFFFFFF75F7FFFF538
:10FA80007BFE7DFFFD6EDBEBBE9DEEFBBEBBEEBBEA
:10FA9000ED9E9BEEFDB1FDFFFF6FFFFCF7EF7FFFDB
:10FAA000FCCF7FFFFCF3CF7FFFBFCBFFFFFFDF7DEE
:10FAB000FFDEFFEF7DDF77EF7DF7DD77EFFDFFEA1C
:10FAC000FFFFFFFFFDFFDFBFFFFDDF7FFFFDF7DF74
:10FAD0007FFFFDFFF4FFFFFFFFFDFBDFBBFFFDDF4F
:10FAE0007FFFFDF7DF7FFFFD3FF9FFFFFFFFFFFF18
:10FAF000FFFFFFFFFFFFFFFFFFFFFFFFFF9FFCFF79
:10FB00007FFEF9E38F3F7EF8E13FFEF8E1875FFE7D
:10FB1000F9659FDEFFFFFFFFE5D75DFFDDF77DF7AE
:10FB2000DD77D7FDE7DFFF77FEFFFFFFFFFBFFBEBF
:10FB30003FEEF99E7BEEB9E7DE7FEFFD0FFFFEFFA4
:10FB4000FFFFFBFFFFEF3FF6E79F3FFEFAEBBFBF74
:10FB5000FE0DFFFFFFFFEFFFFEFEEEAFFFFCF3AF7A
:10FB6000BFFFFEF3EFFFE8FFFFFFBFFDF6DAEFAFE9
:10FB7000FDD96FBFBDF6DB6FBFBD7FE3FB5F7E6D61
:10FB8000F5D657777DF5575F75F5D5575A7DB52F63
:10FB9000FAFFFFFF3DBFFF73FF3DDBF3CF39FFFCF3
:10FBA000FBEFBFFF5FF9F7FFFFFFFFFFFFFFFFFF67
:10FBB000FFFFFBFFFEFFDFBFFFA7BEFFFFFFF2FF60
:10FBC0003FBFFFF32B6FFCF3CFF7BEFBEDF70FFC4E
:10FBD000EFFFFFF5FB5E7FFDE5567FFDC5D65F7E3F
:10FBE000FDD57F8BFFFFFFFFFFFFFFDFEEFFF6F787
:10FBF000FFBFFFFFFFF7FFFF8DFFFBFFFDFC7F7FD8
:10FC0000DFFFEBF97FFFF77FFFFFDFFFFFE5FFFF80
:10FC1000FFFFBFF7FFFFFFDFFECBFFFFFEFFEFFFA2
:10FC2000BF7FF2FFFFFFFFFFBFDFFDFFFFFFDFFF33
:10FC30007FEFFFDFFEFFFEF9FFFFFFFFFFFFFFFF8C
:10FC4000FD737FFFFFF7DF7F7FFF7F7FDCFFFFFF1D
:10FC5000FFFFFFFFFF79CFFFFFFFFFFFFFFFFFBFAA
:10FC60003EFEFFFFFFFFBFD7DFDFFFFEDFFAFFFF34
:10FC7000F7DFDFFFDF1FFB7FFFFFFFC7FFFFFFFF98
:10FC8000EFCBEDBFDDFFFBFFFFF785FFBFFFFFFF02
:10FC9000FFFEDFDFDFFF59DFFFEFFEFBDFFFF7CB0C
:10FCA000FCBF7FF6F9E79D7F9EF91E7FFEF9E79F77
:10FCB0007FFAF93FECFFD77FFB6FF5CF7FEFB9DD20
:10FCC00077DFFDF7DE7FFFF5DF73BF77DF6FFFFDC7
:10FCD000F6DD3EFFF4D75E7FFDF1C35FFFBFF8F7AF
:10FCE000DFFDF5FDFFF7FEFFFFFFFFFFFFFFFFFD5D
:10FCF000FFFF5BFCFFFDF7DF7BFFFDF7DFFFF4F3AA
:10FD0000CF3F3FFDF3CFFE4FFE3DFFFCF3CF3FBFA4
:10FD1000FCF11FFFFCF3CF3FFFFCF3FF4FFFDF7F42
:10FD2000FFEDF7D67FFFFBBFFFFEFBEFBFFFF6FB4C
:10FD3000FF9FFFDF7EFAF9A79F7EFAE9977EFAE937
:10FD4000A79F7EFAE9FFD9FFEFBFFBFFFBFFFBFF99
:10FD5000FFFFFDFFE7DFEEBFFDFEFFE1FDDDFFBFC3
:10FD6000FFFFFBEFBF7BFBE7BFFFFEFFFFFFFF7F58
:10FD7000F3FEFBFFFFFFFAFFFFFF7F7F7FFFDFFB4D
:10FD8000FBFFFDFF3FFAFFFFF5C7FFBFFDB7CFBE8B
:10FD9000FDF3D77F7FFFF3CFFF3FBCFFFBEDBFFF3E
:10FDA000FEFBEBBFFFFBEFBBFFFEFBEFBFFFBFDECA
:10FDB000DBFFFEFFFD2FFFFFFF37FFFEF3CFFFFF4F
:10FDC000FFFBFF2FFFFFFEFFFFFEFFFFFFFFF7DF41
:10FDD000FFFFFFFFFF7FFBFFA7FFFFFFFFFFFDFF11
:10FDE000FFFFFFFBFFFFFFFFFFFFBFFCDFDDFFFFAC
:10FDF000FFFFFFFFFFBFFFFFFFFFFFFFFFFFFFFF53
:10FE0000FFFBEDFFFFFFFBFFBFFDFFFFFFFFFBFF62
:10FE1000EFFFFFFEFFFF7DF4FFFFFFFFFFFFFFFF90
:10FE2000FF7FFFFFFFFFFFFFFFFFFF7EF8FFFFFFEA
:10FE3000FFFFFFFFFBFFBFFFFFFFFFFFFFFFFFFF16
:10FE40001FBCFFFEFFFFFFFFFFFDFFFFFFFFFFFFE8
:10FE5000FFFFFFFFFF8FFEFFDF7FFFFDF7DF7CFF70
:10FE6000FDDF7FFFFDF7DF7FFFFD7FFF3FFDFDB77C
:10FE7000CF7F7FFCF777FFFCF7CF7FFFFDF7F7839E
:10FE8000FF7FFEFFBFFFFFFF77DFFBFF7FFF7FF7F7
:10FE9000FF7FFFFFC7F77FDF7F6FDFF7FF5DFF7734
:10FEA000FF5DF7FFF5DF5FF7FFE0FF4ED75FC7FAB3
:10FEB0003DE7F77B7FA7F57F6AF7D7F57735F0FF4A
:020000021000EC
:10A00000FF04E8FAF9DAFF5E7DEFD7F55EFDEDF5C6
:10A010005E5EEFD5DF5E7DEFFD4FFFDF76FFEDF794
:10A02000DF76FF6DDFF6F76DF7DF76FFFFFD8BFF65
:10A03000FFFF77FFFFF7FFFFFFFFFF7FFFFFFFFF40
:10A0400077FFFFC3FF5E7EFFF5F75F7EFFE55F1ED4
:10A05000FFE5F75F7EFFFEFFE6FFF7F967DF7FF6BC
:10A06000F9779FF7C9679F7FF7F9273FFFF4FFFB59
:10A07000FABFFFFFFBFABFAFF9FA9FCFFFF9FC5F12
:10A08000BFBFE8FFFEFFEFFFFFFEFFEFFFFFFBFF9D
:10A09000FFFFFEFFFFFF1FFCFFBEFFEFFFFFBEFF46
:10A0A000EFDBBEFFEFF3FF3EFFDFFDDFFEFFFFFF55
:10A0B000FFFAEFFFBFFFE3BFFFFFF7FBFFFFFF7FED
:10A0C0004FFFBFFFFFFBFFB7FFFFFBFFFFFEFFFFE1
:10A0D000BFFFFFFFFF87FEFFFFFFFDFEFFFFFFFF4C
:10A0E000FEEFFFFFFFFFFFFFBFFFCFFFFFFFFFFF01
:10A0F000FFFFFFFFFFFDFFBFFFFFFFFFFFFFFFE0D1
:10A10000FFFFFFFFFFFFFFFFFFBFF7FFFFB7FFFFEF
:10A11000CFFFFFFF72FFEFBFFFFCFBAFBFFF7CEE87
:10A12000BFFFDEFBEFB7FFFE3FBAFFF7DF7FFFF5B4
:10A13000F7DF77EDF6DF7FFFFDF79F7FFFFFFD7F06
:10A14000BED9E39F7FFED9E74FC779E79F3FBE7D2A
:10A15000677F1F7EFF78F7CF7FFFF0F74DEFFCD7CB
:10A16000CF7FEDFCF7DFBF1FDF9D7FFE79E79D7F8F
:10A17000FEF99F7FFEF9E69F7FFEF9B58BFFFFE6B4
:10A18000FE7FEFFFE6FE6FFEE6FE6FEEFFE6FEBB34
:10A19000DDC3FFD7DF7FFFFDD7DF7FFDD5CF7FFD9D
:10A1A000FCD5CF7FFFFF63FFD96FFFBDD6DB6FBF4D
:10A1B000FDDA6FBEF5F75F6DB77DFF70FDBFFFFF86
:10A1C000DEFBDFFFFFFFFFFFFF7FFFFDFFFFFFF96C
:10A1D000F9FCFFFFB7CB6EFFFFF7FEFFFDFEBFDF11
:10A1E000FEFFFFFF9F7DFFF9FECFFFFFE99E9FACC3
:10A1F000F1FF9FBFFDF9FFFFFF7FFEFF77FFFEFF2F
:10A20000FBFFFFFF3FFFFFF3FBF37FFFFFFF2EDFAF
:10A21000FFFEFBEFBFFFFEF3EEBFFEFBEBBFFEFE5C
:10A22000FBEFFB83FF3FB7FDFFD2EFF5FFFEEFFD36
:10A23000FFF2FF2FFFFD7FDFDBFFFFDFDFFFFDFF13
:10A24000FFFFFEF7F7FF7FEFF2EFFFFFFFE8FFFFF3
:10A25000EFFFFFFFB7FFFFF7BDFF7FFFFFFEEFFF41
:10A26000BF7FF07FFFFFEFFFBFFFFFF7EFDFBFF71D
:10A27000FFFBFFFFFFFFFEFBFF7FFFFFDFFFFFFE98
:10A28000FF7DFFFDF7FFFFFFFFFFFF3FFD7FFDFFAE
:10A29000FFFF3EF9EF957FFDFFDFFF7FFDFFF7FF3B
:10A2A0008FFE7FFEFFFFFFFFFAFFDFFFF9FFF7FFE3
:10A2B000FFFDFFDFFE47FFFFBFEFFFFF1DFB9FF529
:10A2C000DFFFFDFFFEDDFFFF7FFF97FFFEFFFFF7D4
:10A2D000DFAFF67DFF66BFDEFFFFFFFFFFFFFFD7AB
:10A2E000FFFFFFDFFFDF7FFFFFFB77FBFEFFFFFFCF
:10A2F000FBFFFFFFEFFFFFFFFFFFFFBFFFFFFFBF02
:10A30000FFFFFFFFFFFFFBFF7FF0FFFFFFFBFDFFF6
:10A310003FFFFFFFFFFFFEFDEFFFFFFFFF3FF8BF27
:10A32000BFFF7FFFDFEABF7F7DBAFFBEFEFFEFFF0B
:10A33000FFFF7FFDFFFFFFFF7FBF9D7FFFEFF9F76F
:10A34000EFFFFFFFFFFFF34FFEFFF3FFFFDDFFFE19
:10A35000FFFFDF7EFBFFFFFFFFFFFFFD17FCEBAF03
:10A36000F3FFFFEBFDEFDFFFE793BFFFFFFFFFFF13
:10A37000FF9AF5FFF3FFFFFFEC7FFFFEFFF35FFFA8
:10A38000FFFFFFFFFFAFD9FBFFFFFD3FFD7F5FFF3B
:10A3900097DFFFF9FFFFFFFFFFBFF668FFFFFFFF3B
:10A3A000DFFEFBE9BFFFFBFFFFFFFFFFFFFFDFEF6C
:10A3B000F2FFFFFFFFDFFDB7DF6DAF3DD3FFFBFF18
:10A3C000FFFFFFDF9FE8FFFFFFFFFFFE9AFDAFDB10
:10A3D0005BA9FFFFFFFFFFFFFFFBFDFFFFBFFF5F6D
:10A3E000E7FD75DE7FBDB57FFFFFFFFFFFFFF7FED7
:10A3F000FFFFFFFFAFB5F65E6BBF86FAFFFFFFFF03
:10A40000FFFFFF0FFFEDFFFF7FFBF7FF5F7FFEFF0B
:10A41000FFEFFFFFFFFFFFFF99FFF9FFFF7FBEFD8B
:10A42000FF7B6FFEF7FFE7FFFFFFFFFFFF87FFDA0E
:10A430007FFFFD77DA6BBFFDDF7DFFF1F7DF7FFF89
:10A44000FD7E6FFFFDFFDFFFFFFDFFDBFFFFFFFF77
:10A45000FFFFFFFFFF6F6FF5DFFFFFFBFF7FFFFFDA
:10A46000F7FFFFFFFFFFFFFFFFFFDFBFF97FFBFFEE
:10A47000FFBFF6DB6FAFF5DAED3FFEFFFFFFFFFF3B
:10A48000BFFC6FFBFF575F65F75D577DF5E71FFF6B
:10A49000FFFFFFFFFF0FFEFFFEFFEFFFFFDE7BFB77
:10A4A000FFFEBB2FFFFFFFFFFFFF47FFDF9F7FF692
:10A4B000F9C71F7FF6799F7D36F9E79F7FFEF98701
:10A4C000FFBFFFFDFBEFBFBFFEFBFFFFFCBBFFFFBE
:10A4D000FFFFFFFF87EFF7FFFFFDF7DF5F7FFFFB6A
:10A4E0007FFF7DFFFFFFFFFFFFA0F7EF7FFFFEFB7A
:10A4F000EFFFFFFFEF3FFFFEFFFFFFFFFFFF11FF3B
:10A50000EDBF7FFBEDB7FFFEFBB79F7FF3FFFFFFC4
:10A51000FFFFBFFBEFFFFFFFBFF4FECAEF7FFFFFB0
:10A52000FFFFFFFFFFFFFF9DFCFF575F7FAD74172D
:10A530005B6FF5D71F7CFDD5D75F7FFD3FF6FFFF33
:10A54000F3FFFFFEFF7FFDFFEFF3BFFDFFFFFFFF08
:10A55000FF27FEFF7F79FFFDEFDFFFEFFDFFFCFF31
:10A56000FFFFFFBFFFEF85FFFFFFFFFF7FFBDD77F3
:10A57000FFF5EDF7FFFEFFFFEF7F7F927FFFFF7F8D
:10A58000F1ED97DB7FFD81EBFEFBEFBBFFFFFF678C
:10A59000E5FFFFFEFFF5F7EF7FFFEEFEFFFFFFFF9A
:10A5A000FFFFFF7B3FE3FE7FFF1FF7FFF47FDF7EB0
:10A5B000FCDD3FFFFF7FFF7FFBFFB8F7FFDF6FFF93
:10A5C000FDDEDFEFBFF7FBAFFDFFF7BF8FFB9FFCAB
:10A5D000FBFFFF5DFFFFF9FFDFDEBFC7FEFEFFBF32
:10A5E000FFFFFB3EFEFFFFFFFFF7FFEFFFFFCFFD8B
:10A5F000FFF3FFFFFFFFFFFF3FFFFFFF7FFFFFFFB7
:10A60000BFFFFFE4FFFFF8FFFFFFFFFFBFAFFFFB50
:10A61000FFFEFFDFA7FFFFF32FF7DEFBDFFFFFFFEC
:10A62000FFFF86FFFF5FBFFBFFDE7FFFADDF7FFF2A
:10A63000FDFEFFFFFFFFFFE0FFFFEFFEFFFFEFB7B5
:10A64000BF76F5CF3EDFFFFDFFFFFF7FC4FFFFFFBB
:10A65000FFFFBFDEF7DFFDFF74DFFFF3FFFFFFFE4D
:10A660000F58FFFFFFBF3FCFFFFBFFFF7DFACFE596
:10A67000FBFFFFFFBF5ABCFFFFFFFC537FB7F6771E
:10A680006BFDDFD2FFFFFFFFFF5F3FF6FFFF3FFFE6
:10A69000FDF7FEFEFFB9DFFFEBFFFFFFFFFFFF1E31
:10A6A000FFFFFFFFFFDD647BAFB47F13EF35FBFFE0
:10A6B000FFFFF5FFA7FDFFFFFFAF79E5BD67DEFDFB
:10A6C0009DF7EAFDFFFFFFEAB789FFFFFFFFFFF5F8
:10A6D000D77E677DD7537F6DFFFFFB7FAD7EE3FFA6
:10A6E000FFFFFFFFFF6BEFB5F77BA1BDFAFFFFF99F
:10A6F000BFCE7FF2DDFFFFFFFFFF7FFBF7FFFFFF16
:10A70000EDE6FFFFFDFDFF3FF95FFFFFFFFFFF7F6E
:10A71000FFFFFFFFFF7FFEFFEFFFF1FF9FF8DFFD71
:10A72000F7DF7EFF7DF6DFFFFDF69F6FFFFDF7DFB2
:10A73000FF57F6FFFFFFFFF7FF6FFFFDFF6FFFFF04
:10A74000F6FFFFFFFFFF76FFFFFFFFFFFDFFF77F35
:10A75000FFFFEFFFDFFDFFFDFFFFFF9BFEFFFFFEA3
:10A760007FFBADBDF65BBFBDF6F2EFFFBFFEFA7F2C
:10A77000C7FFFF7FFEF7D757DFFDF7777F3DF1ED8E
:10A780007F5F7EF9FFE9FFFFBFFFFFBEEFAFFBFE7C
:10A79000EFBFBF76FBFFFFBFFEFFF0FFFFD9E79FD4
:10A7A0007DF6F1E79FFDF9471B7FBEF94797DFF97B
:10A7B000FFFFEFAFFFFEFFEFBFFFFBEB2FFFFEE75B
:10A7C000EBFFFB7FFCF7FFF7D7DFFFFFFFFFBFFDCE
:10A7D000F797DFFFFFF5FFF7AFFEFFFFFBEBBFFFD4
:10A7E000FEFBEFFFFEFBEFBFFFFFFFFFFF5FFFFF83
:10A7F000FFFDB5F77EFBEFBF7FFBEFB7B7FFFBFFBA
:10A80000FFFF27FDFFFFBFF69BFFBFFDF6273FF5CC
:10A81000FEFFFFFFFFEFFFC6FF7FF5F5575F7DFDF2
:10A82000F5D76FD5E5075F7CFDD5D7BFEFFFFFFFFD
:10A830003FFBBCFFCD3EFB7FFD7FF0D3BFF3FFFFAF
:10A84000FFE7FFFFFFEFF3FFFFFFF7DFFFFBD77F20
:10A85000FFFFBEFFFF97BBFFFFFFFFFFF7EF7DF797
:10A86000FFCF3FDF7DFFFFFFFEF67FF8DFFFFFDF5B
:10A870007F6FFDFDFF1DFFFEDFFFFFFFFF87F71B63
:10A88000FEFFFFFFFFFFFFBDFBFFEFEDFFFFFFDB65
:10A89000DFEFF7FF4FFEFDFFFB7DD7DFFFBFD3E705
:10A8A000CFDD7DFF3FFFEF7FFD8FFFFFFFFFFFF35A
:10A8B000FFFFF7DEFBBFD9F76B6EFFFFFAFDC3FFAB
:10A8C000FFFFFFFFF7FFFF7FB7FDDBEEF7FEF7FBB4
:10A8D000FFFFFFE4FFFFFFFEFFFFE3FEDFEFF0FF00
:10A8E000DBFFF8FF8FFEFB7EF6FFFFFFFFFFFFF7AA
:10A8F000FDF93FF4FFFFFFFBFFBFFFFF7FF2FFFF0C
:10A90000BFFBFF7FFFEFBFFBBBFEFEFFFFDFFFFFD5
:10A91000FEDFFDFFFFFFFFFFFFFFF5C77FFCBFD797
:10A92000F7DCFDFFDFFFA7FEFFFFFFFFFFFFFFFEDE
:10A93000FFF6FFCFFFFFFB7EFFEFFF0FFDFFCFFF17
:10A94000FFF7FF2EF3DFFFFF2FFD37DE7FFFFDDF79
:10A95000A2F5FFFFFFFFFBFFA7F77FFD3F5FFCD3E3
:10A96000CF3FFEFCBFC6FBFFFFFF3F7FD6DF2D378B
:10A97000B7594B9DF5D75E7F3DFF6FFFFFFFFFDFB0
:10A980007FEAEFE79EB7EDB7FE7AEAAFB3CE2DF7D9
:10A99000BBFEFFFF5FEFFFF77FFFAFD0443BDDB4AF
:10A9A000D25FFAFFE86FFFFFFFBFF7EFBBEFDB6F90
:10A9B000A9AF865AEAA92FDB3BFDFFFFFFFF5F67C8
:10A9C0009DFDD77FEF75D65F7F05F557FB67FEFFCF
:10A9D000FFFFFFAFB5FEFE6BFFD32AABAFBFDE3A82
:10A9E000CBF91FFEEDFFFFFFFFF1FFFF7FFBDFDB7A
:10A9F000EFFFFFD6FFEFFD2DFDFFFFFBFFFFF9FF90
:10AA0000FFEF7FFF19E7FF7DD6FB777F8CFFDF7FAE
:10AA1000FFFDF7DF7FBFFD9F6BBEE9771A7DAB7946
:10AA20007A6DFFFFFFFF7FFFFFFFDBFFFFF7EF7F89
:10AA3000FFFDFFDDBFEFF2FFFF7FFFDFFFFFFFFB4B
:10AA4000FFFF7DFFF5DFFF7FFDFF7EFAFFFFFFFFCA
:10AA5000BFF6FAEFBFFDE3CB2FFEDEE77F27FFFF58
:10AA6000FDFFFFDFFF5F7DF9E65EEDF1C512DBED77
:10AA7000F3DF57FFEFFEFFFFFFFFBFBFEEFBEFF778
:10AA80007C5A6BFFFFF3FF6BFF77FFFF9F6FFEF0BA
:10AA9000479F3DFC791F6DA4F9E69B7FF4F987FF82
:10AAA000FFFFFFFFF97FFF7EFBFFFFF8F3EF7FFF64
:10AAB000F1E2FF81EFFFFFFFFFF7BF7FFFFDFBDF4D
:10AAC0007FFDFDFFFF7FFDFFA0F7FFFFFFDFFFFF23
:10AAD000BFF7FEFFBFFFFCFFDBFFFFFEFFD4FFFE63
:10AAE000FFFEEFEFEFDFDFFBAFD77EFBEFBFFF5FD8
:10AAF000FBFFD8FFFFFFFFBFBDDFD3FF7FE49BFF5E
:10AB0000BFFCD7FFEFFF3FFCFE535F7DFDD5D75D58
:10AB10007D6DD75F7BBCB5D75F74FD2FFEDFBFEFC8
:10AB2000FFCFFEFBFF7FFFF3FCCFF5B2FCFFCFFDB5
:10AB300007FEFFFFFFFEFFEFFDFFFFEFFFCFB5FFBB
:10AB4000BDFFFFF4FB957FFFDFFFFF7DFFDFF3FF1E
:10AB5000FFD7BFFFFF3BFDFFFF7F98FFFFFFDCFB41
:10AB6000F1FEFFFFFFD15E6B7DFF5FF56DFF7FE8BC
:10AB7000DFFDFEDFFFDDFFFBED7FEE6FBFFEFFFBC6
:10AB8000FEFEFE7FE1FEFFCFFFE7FD7FDFFF6FBC34
:10AB9000FF3FFBBFF3FEFFFFBFB9FFFFCAFF3FF759
:10ABA000FED1FFAFFF6BEFFFF9FEFF7FFF3FFDFF21
:10ABB000EFFF7FDF7DFFF7FF9BAFBF5BFFFDFDBFBB
:10ABC000FCFFFF3E3BFFFFFFFFFDFFF8E2EF7B7C5A
:10ABD000F37F7FDFFFF3FF55BFDEFEDFFFFFF7DF11
:10ABE000DBF6F77FFDF5FF7FFDFFEDBFA7FB7FFFE6
:10ABF000FFFFEF3FFDF77FFFE7EEBBFFBFFFFEF775
:10AC0000FD8AFFFFEF7FEDFBCF5DFD8DFBB7F2FF10
:10AC1000F58D7EFFFFFFE2FEFFF7FFFFFF6FFF7F77
:10AC2000FFFFFFB6F7FFEFCFFCFF7FD6FFFFFFDF91
:10AC3000FFE7DF3CDFE5FFF7D9FFFFFD37D9FF4F27
:10AC400050FFDFFFEFE7FF2FD3EFF37FF1CCFFFFE4
:10AC5000FCB3ECFF9ABD67FDFFF2FF299FE71FF3EE
:10AC6000FB25D6FF2F3DF5F77FFFF6B79E7FFEFF52
:10AC7000A7FF6CB27F9B68EBFFA7CEFAFBFF2EFE0F
:10AC8000F77BBBFCD37FFBFDECFF322DB4FF5E2EC8
:10AC9000DDBCFF87FDF5FE6F7FA8BFBD1BF6FD96EF
:10ACA0007EEAFFAF9E5BEEBF97FF57FFFFEDF5D744
:10ACB0005FEF7DDF5B5DE5FFD6537FF77FE1FFEB65
:10ACC000FCFFC6DA6BEFA3FD3BA9BFFEEFCAA1BF35
:10ACD000FFEFE0FFEFFFFFFF9F7FBBF9F6FFBDFF38
:10ACE000FEFB6FFBEDB6F7FAFFE7BFFDE6FF7FFF68
:10ACF00079DEF7BF7DF6D9F7FF7DE69FF9FFF177A3
:10AD0000DF6FFFDDF69BEFE9F6197CB6F9F719FE68
:10AD100097F6FF7FFFFFFEFFEFBFFDF33FFFFCFF56
:10AD2000DB7FFFFCFF6EFFFFF7F7FFFFFFFF7F7F7B
:10AD3000FFDF7FFF7FF7EF7FFFFF97FF7FF6FCDFEF
:10AD4000FBAFFD7BC27FFEDBE2CB2F9EDE627FDBB3
:10AD5000FF7FFFEDD7DD57FF7FD51FFF75F1C4D70C
:10AD60005F3EF1DFCFFFDFFEBFFFFBFFFFB2FCFF67
:10AD7000FF91F49AA9AFB7F4BFF2FFBFF9479F7FE5
:10AD80007EF9479FE7B9461B6DF4D1459BFFF8FF5D
:10AD9000E7DFEFBFFFFBFFAFFFFFCFAFBFF8F2EB87
:10ADA000AFFF57FCFFFFFFD75FFF5DF7D7BFFDEF9A
:10ADB000D75F7FF9F5D5FFDFFEFFFFF7FFFFFFFE4F
:10ADC000FFEFFFFFFFEFBFFFFEBBEFFF1FFFFFFB2C
:10ADD000EFBFFF7EF3FBB57FFBEFB5DF5E7EFDB51A
:10ADE000FF9FFFFFBEDDF6FF7FFFF4EEF7FFF7CE1C
:10ADF000FF297FFDE6FF43FF7FF5F5965F7DFDD1DF
:10AE0000D23FEDF5571F2FFC35D7BFEEFFFF8FBEAA
:10AE1000FFFFCB7EF7ECCFBE76FFD7FF3FBF7FF7BC
:10AE2000A3EFFFFFEFFFFF7576AFDFF7FFFB3EFFFE
:10AE3000DFD7F7BFDFB877FFF7FDFDFDDF7FBFFF8F
:10AE4000DE97FFFFCFFF7FF9FE97FCF77FFDD75B13
:10AE5000FDFDE197DFFB65577F7FFFF1F7FF4FFEB9
:10AE6000FFFBB7EF7FBFF7FE6FCBFFF9DFEFFBBD57
:10AE7000FEDFFD67FFFDF777F1C7FFF77BFCF7C546
:10AE8000BDB1DFFFFFFFFFFEBFFF7FFEFFD67B7F71
:10AE9000FBFDF7F3FFD7FEFBFEFFFFFFFDC9FFFC45
:10AEA000FE7FF7F7FFFEEBFF7DFFFEFDED7FEEFB84
:10AEB000BFFFEABFE3FF3FFFF877EF7F7FF0F79731
:10AEC0007EFCFDFFFF7F7FF6FFF7FDDFFEFDFBF75A
:10AED0007F6FD5FFFF6FDEFFFFFDFFAFDBFFFF5F83
:10AEE0003CF3DF7BEDB6EB9F9EBFFB7EFBFFFDD708
:10AEF0007FF9EFFFFFEBFEFBFC83EFFFFDFFDD7F44
:10AF0000FFF9F7FA7F27FEFFFBBFFFFF7FFFDDFFA3
:10AF10007FFFEFEBAEBE7EFDFFF765FDFFE73FDD98
:10AF20007FFECFF3DDFFFBFFDFF7FFFF2FBDBFBAD3
:10AF3000D5FFF39FF8DFFF95F3FAF7F3CFF7F3CFE1
:10AF4000FF5FFEBFCAEBFFFFCFF7FDFFF97FB5BE86
:10AF5000FE4EBBF4DFFF4F9DF7E7FFFFFFF3CFFE91
:10AF6000F7DFB7FEF35FF3FDFEFBFFA7FE2FF7BD94
:10AF7000BEFF5EBAFDEFD7D7B78F97DE33C936FB7A
:10AF8000DEFBFFD9FEFFFFBFC5FAF7ABA67EBFC948
:10AF9000EFBE5C6EFDEFFEDBECFFF7FFFF5FFF9B9C
:10AFA000F5D6FFF7D5765FFDE55FD6FBE7FEFFFF41
:10AFB000EF5FAFFDFD7A6ABFCF72786FBFFF7FA9E9
:10AFC000F146FEFDFEFBFFFFFFE71B7FFEFEDF3EBF
:10AFD000BBF9FFDBEFE714FF75FEF97FFE7DFF9FF6
:10AFE0007F7EE6FBFFBFFFF75BE7F79E7F1F7FFEDD
:10AFF000FD769F6BBFED9E7FAFBDC6DB67F5B97A6F
:10B0000066FFFFFFDF3FFFFFF7DB6FFFFFDF7FAF75
:10B01000FDF6FFFF6DF3FFFF7FF7DFFFFFFDFBDFB7
:10B02000FFFFF7F77FFFFEFFFD3FF8FF67DFFFB68B
:10B03000FEF7BFBFDFE7EBBFBFFCFF9F2DFE5FFD4D
:10B04000FFF7DF7F5F7DFBFC57FF91457F5F6DF76B
:10B05000DF16FF4FFEFFFDDFDDBFF7DFAFFFFFF5C0
:10B060005AFFAFF9F78B6BFF27FFFF9B7FFEF1E7DE
